:020000040800F2
:10000000703700201705000885040008090900085A
:10001000890400088B0400088D040008000000001B
:100020000000000000000000000000008F04000835
:1000300091040008000000009304000895040008E3
:1000400097040008990400089B0400089D04000818
:100050009F040008A1040008A3040008A5040008E8
:10006000A7040008A9040008AB040008AD040008B8
:10007000AF040008B1040008B3040008B504000888
:10008000B7040008B9040008BB040008BD04000858
:10009000BF040008C1040008C3040008C504000828
:1000A000C7040008C9040008CB040008CD040008F8
:1000B000CF040008D1040008D3040008D5040008C8
:1000C000D7040008D9040008DB040008DD04000898
:1000D000DF040008E1040008E3040008E504000868
:1000E000E7040008E9040008EB040008ED04000838
:1000F000EF040008F1040008000000000000000008
:100100000000000000000000F3040008F5040008EF
:100110000000000000000000F7040008F9040008D7
:10012000FB040008FD040008FF04000801050008A6
:100130000305000805050008070500080905000873
:100140000B05000800000000000000000000000097
:10015000000000000000000000000000000000009F
:1001600000000000000000000D0500080F05000859
:100170001105000800000000130500080000000041
:08018000000000001505000855
:10020000DECEA5ED02003078463337320000000024
:1002100000000000000044523234305F3135303786
:100220000000000000004170706C69636174696FC8
:100230006E00000000000000000000000000000050
:100240000000000000000408FE00DAF7DECEA5ED95
:100250000200307846333732000000000000000012
:10026000000053504C6174436F6E74726F6C6C6518
:1002700072004170706C69636174696F6E00000098
:10028000000000000000000000000000000000006E
:0802900000000000FE00DAF797
:100298007105000818000000A90700080300000005
:1002A800E50D000806000000E9100008090000003C
:1002B8001D16000802000000F916000810000000D2
:1002C800B5180008FF000000691E00080C000000B7
:1002D8008121000800000000B52200080500000088
:1002E8006137000812000000893A00080A0000007F
:1002F8003D3D00080A0000005945000814000000B0
:10030800E549000808000000FD500008070000004B
:10031800A5570008100000008D5B000813000000BE
:100328002D6D00081300000005E700081600000006
:1003380021F1000817000000BD2001081600000088
:10034800E5210108170000007132010815000000BE
:100358002F49072291438D462E492F480A1A06D065
:100368000722914381F30988022282F314882B48DB
:100378002B492C4A00F039F82B482C492C4A00F01C
:1003880034F82C482C492D4A00F02FF82C482D49D8
:100398002D4A00F02AF82D482D492E4A00F025F85C
:1003A8002D482E492E4A00F020F82E482E490022CA
:1003B80000F026F82D482E49091A082903DB0022E7
:1003C8000260043001601F481F49884205D0026856
:1003D800043003B4904703BCF7E700208646EC4698
:1003E80000200021234A9047FEE7884207D0521A8E
:1003F80005D0037801300B700131013AF9D170470B
:10040800884202D002700130FAE770471A487047F4
:1004180070370020703F002070370020709101086D
:1004280088010020F0010020700500087005000810
:1004380020640108D8910108703F0020703F002017
:1004480070050008700500087005000870050008B0
:100458007005000870050008206401082064010880
:1004680070910108F001002024340020703400202D
:100478007034002069270008FFFFFFFFFEE7FEE752
:10048800FEE7FEE7FEE7FEE7FEE7FEE7FEE7FEE73C
:10049800FEE7FEE7FEE7FEE7FEE7FEE7FEE7FEE72C
:1004A800FEE7FEE7FEE7FEE7FEE7FEE7FEE7FEE71C
:1004B800FEE7FEE7FEE7FEE7FEE7FEE7FEE7FEE70C
:1004C800FEE7FEE7FEE7FEE7FEE7FEE7FEE7FEE7FC
:1004D800FEE7FEE7FEE7FEE7FEE7FEE7FEE7FEE7EC
:1004E800FEE7FEE7FEE7FEE7FEE7FEE7FEE7FEE7DC
:1004F800FEE7FEE7FEE7FEE7FEE7FEE7FEE7FEE7CC
:10050800FEE7FEE7FEE7FEE7FEE7FEE7FEE7134845
:10051800854600F022F84EF68850CEF200000168B9
:1005280051F47001016000BF00BF00BFF1EE100A76
:1005380050F04070E1EE100A4FF0000080F314888C
:100548004EF63C71CEF20001086850F04070086029
:10055800034804490160FFF7FBBE70470080002094
:0805680008ED00E000000008AE
:1005700000B583B04FF0010003F06CFA4FF00300B8
:100580004FF0000140F2F952C0F6000202F032FCD6
:100590004FF0010040F20961C0F6000140F2E9525B
:1005A000C0F6000202F026FC4FF008004FF00901EF
:1005B00002460EF0DFFC4FF0070300934FF00003FC
:1005C000019318464EF68531C3F6D16141F6B86203
:1005D000C3F6856210F0D0FE46F24040C0F601003E
:1005E00005F060FD03B000BD08B519B94FF0030078
:1005F00012F008FE08BD00BF08B5012903D14FF075
:10060000010012F0FFFD08BD08B54FF00A0000F030
:10061000FBFD08BD08B501464FF00B0000F0F4FDEE
:1006200008BD00BF46F25C43C0F601031A684EF6EF
:100630000C50CEF200000260FEE700BF08B5FFF7E5
:10064000F1FF00BF51E8002FBFF35F8F41E80003C7
:10065000012B3FF4F7AF1046704700BF13461A4610
:100660002DE9F00F092AC0F00980B1E8F80FA0E8E1
:10067000F80FA2F10902092ABFF4F7AF4FF00C03FB
:1006800003FB02F21D4B1A44974600F032B800BF3C
:1006900000BF00BF00BF0B68036000F02AB800BFB6
:1006A00000BF91E8180080E8180000F022B891E837
:1006B000380080E8380000F01CB891E8780080E845
:1006C000780000F016B891E8F80080E8F80000F033
:1006D00010B891E8F80180E8F80100F00AB891E854
:1006E000F80380E8F80300F004B891E8F80780E820
:1006F000F807BDE8F00F7047134600008A060008AF
:1007000013461A462DE9F00F0B460C460D460E46D1
:100710000F46884689468A468B46092AC0F00780DC
:10072000A0E8F80FA2F10902092ABFF4F9AF4FF0CF
:10073000080303FB02F2144B1A44974600F020B85A
:1007400000BF00BF046000F01BB800BF80E83000AD
:1007500000F016B880E8700000F012B880E8F000F1
:1007600000F00EB880E8F00100F00AB880E8F0036D
:1007700000F006B880E8F00700F002B880E8F00F5B
:10078000BDE8F00F704713463C070008EFF31180F7
:100790004FF0800181F3118870474FF0000000BFD7
:1007A00080F31188704700BF30B440F20003C0F6F8
:1007B000000340F28812C0F60002D01A4FEAA001EE
:1007C000B1F5C47F04D81346264A9A4201D324E0E7
:1007D000FEE7254D254C601B20F003054FF000037C
:1007E00040F20002C2F2000240F20001C0F6000135
:1007F00005F10400C5F380045D589D5003F1040326
:10080000834226D109E05C589C5003F104035C58F4
:10081000D45003F104038342F5D14EF60853CEF2CF
:10082000000340F20002C2F200021A604FF0B5016C
:10083000CBF26B1143F27040C2F2000001604EF641
:100840001453CEF200031A6842F01001196030BC54
:100850007047002CD7D05C589C5003F104038342AE
:10086000D1D1DAE700000008040000088B0100087D
:1008700030B4034600283FD002F1100440F20000DB
:10088000C2F2000040F82430002A0ADA12F10C0FFC
:1008900036DB02F10C024EF61850CEF20000115475
:1008A0002EE04EF20015CEF200054CB211EA2404FF
:1008B00038BF80244EF20041CEF20001545413465A
:1008C000002AB8BF02F11F034FEA631005EB800155
:1008D0004FF01F03C8F200031340002B05DA03F1A9
:1008E000FF3262F01F0303F1010358B24FF001021F
:1008F00002FA00F30B6003E0002AC7DB014DD4E7E6
:1009000030BC704780E100E01EF0040F0CBFEFF335
:100910000880EFF3098020E9F00F00F001B800BF74
:1009200010B5026843F22443C2F200031A60416822
:10093000596082689A60C168D96002691A61416928
:10094000596182699A61C169D961026A1A62416A10
:100950005962826A9A62C16AD962026B1A63416BF8
:100960005963826B9A63C16BD96300F140001864CC
:100970004EF62850CEF2000002685A6415F010FDC1
:10098000002800F0FB8146F26040C0F6010015F03F
:100990000DFD4EF62C54CEF200042368002B05DA30
:1009A00046F27040C0F6010015F000FD4EF62C51E5
:1009B000CEF20001086810F0020F05D046F2804028
:1009C000C0F6010015F0F2FC4EF62852CEF20002FD
:1009D0005478002C72D046F29840C0F6010015F011
:1009E000E5FC4EF62853CEF20003597811F0010FC2
:1009F00005D046F2A840C0F6010015F0D7FC4EF62F
:100A00002850CEF20000427802F00204E3B22BB18B
:100A100046F2C840C0F6010015F0C8FC4EF6285159
:100A2000CEF20001487800F00402D4B22CB146F2B4
:100A3000EC40C0F6010015F0B9FC4EF62853CEF29A
:100A40000003597801F00800C2B22AB146F21050F2
:100A5000C0F6010015F0AAFC4EF62854CEF20004B0
:100A6000637803F01001C8B228B146F23050C0F6E6
:100A7000010015F09BFC4EF62852CEF2000254788D
:100A800004F02003D9B229B146F25050C0F601005B
:100A900015F08CFC4EF62850CEF20000427802F0A1
:100AA0008004E3B253B14EF63851CEF2000109682A
:100AB00046F27050C0F6010015F078FC4EF6285052
:100AC000CEF20000428894B2002C5ED046F29050E4
:100AD000C0F6010015F06AFC4EF62853CEF2000372
:100AE000598811F0010F05D046F2A050C0F6010060
:100AF00015F05CFC4EF62850CEF20000428802F061
:100B00000204A3B22BB146F2CC50C0F6010015F09E
:100B10004DFC4EF62851CEF20001488800F0040248
:100B200094B22CB146F2F050C0F6010015F03EFC34
:100B30004EF62853CEF20003598801F0080082B225
:100B40002AB146F23060C0F6010015F02FFC4EF6D7
:100B50002854CEF20004638803F4807188B228B16F
:100B600046F26060C0F6010015F020FC4EF62852F7
:100B7000CEF20002548804F4007399B229B146F20F
:100B80007C60C0F6010015F011FC4EF62850CEF244
:100B900000000278002A63D046F29460C0F601009B
:100BA00015F004FC4EF62854CEF20004237813F01E
:100BB000010F05D046F2A460C0F6010015F0F6FB67
:100BC0004EF62851CEF20001087800F00202D4B2AD
:100BD0002CB146F2C460C0F6010015F0E7FB4EF6FA
:100BE0002853CEF20003197801F00800C2B22AB1EE
:100BF00046F2DC60C0F6010015F0D8FB4EF6285432
:100C0000CEF20004237803F01001C8B228B146F2F6
:100C10000070C0F6010015F0C9FB4EF62852CEF266
:100C20000002147804F02003D9B229B146F22470EE
:100C3000C0F6010015F0BAFB4EF62850CEF20000C7
:100C4000027802F08004E3B253B14EF63451CEF292
:100C50000001096846F24470C0F6010015F0A6FBD9
:100C600043F22444C2F20004216A46F27070C0F6D6
:100C7000010015F09BFB616A46F28470C0F601002A
:100C800015F094FBA16A46F29870C0F6010015F0C9
:100C90008DFBE16A46F2AC70C0F6010015F086FBF0
:100CA000216846F2C070C0F6010015F07FFB616854
:100CB00046F2D470C0F6010015F078FBA16846F248
:100CC000E870C0F6010015F071FBE16846F2FC70B7
:100CD000C0F6010015F06AFB216946F61000C0F667
:100CE000010015F063FB616946F62400C0F60100BF
:100CF00015F05CFBA16946F63800C0F6010015F05E
:100D000055FBE16946F64C00C0F6010015F04EFBBC
:100D1000216B46F66000C0F6010015F047FB216C20
:100D200046F67400C0F6010015F040FB616B46F614
:100D30008800C0F6010015F039FBA16B46F6AC0047
:100D4000C0F6010015F032FB43F26C40C2F2000025
:100D5000026846F6D000C0F601001146126815F090
:100D600025FB40F21073C2F200031A6846F6E80051
:100D7000C0F601001146126815F018FBFFF75EFC83
:100D800010BD00BF00B504F0D3FB002808BF5DF81C
:100D900004FBEFF30981EFF3118221E9F40F5DF811
:100DA00004EB1EF0100F08BF21ED108A41F804ED8E
:100DB0000B4C2268002A18BF516004F02BFC2268FB
:100DC000516851F804EB1EF0100F08BFB1EC108A07
:100DD000B1E8F40F82F3118881F3098870470000AD
:100DE0006C34002008B540F68550C0F600004FF086
:100DF000FF016FF00102FFF73BFD08BDF8B50746A4
:100E00000C461E460799089D14F0030F00D0FEE71C
:100E100022B1A4EB8500A0F1480401E004F14800F0
:100E2000012D01D8A16205E02A46FFF717FCA7EBC8
:100E30008507A7624FF0000363604FF01130E06256
:100E40004FF0223121634FF0333262634FF044336D
:100E5000A3604FF05530E0604FF0663121614FF0F4
:100E6000773262614FF08833A3614FF09930E061CF
:100E70004FF0AA3121624FF0BB3262624FF0CC33A7
:100E8000A363E663069820644FF0807161646FF09D
:100E90000202226005F11200F8BD00BF62B64EF6F4
:100EA0000453CEF200031A6842F08050186000BF6D
:100EB0004FEA001046F60013C0F601031A5847F235
:100EC000F011C0F6010151F82200704738B5044610
:100ED0000D46FFF7EDFF46F60013C0F6010303EBE6
:100EE00004146168012902D0022903D101E0856060
:100EF00038BD456138BD00BF10B540F20403C4F6EB
:100F000000031A681A6040F20443C4F600031C6828
:100F100046F6AC11C0F60101486824EA000446F622
:100F20009412C0F60102506804431C6040F60403AA
:100F3000C4F600031868186040F60444C4F60004C0
:100F40002368236041F20404C4F600042068206092
:100F500041F20443C4F600031C68496924EA010411
:100F6000526944EA0200186040F20C01C4F6000124
:100F70000C6846F69C22C0F60102136824EA0304BA
:100F800046F6DC13C0F60103186804430C6040F217
:100F90000C41C4F600010C68506824EA000458684B
:100FA00004430C6040F60C01C4F600010C68906824
:100FB00024EA0004986804430C6040F60C41C4F62F
:100FC00000010C68D06824EA0004D86804430C606F
:100FD00041F20C01C4F600010C68106924EA000417
:100FE000186904430C6041F20C41C4F60001086822
:100FF000526920EA02005B6940EA03040C604FF08A
:10100000000340F21401C4F600010B6046F63012F2
:10101000C0F60102546840F21440C4F600000460B7
:1010200040F61401C4F600010B6040F61444C4F607
:101030000004236041F21400C4F60000036052690A
:1010400041F21443C4F600031A6040F20001C4F6F2
:1010500000010C6846F6F412C0F60102106824EA9A
:10106000000446F64813C0F60103186804430C60F8
:1010700040F20041C4F600010C68506824EA000404
:10108000586804430C6040F60001C4F600010C6887
:10109000906824EA0004986804430C6040F600411C
:1010A000C4F600010C68D06824EA0004D868044340
:1010B0000C6041F20001C4F600010C68106924EADA
:1010C000000418692043086041F20041C4F60001A1
:1010D0000868526920EA02005B69184308604FF013
:1010E000010002F005FC10BD08B541F21403C4F282
:1010F00002031A6842F4FC001860FFF7FDFE08BD09
:101100002DE9F0019DF814709DF81860079D46F6D2
:10111000C414C0F6010454F820004FEA4104FF2F24
:1011200012D0D0F80C8046F6B42CC0F6010C5CF856
:10113000277007FA04FC4FF0030707FA04F728EAC0
:1011400007074CEA0707C760FF2B11D0D0F804C08F
:1011500046F69427C0F6010757F8237007FA01F7FF
:101160004FF0010303FA01F32CEA03033B4343600E
:10117000FF2E10D0876846F61C23C0F6010353F8F3
:10118000266006FA04F64FF0030303FA04F327EA95
:10119000030333438360B5F1FF3F16D04FEAD10319
:1011A00003F1080350F8236001F007014FEA8101C1
:1011B00005F00F0505FA01F54FF00F0707FA01F1E9
:1011C00026EA0101294340F82310FF2A10D00168C4
:1011D0004FF0030303FA04F321EA030346F60C215C
:1011E000C0F6010151F8222002FA04F41C43046005
:1011F000BDE8F001704700BF46F6C413C0F6010316
:1012000053F820000069704746F66023C0F60103DA
:1012100053F820307BB139B146F66011C0F60101B8
:1012200051F820201360704746F62C22C0F60102C8
:1012300052F820000360704700EB800046F6C4239C
:10124000C0F6010353F82000A0F10200112800F2BB
:101250008880DFE800F009121B242D3686868686FA
:101260003F48515A636C757E41F21C00C4F2020083
:10127000036861F300030360704741F21C03C4F28A
:1012800002031A6861F341021A60704741F21C03BD
:10129000C4F20203186861F382001860704741F2DB
:1012A0001C00C4F20200026861F3C30202607047CE
:1012B00041F21C00C4F20200036861F304130360EE
:1012C000704741F21C03C4F202031A6861F345122D
:1012D0001A60704741F21C03C4F20203186861F3FC
:1012E00086101860704741F21C00C4F202000268C8
:1012F00061F3C7120260704741F21C00C4F20200A1
:10130000036861F308230360704741F21803C4F2D5
:1013100002031A6861F310421A60704741F2180321
:10132000C4F20203186861F351401860704741F23B
:101330001800C4F20200026861F392420260704732
:1013400041F21C00C4F20200036861F34923036008
:10135000704741F21803C4F202031A6861F3D342E2
:101360001A60704700EB800046F6C423C0F6010304
:1013700053F8202047F2A011C0F6010151F82200D5
:10138000704700BF2DE9F84F04468A4691469846BB
:101390009DF928709DF92C609DF93050FFF7E2FF10
:1013A00004EB840246F6C423C0F6010303EB820378
:1013B0005A68022A94BF8369C369016A02F1FF3C3B
:1013C000BCF1030F2ED8DFE80CF0021802186FF3FF
:1013D0000103BAF1000FC8BF6AF38203B9F1000F2D
:1013E000C8BF69F3C303B8F1000FC8BF68F30613A1
:1013F000002F17DD67F3C71314E06FF30923BAF169
:10140000000FC8BF6AF38A23B9F1000FC8BF69F3A0
:10141000CB23B8F1000FC8BF68F30E33002FC8BF4D
:1014200067F3CF3302F1FF37032F2FD8DFE807F040
:10143000020D1823002EC8BF66F30001002DC8BF9F
:1014400065F341016FF3C30122E0002EC8BF66F3CC
:101450000411002DC8BF65F345116FF3C71117E0E4
:10146000002EC8BF66F30821002DC8BF65F34921CF
:101470006FF3CB210EE0002EC8BF66F30C31002DB8
:10148000C8BF65F34D316FF3CF3103E0022A01D8B5
:10149000836100E0C361016204EB840446F6C4206A
:1014A000C0F6010050F82430102B0FD0112B19D0AA
:1014B0000F2B21D146F6C022C0F60102116844F27A
:1014C0004400C4F201000160BDE8F88F46F6C02078
:1014D000C0F60100026844F24443C4F201031A60FA
:1014E000BDE8F88F46F6C023C0F601031A6844F63B
:1014F0004401C4F201010A60BDE8F88F38B5044622
:101500000D46FFF72FFF04EB840146F6C423C0F617
:10151000010303EB8104626802F1FF3103290AD859
:10152000DFE801F002040608456338BD856338BD75
:10153000C56338BD056438BD40F2F013C2F2000344
:101540001B689BB1A8B91A686FF300021A604FF0CC
:101550000000586240F2F411C2F2000108801A68DB
:1015600042F0010018604FF0010070474FF000009A
:1015700070474FF00000704710B483B040F2F01392
:10158000C2F200031B6803B310BB40F2F412C2F2B4
:101590000002586A148840EA0440019000BF00BF6E
:1015A00000BF00BF00BF586A148840EA04400090A2
:1015B000019C00988442ECD1DDED017AB8EEE70A97
:1015C00081ED000A4FF0010004E04FF0000001E05F
:1015D0004FF0000003B010BC704700BF40F2F013A2
:1015E000C2F200031B689BB1A8B91A686FF300022E
:1015F0001A6059624FEA114140F2F410C2F2000041
:1016000001801A6842F0010119604FF00100704733
:101610004FF0000070474FF00000704741F2240384
:10162000C4F202031B6847F20402C4F2000212680B
:1016300040F2F611C2F200014FF000000870C2F350
:10164000400242EAD36010F0010F04D008464FF088
:101650008001017023E04FEA136303F01001CAB266
:101660003AB140F2F613C2F200034FF001021A70D1
:1016700015E003F00400C1B239B140F2F610C2F235
:1016800000004FF04001017009E013F0600F06D038
:1016900040F2F613C2F200034FF020021A7041F23A
:1016A0002403C4F202031A6842F08070186047F203
:1016B0000001C4F200010B6843F008020A6043F223
:1016C0006C40C2F20000016840F2F813C2F200035D
:1016D0001960704740F2F613C2F2000318787047A1
:1016E00008B54FF2AC71C1F6FF714FF00C0213F068
:1016F00077F84FF00C0008BD10B542F20803CEF2A7
:1017000004031A6842F01000186041F2B170C0F68C
:1017100000004FF00F014FF03602FFF7A9F841F239
:101720001C01C4F202010C6844F010030B6041F28A
:101730000004C4F2000447F28C02C0F601021068F3
:10174000206047F2FC11C0F60101886911F006FE25
:1017500015A3D3E9002312F045F84FF000024FF033
:101760000003C3F6F07311F0F7FE11F063FE41F2CF
:101770002C03C4F20003188041F22800C4F20000D8
:101780004FF00002028047F29001C0F601010868A4
:1017900041F20C03C4F200031860228842F00101F8
:1017A000218010BDAFF300802D431CEBE2362A3FB1
:1017B000684620F007018D4601B541F21003C4F2DE
:1017C00000034FF000021A6004F0C2F9BDE80140C6
:1017D0008546704770B50446B0F5CC7F2FD940F2EE
:1017E0003233984216D940F26560844215D940F6EA
:1017F000CB418C4214D941F69712944213D943F24B
:101800002F36B44212D946F25F639C4298BF062538
:101810000ED90FE04FF001050AE04FF0020507E096
:101820004FF0030504E04FF0040501E04FF005051B
:10183000072D06D1FEF702FF4FF0070501E04FF03C
:101840000005FEF7A3FF064604EB84044FEAC4003C
:1018500047F29401C0F6010151F83520B0FBF2F3D4
:101860009CB2012C05D9B4F5805F04D3FEF7E6FEE7
:1018700001E04FF0020443F20000C4F2000045F220
:101880005551016047F29402C0F6010202EBC50512
:101890006B6843F20401C4F200010B6043F20802DA
:1018A000C4F2000214604AF6AA2303603046FEF731
:1018B00077FF70BD08B543F20003C4F200034CF695
:1018C000CC421A604FF0C800FFF784FF08BD00BF8C
:1018D00043F20003C4F200034AF6AA221A607047DA
:1018E00010B5044643F20C03C4F20003186810F06C
:1018F000010F74D04FF0320005F0D4FB43F20C011D
:10190000C4F200010A6812F0010F68D04FF03200F3
:1019100005F0C8FB43F20C03C4F20003186810F092
:10192000010F5CD04FF0320005F0BCFB43F20C011C
:10193000C4F200010A6812F0010F50D04FF03200DB
:1019400005F0B0FB43F20C03C4F20003186810F07A
:10195000010F44D04FF0320005F0A4FB43F20C011C
:10196000C4F200010A6812F0010F38D04FF03200C3
:1019700005F098FB43F20C03C4F20003186810F062
:10198000010F2CD04FF0320005F08CFB43F20C011C
:10199000C4F200010A6812F0010F20D04FF03200AB
:1019A00005F080FB43F20C03C4F20003186810F04A
:1019B000010F14D04FF0320005F074FB43F20C011C
:1019C000C4F200010A6812F0010F08D04FF0320093
:1019D00005F068FB43F20C03C4F200031B682046C9
:1019E000FFF7F8FE10BD00BF02469CF8043043B17B
:1019F000DCF8000040B140F22421C2F2000141F8BD
:101A00002200DCF8000050B940F22423C2F20003A7
:101A100053F8220049F64042002808BF104670479C
:101A20004FF0010303FA00F04BF218010140081CCB
:101A300018BF0120704700BF08B540F2FC10C2F289
:101A4000000047F21011C0F6010102F0EFFF41F271
:101A50000403C4F202031A684FF0020161F38F32EB
:101A60001A6041F21800C4F20200036843F40072E5
:101A70000260016841F00103036042F20440C4F2D5
:101A800001004FF00002026047F22C11C0F6010184
:101A9000086842F20C43C4F20103186047F2CC021A
:101AA000C0F60102116842F21040C4F20100016068
:101AB00047F2F003C0F601031A6842F22C41C4F267
:101AC00001010A6047F20C10C0F60100026842F200
:101AD0000843C4F201031A60196841F00400186059
:101AE0001A46136813F0040FFBD108BD38B50D4634
:101AF00040F2FC10C2F200004FF0000102F0AEFF15
:101B0000122D07D140F20003C4F201031A6842F01B
:101B10008070186042F20044C4F20104616B65F306
:101B200004016163E36C4FF0050005F0BBFAA368A4
:101B300043F48002A2602046046814F0020FFBD038
:101B400042F20041C4F20101CC6C122D09D140F2E5
:101B50000003C4F201031A686FF318621A604FEAB7
:101B6000440440F2FC10C2F2000003F085F8204665
:101B700038BD00BF10B52DED028B08EE101A47F2EC
:101B8000D004C0F6010404EB8004F7EE007AB4EE52
:101B9000E78AF1EE10FA09DC084612F035F8002861
:101BA0009FED210A18BFB0EE408A01E0B7EE008A2F
:101BB0002378012B1CD16078FFF7D4FB90ED0B1A32
:101BC0006478F8EE411A21EE888A18EE100A11F0B6
:101BD0006BFC4FF000024FF00003C3F6E07311F00E
:101BE000BDFC11F027FC01462046FFF787FC18E0FA
:101BF000022B16D16478DFED0D0A28EE208A18EE4C
:101C0000100A11F051FC4FF000024FF00003C3F630
:101C1000E07311F0A3FC11F00DFC01462046FFF724
:101C200055F9BDEC028B10BD0000000000F07F45AF
:101C300010B54FF000044FF000002146FFF79AFF67
:101C40004FF001002146FFF795FF4FF002002146BB
:101C5000FFF790FF4FF003002146FFF78BFF4FF097
:101C600004002146FFF786FF4FF005002146FFF7ED
:101C700081FF4FF006002146FFF77CFF4FF0070081
:101C80002146FFF777FF40F20C03C4F600031A6801
:101C900047F21411C0F60101086822EA000247F277
:101CA0004C11C0F60101086802431A6040F20C436F
:101CB000C4F600031A681A6040F60C01C4F600016D
:101CC0000868086040F60C43C4F600031A681A60FE
:101CD00041F20C01C4F600010868086041F20C43AF
:101CE000C4F600031A681A6040F20000C4F600004F
:101CF000036847F23011C0F601010A6823EA0203C3
:101D000047F2F401C0F601010A681343036040F290
:101D10000040C4F600000368036040F60001C4F60A
:101D200000010A680A6040F60040C4F6000003683B
:101D3000036041F20001C4F600010A680A6041F242
:101D40000040C4F600000368036010BD08B5012818
:101D500005D84FF000000146FFF7C8FE08BD4FF060
:101D6000FF3008BD08B5FFF7F1FF07EE900AB8EEA7
:101D7000677A9FED030AC7EE000A10EE900A08BDCD
:101D800000F07F4538B50D46044600B3132801D94D
:101D9000FEF754FC47F2FC13C0F6010353F824008D
:101DA00055B1B0FBF5F14FEA114202F10103B0FB6E
:101DB000F3F0B0FBF5F502E04FF000052A4647F2DC
:101DC000A011C0F6010151F824309A62DD6238BDDD
:101DD00030B583B000918DF80420082816D14FF05B
:101DE00000042046FFF71CFE38B1EC462046FFF702
:101DF000FBFD01462046FFF7C5FF04F1010425461F
:101E00002046FFF70DFE002829D020E047F2D0033E
:101E1000C0F6010313F82010012916D147F2D002B1
:101E2000C0F6010202EB8000447804EB840346F61E
:101E3000C421C0F6010151F82340EC462046FFF7CB
:101E4000D3FD01462046FFF79DFF03B030BDEC46B1
:101E50002046FFF7C9FD01462046FFF793FF04F136
:101E60000104142CBDD1F0E7F0B585B0FFF7E4FD17
:101E70004FF02D004FF00101FFF7DEF94FF00900A0
:101E80004FF00101FFF7D8F94FF008004FF00101C2
:101E9000FFF7D2F94FF031004FF00101FFF7CCF915
:101EA0004FF030004FF00101FFF7C6F94FF00D0081
:101EB0004FF00101FFF7C0F94FF010004FF00101A2
:101EC000FFF7BAF94FF00F004FF00101FFF7B4F937
:101ED0004FF0000400944FF00106019602944FF079
:101EE0002D00214632464FF00603FFF74BFA46F627
:101EF000C425C0F6010595F89003D5F89413009415
:101F00000194D5F88C3302934FF003022346FFF778
:101F1000F7F80094019602944FF0090021463246EA
:101F20004FF00603FFF72EFA95F8C000D5F8C4105D
:101F300000940194D5F8BC2002924FF0030223468E
:101F4000FFF7DEF80094019602944FF00800214656
:101F500032464FF00603FFF715FA95F8AC00D5F8B6
:101F6000B01000940194D5F8A87002974FF00302C6
:101F70002346FFF7C5F80094019602944FF0310014
:101F8000214632464FF00603FFF7FCF995F8E003CF
:101F9000D5F8E41300940194D5F8DC3302934FF0A4
:101FA00003022346FFF7ACF80094019602944FF029
:101FB0003000214632464FF00603FFF7E3F995F86B
:101FC000CC03D5F8D01300940194D5F8C82302921D
:101FD0004FF003022346FFF793F800940196029412
:101FE0004FF00D00214632464FF00603FFF7CAF9C5
:101FF00095F81001D5F8141100940194D5F80C71DE
:1020000002974FF003022346FFF77AF800940196F7
:1020100002944FF01000214632464FF00603FFF7BE
:10202000B1F995F84C01D5F8501100940194D5F808
:10203000483102934FF003022346FFF761F8009402
:10204000019602944FF00F00214632464FF00603EE
:10205000FFF798F995F83801D5F83C1100940194F0
:10206000D5F8345102954FF003022346FFF748F8A4
:102070004FF0080021462246FFF7AAFE4FF0000766
:1020800020463946FFF776FD30463946FFF772FDA8
:102090004FF002003946FFF76DFD4FF0030039465F
:1020A000FFF768FD4FF004003946FFF763FD4FF07E
:1020B00005003946FFF75EFD4FF006003946FFF791
:1020C00059FD4FF007003946FFF754FD47F2A015C0
:1020D000C0F6010547F24817C0F601073046FFF782
:1020E0009FFCB8B113E02046FFF79AFC10B16B6873
:1020F0003A681A6004F10104204605F10405FFF76F
:102100008FFC78B10BE0FFF793FD05B0F0BD686878
:102110003968016006F1010405F10405E3E7686828
:102120003968016004F1010405F10405142CDAD1C9
:10213000E9E700BF10B5044641F21803C4F20203F8
:10214000186810F4007F01D1FFF776FC4FF0000013
:102150004FF01101FFF7CAFC4FF2BA71C1F6FF71DF
:102160000A8807EE902AB8EE670A06EE900AB8EEE3
:10217000667AC0EE070AC4ED000A4FF0010010BDF8
:1021800008B572B647F27413C0F601031A684EF62A
:102190003470CEF20000026047F26411C0F6010113
:1021A0000A684EF68853CEF200031A6047F27C109C
:1021B000C0F60100016842F20802CEF2040211608A
:1021C00047F27013C0F60103186842F20C01CEF218
:1021D0000401086041F20003C4F202031A6842F4E9
:1021E0008030186019460B6813F4003FFBD047F2AB
:1021F0006812C0F60102106841F20401C4F2020143
:10220000086047F26C13C0F601031A6842F200003E
:10221000C4F20200026041F20001C4F202010B6844
:1022200043F080720A600846016811F0007FFBD01D
:1022300041F20403C4F202031A684FF0020060F393
:1022400001021A6019460B6803F00C02082AFAD141
:1022500041F21800C4F20200016841F0010303607A
:1022600042F21C02C4F20202106846F22041C0F69B
:1022700001010A6847F27813C0F601031B68504059
:10228000184215D046F22041C0F60101087800F04E
:102290000401C8B260B942F21C01C4F2020108682C
:1022A00020EA0300134018434FF0FF3100F0A4F977
:1022B00008BD00BF41F21403C4F202031A6842F0E1
:1022C00001001860704700BF70B41646002A47D05E
:1022D00040F20802C4F20202146814F0010F06D0A2
:1022E00040F20C05C4F202052A68002AFCD140F233
:1022F0000804C4F202044FF00005256047F2801282
:10230000C0F60102156840F20402C4F20202156030
:1023100040F21002C4F20202116040F21401C4F251
:102320000201086040F20C00C4F20200066047F2AD
:102330008412C0F6010211682160206840F0010299
:1023400022606BB140F20C01C4F202010B68002B59
:10235000FCD140F20800C4F202004FF0000202601B
:1023600070BC704742F21003C4F20203186810F008
:10237000800F0DD042F20401C4F2020140F2231298
:10238000C4F267520A6048F6AB13CCF6EF530B6009
:1023900042F21000C4F20200016801F08002002A3B
:1023A00014BF02200020704742F21003C4F202035F
:1023B000186810F0800F07D142F21001C4F2020138
:1023C0000A6842F080030B60704700BF40F20003D0
:1023D000C0F60003984208D340F20001C0F60401A1
:1023E00088422CBF0020012070474FF0000070474A
:1023F0002DE9F04706460D46FFF7E8FF002855D0C7
:102400002846FFF7E3FF002853D0AE4254D8FEF72A
:10241000BDF98246FFF7A6FF0446B8BB41F28830FB
:10242000FFF75EFA47F29413C0F601031A6842F20E
:102430001000C4F20200026042F21409C4F2020960
:10244000804642F20C07C4F20207FFF741FAC9F8CE
:102450000060D8F8001041F04003C8F8003006F5DD
:1024600000663A6812F0010FFBD1386810F0200FB7
:102470000AD0396841F020033B60B542E5D24FF005
:102480006400FFF72DFA01E04FF0020447F29812C2
:10249000C0F60102106842F21001C4F202010860A5
:1024A000FFF782FF5046FEF77BF907E04FF002048A
:1024B00004E04FF0020401E04FF002042046BDE8C2
:1024C000F08700BFF8B507460C4616460846FFF7EA
:1024D0007DFF002800F0898006F1FF302018FFF70B
:1024E00075FF002800F0848040F22073C2F20003E0
:1024F00053E8002F02F1010243E800210129F7D03F
:10250000FFF730FF054600284BD147F29C11C0F67B
:1025100001010A6842F21000C4F20200026014F0E5
:10252000010F09D037F8013C24F8013C04F1010403
:1025300007F1010706F1FF36012E25D904F1020249
:1025400007F10200A6F1020C4FEA5C0C04F1040E44
:102550000EEB4C0E42F20C01C4F202010B6813F0B8
:10256000010FFBD130F8023C22F8023C02F10202DA
:1025700000F102007245F1D10CF101024FEA420074
:1025800024183F1806F001060EB13978218047F271
:102590008814C0F60104226842F21003C4F2020358
:1025A0001A60FFF701FF40F22073C2F2000353E804
:1025B000002FA2F1010243E80024012CF7D053E8D8
:1025C000002FB2F1004F0DD14FF0000243E800247C
:1025D000012CF4D04EF60450CEF20000016841F018
:1025E00080510160BFF32F8F04E04FF0020501E03E
:1025F0004FF002052846F8BD30B585B004460D46BB
:1026000068464FF0FF014FF0100212F00DF9E3B2EF
:1026100003F00402D0B2002840F0A28003F00201CF
:10262000CBB223B14FF011008DF8000003E06FF042
:1026300055028DF80020C4F307218DF80210C4F371
:1026400007438DF804304FEA14648DF806408DF886
:102650000850FEF79BF80546FFF784FE002873D16B
:1026600042F20800C4F2020040F22312C4F26752A0
:10267000026048F6AB11CCF6EF51016042F2100354
:10268000C4F202031C6814F4007F5DD047F28C1082
:10269000C0F60100026842F21001C4F202010A60B1
:1026A0000B6843F040040C6042F20C00C4F20200DC
:1026B000026812F0010FFBD142F21003C4F20203D0
:1026C0004FF00001196042F20804C4F2020440F223
:1026D0002310C4F26750206048F6AB12CCF6EF52DC
:1026E00022601B6813F4007F2ED047F29011C0F6D1
:1026F00001010C6842F21000C4F2020004604FF6BF
:102700000003C1F6FF7303F11002934213D24FF09E
:1027100010044FF00001184642F20C02C4F202020B
:102720003DF801300B52136813F0010FFBD101F19A
:102730000201A142F4D142F21004C4F202044FF0AB
:1027400000012160FFF730FE4FF0000442F210005C
:10275000C4F2020004602846FEF722F8204601E099
:102760004FF0020005B030BD08B543F27040C2F230
:10277000000043F27072C2F20002131A4FF0FF31F0
:102780004FEAA302FDF7BCFF01F04AFDFEF786FB0E
:102790004FF0000008BD00BFBFF36F8F704700BF50
:1027A00047F24C23C0F60103185C00EB400147F2EE
:1027B0006832C0F6010252F821305B6A704700BFF0
:1027C00038B547F24C23C0F601031B5C03EBC3048E
:1027D00040F27422C2F2000202EB840282F821105D
:1027E00014693CB140F27425C2F200051346D26967
:1027F0009B69A04738BD00BFF8B506460F4647F2B3
:102800004C23C0F601031D5C05EBC50040F27424A7
:10281000C2F2000404EB8004D4F810C0BCF1000F35
:1028200007D0E2698A4204D030464FF00001A36924
:10283000E047E76163695BB105EBC50040F27422D4
:10284000C2F2000202EB8002304639469269984794
:1028500094F8201079B127696FB105EBC50540F2F6
:102860007423C2F2000303EB8505304694F821106F
:10287000E269AB69B847F8BD47F24C23C0F60103E3
:10288000185C00EB400147F26832C0F6010252F8D2
:102890002130186840F080011960704747F24C23DE
:1028A000C0F60103185C00EB400147F26832C0F645
:1028B000010252F82130986940F0020199611A68CA
:1028C00042F080001860704747F24C23C0F60103C5
:1028D0001A5C02EB420347F26832C0F6010252F87A
:1028E0002330DA6912F0800F1ABF996201200020AC
:1028F000196841F080021A60704700BF47F24C230C
:10290000C0F60103185C00EB400347F26832C0F6E2
:10291000010252F82300C36913F0800FFBD08162DB
:10292000704700BFF8B5044600EB400247F2683339
:10293000C0F6010353F82260F569356205F0010223
:1029400015F0020F1CBF42F00202D2B215F0040FC4
:1029500018BF42F0080215F0080F18BF42F0040239
:1029600015F4807F05D0706810F4804F18BF42F0D6
:10297000100215F0200F00D1E2B104EBC40140F2C7
:102980007427C2F2000707EB81039F688FB1716A59
:1029900004EBC40040F27423C2F2000303EB800393
:1029A00047F20030C0F60100005DC9B29B69B8472C
:1029B00000E0736A326812F0800F1CD015F0800FAF
:1029C00019D031686FF3C711316004EBC40040F2D5
:1029D0007423C2F2000353F8203063B140F2742232
:1029E000C2F2000202EB800247F20030C0F60100A2
:1029F000005D9169984715F0400F17D004EBC401B2
:102A000040F27423C2F2000303EB810253686BB1FE
:102A1000084640F27421C2F2000101EB800247F245
:102A20000030C0F60100005D91699847F8BD00BF15
:102A3000684620F007018D4601B54FF00300FFF70F
:102A400071FFBDE801408546704700BF684620F031
:102A500007018D4601B54FF00200FFF763FFBDE8A7
:102A600001408546704700BF684620F007018D464B
:102A700001B54FF00100FFF755FFBDE80140854665
:102A8000704700BF2DE9F04385B016461F4647F258
:102A90004C23C0F601031C5C04EB440247F268358A
:102AA000C0F6010555F8224047F20433C0F6010391
:102AB000185C00EB400247F20835C0F6010505EB53
:102AC000C2058846002956D0002E57D0287B296998
:102AD0009DF8342000924FF0010301936A6902923D
:102AE0004FF003023B46FEF70BFB40F22073C2F2AD
:102AF000000353E8002F02F1010243E800210129FD
:102B0000F7D021684FF000002060012E14BF00268E
:102B10000126626866F3CF32626047F2FC20C0F69D
:102B200001000268B8F1010F14BF4FF000084FF028
:102B3000010868F3C302A260216053E8002FA2F1EC
:102B4000010243E80024012CF7D053E8002FB2F132
:102B5000004F0DD14FF0000243E80024012CF4D0C7
:102B60004EF60450CEF20000016841F08051016041
:102B7000BFF32F8F17E04FF0010901E04FF000097C
:102B8000287869689DF8303000934FF00102019277
:102B9000AB6802934FF003023B46FEF7B1FAB9F17E
:102BA000000FA2D092E705B0BDE8F0832DE9F84F01
:102BB00081468B4690461E469DF828A047F24C233E
:102BC000C0F601031D5C05EB450247F26830C0F614
:102BD000010050F822409DF82C70012F14BF0027EF
:102BE0000127082E06D0072E02D1B8F1000F01D11F
:102BF000FDF724FD0AF1FF31CBB2012B01D9FDF71E
:102C00001DFD47F25832C0F6010252F82500B0FB14
:102C1000FBF1E1604FF0200267F38612BAF1010F79
:102C200004D0002F0CBF0223002301E04FF000036B
:102C300063F30D3267F38E326068C0F3C03363F321
:102C4000CF3262604FF06D01B8F1020F14BF002364
:102C5000012363F3492118F1000818BF4FF0010860
:102C600068F38A21082E18BF4FF0000868F30C3172
:102C700021604846FFF794FDBDE8F88F2DE9F84341
:102C8000054647F24C23C0F60103185C00EBC00276
:102C900040F27424C2F2000404EB820447F268316B
:102CA000C0F6010100EB40064FEA860301EB030882
:102CB00051F80390FDF76AFD064694F82000B8B17C
:102CC0004FF00007C9F800703846394698F90420DB
:102CD000FDF7CEFD28463946FFF772FDE3681BB1CC
:102CE0002846E169A26998474FF0000284F8202045
:102CF0003046FDF755FDBDE8F88300BF2DE9F04FE4
:102D000085B005468B469246994647F24C23C0F65D
:102D100001031E5C40F27428C2F2000806EBC607ED
:102D20004FEA870708EB070406EB460047F26831D5
:102D3000C0F6010101EB8006FDF728FD039041F28A
:102D40001C03C4F20203186847F25021C0F60101C7
:102D50000A6820EA020E47F25032C0F601021068FB
:102D60004EEA0000186041F21803C4F2020318682A
:102D7000496820EA010052681043186047F2E821D0
:102D8000C0F6010105EB8503C818C95C4278837859
:102D900090F803C0CDF800C0007901902846FFF7F5
:102DA00071FE9DF8382000929DF83C100191284654
:102DB000594652464B46FFF7F9FE109B48F807303C
:102DC0001298A060119A62601399E160149BA3614C
:102DD000B0684FF00F0196F90420FDF749FD4FF060
:102DE000010084F820000398FDF7DAFC05B0BDE887
:102DF000F08F00BF47F24C23C0F60103185C00EBD4
:102E0000C00340F27420C2F2000000EB830319619A
:102E10005A61704747F20433C0F60103185C00EBB7
:102E2000400147F25822C0F6010202EB0110704740
:102E3000F8B54FF04C0404FB00F440F62021C2F238
:102E40000001621846F20003C4F2000303EB001312
:102E500045F60045C4F2000505EB80006558002DDD
:102E60006BD094680CB1968801E04FF000061F68A3
:102E700066F30F071F6059686FF309015960D16845
:102E800019B15668A719BFB201E04FF000079E685C
:102E900067F30F069E603E2994BF00270127DE6876
:102EA00067F3CF36DE60DE6816F4004F1DBF4F09B2
:102EB00007F1FF3707F01F07C1F34407DE6867F328
:102EC0008E26DE600368166A66F303032E7A47F2E5
:102ED0009C35C0F6010555F8265065F34A236FF37B
:102EE0000823C3F30115002C14BF022400246C40F6
:102EF00064F30513C3F30134002914BF0321002137
:102F0000614061F30D336FF3CF336FF3C713036089
:102F100040F6DC10C2F200000378191F18BF01212F
:102F200051624FF0010090624FF00003D3621363CF
:102F3000536302F1100000F0BBFCF8BDF8B545F694
:102F40004443C4F200031C6814F4004F52D040F60E
:102F5000DC10C2F20000017801294BD945F6444249
:102F6000C4F20002156805F00F0640F62027C2F2F1
:102F700000074FF04C0303FB067545F60040C4F212
:102F8000000000EB860750F82660C6F3C031EA6AFD
:102F90000A43EA62C6F3C0202B6B03432B63C6F3DC
:102FA000C0116A6B0A436A63C6F3072000F0080386
:102FB000D9B219B14FF00001E9630BE0EA6B4AB1F5
:102FC00026F07F00C3B22BB14FF000016963286A7D
:102FD00003F0CCFAEA6A0AB9686B18B105F110007F
:102FE00000F066FC47F2C433C0F60103196826EA14
:102FF00001063E6014F4806F0DD040F60E20C2F240
:1030000000004FF00102027040F6E013C2F200032C
:10301000186801F083FF14F4006F1CD045F640419E
:10302000C4F20001086840F008020A6040F60D236F
:10303000C2F200034FF00101197040F68140C2F264
:1030400000004FF00002027040F6E013C2F20003ED
:10305000186801F063FF14F4805F1CD045F640410E
:10306000C4F2000108686FF3C300086040F60D2346
:10307000C2F200034FF000021A7040F68141C2F222
:1030800000014FF00100087040F6E013C2F20003A7
:10309000186801F043FF6FEA040445F64442C4F2A5
:1030A00000021460F8BD00BF684620F007018D469D
:1030B00089B500AFFFF742FFBD46BDE889408546B0
:1030C000704700BF45F64043C4F200031A6860F33E
:1030D000CF321A60704700BF40F68443C2F200034B
:1030E0001A5C45F60040C4F2000049B150F82200D5
:1030F000C0F3011147F2AC33C0F60103585C7047CE
:1031000050F82210C1F3013347F2AC32C0F601028D
:10311000D05C704740F68443C2F200031A7845F64B
:103120000043C4F2000353F8221047F2C030C0F647
:103130000100006821EA000181F0100141F4807073
:1031400043F82200704700BF2DE9F00340F68443A6
:10315000C2F20003185C45F6004CC4F2000C0CEB04
:10316000800C4FEA001346F20007C4F2000703EB9D
:103170000708D85983B207EB4307012A31D901F177
:103180000204A2F102094FEA590901F1040606EB13
:103190004906351BA5F10205C5F3400534F8024C7C
:1031A000384620F8044B01F10403B34238D10FE054
:1031B00033F8025C044624F8045B03F1020333F89D
:1031C000025C858004F1040003F10203B342EFD1F5
:1031D00002F0010009F1010901EB490107EB890740
:1031E00000E0104608B109783980D8F8040062F38D
:1031F0000900C8F80400DCF8003047F29832C0F645
:103200000102116823EA01000346C0F3011282F0B3
:10321000030161F30513CCF80030BDE8F0037047FB
:10322000002DC5D033F8024C20F8044B03F1020303
:10323000B342BDD1CCE700BF2DE9F00140F6844395
:10324000C2F200031C5C45F6004CC4F2000C0CEB0F
:10325000840C46F20000C4F2000000EB0414A368E2
:103260009BB200EB4300E3684FEA83534FEA93536A
:10327000934204D2E2684FEA82534FEA9352012A02
:1032800031D901F10203A2F102084FEA580801F115
:10329000040707EB4807FD1AA5F10205C5F3400630
:1032A000044634F8045B23F8025C01F10403BB42DA
:1032B00033D10FE0254635F8046B23F8026C03F197
:1032C0000203A48823F8024C05F1040403F102036D
:1032D000BB42EFD102F0010308F1010801EB480104
:1032E00000EB880000E013460BB103880B70DCF89C
:1032F000000047F2B831C0F601010B6820EA030074
:103300000346C0F3013181F0030060F30D33CCF8C4
:1033100000301046BDE8F0017047002ECAD034F8E6
:10332000045B23F8025C03F10203BB42C2D1D1E784
:1033300008B545F64043C4F200031A686FF3C302B0
:103340001A604FF00000FFF773FD4FF00100FFF728
:103350006FFD4FF00200FFF76BFD4FF00300FFF72A
:1033600067FD4FF00400FFF763FD4FF00500FFF726
:103370005FFD4FF00600FFF75BFD4FF00700FFF722
:1033800057FD47F2B030C0F60100016845F64C43E6
:10339000C4F20003196008BD2DE9F041074640F66C
:1033A0002023C2F200031868002800F0118140F6C3
:1033B0002021C2F200014A683F2A08D940F62024A1
:1033C000C2F20004A5685619E368F51801E04FF051
:1033D000400540F62020C2F20000C16C002900F038
:1033E000008140F62022C2F20002146DA54207D8E7
:1033F00040F62026C2F20006756D6019B36DC5183F
:1034000040F62021C2F20001D1F89820002A00F0F5
:10341000EC8040F62024C2F20004D4F89C60B5424F
:1034200009D840F62020C2F20000D0F8A05071194F
:10343000D0F8A430CD1840F62022C2F20002D2F813
:10344000E440002C00F0D58040F62026C2F20006B1
:10345000D6F8E800854209D840F62021C2F20001E2
:10346000D1F8EC504219D1F8F030D51840F62024AC
:10347000C2F20004D4F83061002E00F0BE8040F6A5
:103480002020C2F20000D0F834118D4209D840F655
:103490002022C2F20002D2F838514C19D2F83C3145
:1034A000E51840F62026C2F20006D6F87C01002876
:1034B00000F0A78040F62021C2F20001D1F880215F
:1034C000954209D840F62024C2F20004D4F8845171
:1034D0005619D4F88831F51840F62020C2F20000C1
:1034E000D0F8C811002900F0908040F62022C2F2E6
:1034F0000002D2F8CC41A54209D840F62026C2F2FB
:103500000006D6F8D0516019D6F8D431C51840F667
:103510002021C2F20001D1F81422002A79D040F60D
:103520002024C2F20004D4F81862B54209D840F64B
:103530002020C2F20000D0F81C527119D0F82032BD
:10354000CD1840F62022C2F20002D2F86042002CD0
:1035500063D0454E4FF00808FDF770F8387A88B10F
:1035600040F20431C2F200010A8812F0020F0CD0BE
:103570004FF0010404F1010442FA04F313F0010FC7
:10358000F8D104E04FF0000401E04FF0010440F2F4
:103590000430C2F200004FF0010202FA04F2018886
:1035A0000A4302807889B060BB89F3603F2B99BFE2
:1035B000013323F001031F3323F01F03F360F2688C
:1035C00081184819B0F5E07F2ED9FDF737F82BE0C8
:1035D00040F62026C2F200064FF000084FF04005EA
:1035E0001EE0224E4FF001081AE0214E4FF0020873
:1035F00016E0204E4FF0030812E01F4E4FF0040873
:103600000EE01E4E4FF005080AE01D4E4FF0060872
:1036100006E01C4E4FF0070802E0134E4FF008087A
:10362000B8F1070F9AD997E740F68443C2F2000336
:1036300003F804803760756006F1200528464FF0D6
:1036400000014FF01C0211F0EFF834627A68B263A7
:1036500006F110004FF006013A682B4600F008F919
:103660002046BDE8F08100BF800C00206C0A0020DD
:10367000B80A0020040B0020500B00209C0B0020F7
:10368000E80B0020340C0020032907D145F64C43F9
:10369000C4F200031A6860F306021A60704700BFA4
:1036A000F0B585B00646002842D041F21C01C4F2B4
:1036B00002010C6844F400050D604FF00004009412
:1036C0004FF0030501954FF00E07029720464FF08B
:1036D0000B012A462346FDF713FD0094019502973E
:1036E00020464FF00C012A462346FDF709FD47F21C
:1036F000B433C0F601031A6845F64047C4F2000728
:103700003A60284603F0CEFC3C6043F2A900C0F6C4
:1037100000004FF00F014FF04B02FDF7A9F845F6FE
:103720004440C4F2000004604FF41C41396011E0D1
:103730004FF000004FF00F014FF04B02FDF798F8EB
:1037400047F2BC33C0F601031A6845F64040C4F2A4
:10375000000002603046FCF75DFF05B0F0BD00BF21
:103760002DE9F04182B047F2C837C0F6010743F6B1
:103770004106C0F6000640F28815C2F200054FF07F
:103780000408CDF8008038464FF0800132462B46C1
:1037900001F010FD40F20834C2F200042060CDF8C0
:1037A000008038464FF08101324605EB080301F0F6
:1037B00001FD6060CDF8008038464FF0820132464E
:1037C00005F1080301F0F6FCA060CDF80080384652
:1037D0004FF08301324605F10C0301F0EBFCE06091
:1037E000CDF8008038464FF08401324605F11003D1
:1037F00001F0E0FC2061CDF8008038464FF08501F3
:10380000324605F1140301F0D5FC6061CDF800806B
:1038100038464FF08601324605F1180301F0CAFC24
:10382000A061CDF8008038464FF08701324605F19F
:103830001C0301F0BFFCE06102B0BDE8F08100BFF5
:1038400008B505464FF000060BE0FCF79FFF2C681B
:10385000616829606660FCF7A3FF22680AB1A0686E
:1038600090472B68B3F1FF3FEFD101F025FBF8E75C
:103870000260B3F1FF3F18BF8360FF290ED143F20E
:103880006C43C2F200031A6822B192F829304FEA61
:10389000530101E04FF007010173704701F07F0110
:1038A0000173704710B14FF000020260704700BF13
:1038B00038B50446FCF76AFF0546A4B1636893B9BE
:1038C000227B40F28810C2F2000050F822106160A2
:1038D00040F82240227B40F20833C2F2000353F842
:1038E000220001F01BFB2846FCF75AFF38BD00BF41
:1038F00010B5044640F2EC40C2F200004FF0000167
:103900004FF0180210F090FFD4B140F25830C2F2DC
:1039100000004FF000014FF0300210F085FF40F240
:10392000CC30C2F200004FF000014FF0180210F04E
:103930007BFF40F2C433C2F200034FF002021A7060
:1039400010BD00BF38B547F20C43C0F6010353F871
:10395000205040F28831C2F2000151F8204047F275
:103960004C42C0F60102105CFDF746FC2840A04224
:1039700014BF0020012038BD47F24C43C0F60103BC
:103980001A5C40F2CC31C2F2000151F8222047F219
:103990000C43C0F6010353F8200002420CBF002084
:1039A0000120704770B440F22073C2F2000353E864
:1039B000002F02F1010243E800210129F7D047F26C
:1039C0004C42C0F60102155C40F2EC41C2F200012B
:1039D00051F8254047F20C46C0F6010656F8202063
:1039E00024EA020041F8250053E8005FA5F1010533
:1039F00043E80056012EF7D053E8005FB5F1004FC1
:103A00000DD14FF0000543E80056012EF4D04EF6DC
:103A10000450CEF20000016841F080510160BFF314
:103A20002F8F14420CBF0020012070BC704700BFD4
:103A300047F25C43C0F60103185C704710B50446BA
:103A4000FDF7DAFB40F2A813C2F2000353F824108A
:103A5000484010BD10B504464FF00100FFF748FF85
:103A600047F2D433C0F6010353F8342040F2C83192
:103A7000C2F200010A6003EBC404606840F2E43360
:103A8000C2F20003186010BD00B585B04FF0000011
:103A9000FFF7E0FF4FF00003009340F2E832C2F27C
:103AA000000201924FF04000029047F24040C0F601
:103AB00001004FF0020143F65D32C0F6000201F052
:103AC00065FA40F2E843C2F20003186005B000BD99
:103AD0002DE9F001804600283CD04FF000034FEA6A
:103AE0008302086850F823404D6855F8236086EA41
:103AF0000407886850F8235084EA050C4CEA07074D
:103B00006FEA070CC86850F8235026EA050707EA51
:103B10000C0705EA0C0C66EA0C06354040F8235009
:103B2000CD6855F82300384345F823000D6955F852
:103B30002300384345F823004D690DB145F8237043
:103B400048688558886885504868845003F10103A7
:103B50004345C4D1BDE8F001704700BF2DE9F843EB
:103B600040F2C838C2F2000840F2BC36C2F2000689
:103B700040F22834C2F200044FF0000540F2E4376E
:103B8000C2F20007D8F8000000EB800001F05CFBF7
:103B90003368002B40F09380204629464FF01802EE
:103BA00010F042FE8BE04FF0060047F2F431C0F611
:103BB0000101FFF78DFF40F2C431C2F200010B7822
:103BC0003BB103F1FF32D3B240F2EC40C2F200004D
:103BD000056040F2C031C2F200010A6822B940F229
:103BE000C030C2F2000005603BB103F1FF33DBB22D
:103BF00040F2EC41C2F200014D6040F2C032C2F22C
:103C00000002106820B940F2C031C2F200010D601C
:103C10003BB103F1FF33DBB240F2EC42C2F20002EF
:103C2000956040F2C030C2F20000016821B940F254
:103C3000C032C2F2000215603BB103F1FF33DBB2C8
:103C400040F2EC40C2F20000C56040F2C031C2F266
:103C500000010A6822B940F2C030C2F200000560DB
:103C60003BB103F1FF33DBB240F2EC41C2F20001A1
:103C70000D6140F2C032C2F20002106820B940F279
:103C8000C031C2F200010D603BB103F1FF33DBB282
:103C900040F2EC42C2F20002556140F2C030C2F282
:103CA0000000016821B940F2C032C2F20002156082
:103CB00040F2C430C2F200000370356062E7D4F80D
:103CC00000902846FFF7BAFE40EA09012160D4F8C7
:103CD00004904FF00100FFF7B1FE40EA0902626074
:103CE000D4F808904FF00200FFF7A8FE40EA090060
:103CF000A060D4F80C904FF00300FFF79FFE40EA5D
:103D00000903E360D4F810904FF00400FFF796FE2B
:103D100040EA09012161D4F814904FF00500FFF743
:103D20008DFE40EA09026261306800F101003060F6
:103D30003B689842FFF426AF35E700BF00B585B079
:103D40004FF00003009340F23852C2F20002019299
:103D50004FF04000029047F26C50C0F601004FF067
:103D6000060143F67D52C0F6000201F00FF940F261
:103D70000453C2F20003186005B000BD2DE9F04FF6
:103D800085B040F284631F46C2F2000740F25460DF
:103D90000646C2F2000640F22051C2F20001029132
:103DA00001F08AF83A68002AFAD014E1A359002BEE
:103DB00051D02846FFF742FE029962586050904366
:103DC00049D0A35910EA030245D0039991F800E0C5
:103DD00047F27459C0F601094FEA451840F20851FC
:103DE000C2F200014FF6FF7C47F26C4AC0F6010AAE
:103DF00040F23C6BC2F2000B204674468646C2F18C
:103E00000003134022EA03021CB95EF80B000342D0
:103E10001ED1180E04D01AF8003003F118030DE07B
:103E2000180C04D01AF8003003F1100306E0180A49
:103E30001ABF1AF8003008331AF80330434419F84F
:103E4000033031F8130060451CBF013021F8130026
:103E5000002AD4D1744605F1010504F10404062DAD
:103E6000A4D1019D6A1E019240F0AC8003990C78A8
:103E700004F10104E3B20B700B2B03D14FF00005EA
:103E80000D7002E0002B40F09A8040F26C62C2F2AA
:103E90000002116891B16FEA010433682340336076
:103EA00040F23C60C2F2000005682C40046040F221
:103EB0006C61C2F200014FF000020A6040F26C64D3
:103EC000C2F20004636893B16FEA030075680540AD
:103ED000756040F23C62C2F20002516808405060D6
:103EE00040F26C64C2F200044FF00003636040F2E1
:103EF0006C60C2F20000856895B16FEA0504B26893
:103F00002240B26040F23C63C2F2000399680C4068
:103F10009C6040F26C60C2F200004FF000058560CA
:103F200040F26C64C2F20004E26892B16FEA0203EC
:103F3000F1681940F16040F23C60C2F20000C568CF
:103F40002B40C36040F26C64C2F200044FF00002E8
:103F5000E26040F26C63C2F20003196991B16FEA4A
:103F6000010035690540356140F23C64C2F200044D
:103F700022691040206140F26C63C2F200034FF0EE
:103F80000001196140F26C60C2F20000456995B110
:103F90006FEA050472692240726140F23C63C2F22A
:103FA000000359690C405C6140F26C60C2F2000091
:103FB0004FF0000545614FF4FA74019402E04FF4AC
:103FC000FA7001904FF0010001F03EF93A68002AC2
:103FD0003FF4E6AE07E04FF4FA74019440F238651E
:103FE000C2F2000503954FF000042546DEE600BF4F
:103FF00010B54FF0000440F28463C2F200031C606D
:1040000040F23C60C2F2000021464FF00602FCF78D
:1040100077FB40F25460C2F2000021464FF00602E6
:10402000FCF76EFB40F26C60C2F2000021464FF0DC
:104030000602FCF765FB40F22050C2F20000214668
:104040004FF00602FCF75CFB40F20850C2F20000A1
:1040500021464FF0180210F0E7FB40F23860C2F240
:104060000000047010BD00BF70B547F24C43C0F6AD
:1040700001031B5C47F20C42C0F6010252F82020FB
:1040800040F28460C2F20000046840F25465C2F25B
:10409000000555F82300104206D104F1010640F254
:1040A0008465C2F200052E6049B140F23C61C2F263
:1040B000000151F82350154341F8235009E040F224
:1040C0003C61C2F2000151F8235025EA020541F893
:1040D0002350104340F25461C2F2000141F8230022
:1040E00040F26C61C2F2000151F8230020EA0202A2
:1040F00041F8232034B940F20453C2F20003186897
:1041000000F00CFF70BD00BF30B447F24C43C0F666
:1041100001031B5C47F20C42C0F6010252F820205A
:1041200040F25460C2F2000050F82300104229D03F
:1041300040F28464C2F20004256805F1010525609F
:1041400071B140F26C61C2F2000151F82340144396
:1041500041F8234040F23861C2F20001097889B980
:104160006FEA020240F23C61C2F2000151F82340C2
:10417000144041F82340024040F25460C2F2000073
:1041800040F8232030BC704730B4034640F2207220
:10419000C2F2000252E8000F00F1010042E8000400
:1041A000012CF7D040F20850C2F2000030F8132082
:1041B00039B140F20851C2F200014FF0000421F879
:1041C000134040F22073C2F2000353E8004FA4F101
:1041D000010443E80045012DF7D053E8004FB4F146
:1041E000004F0DD14FF0000443E80045012DF4D0FD
:1041F0004EF60450CEF20000016841F0805101609B
:10420000BFF32F8F104630BC704700BF40F23863B9
:10421000C2F200031878D0F1010038BF00207047C7
:104220002DE9F84FDFF834814B4FC8EB07004FEA18
:10423000D00707F101074FF0000540F2982AC0F6B9
:10424000000A40F25839C0F6000931E044464FF008
:1042500000066FEA060B0BEB070101F0010B58F8A3
:10426000043CAB4229D135E054F8043CAB4205D1C3
:1042700054F8080C8047FDF72BFB0BE0FF2B09D906
:10428000FF2D07D154F8040C4FF0070154F8082C07
:1042900000F09CFF06F1010604F1080454F8041C28
:1042A000A94240D14CE005F10105B5F5807F02D06F
:1042B000CA45CBD3F7E7BDE8F88FFF2B0FD9FF2D09
:1042C0000DD158F8040C4FF0070158F8082C00F0F5
:1042D0007DFF04E058F8082C9047FDF7F9FA06F145
:1042E000010604F10804BE42DDD0BBF1000FBBD0D3
:1042F00054F8040CA8420AD0FF280DD9FF2D0BD189
:104300004FF0070154F8082C00F060FF04E054F867
:10431000081C8847FDF7DCFA06F1010604F10804E1
:10432000BE42A1D1BFE7FF290FD9FF2D0DD154F80F
:10433000040C4FF0070154F8082C00F047FF04E08C
:1043400054F8082C9047FDF7C3FA06F1010604F172
:104350000804BE4288D1A6E75F030008A002000857
:10436000027840F2ED63C2F200031B789A4206D352
:104370004FF000020270087800F1010008700A781E
:1043800040F2EE63C2F200031878824224BF00209C
:104390000870704710B5A0F10803052B3DD8DFE881
:1043A00003F01F3C2C3C038340F28C60C2F20000FF
:1043B0004FF020014FF0540210F036FA40F2E06066
:1043C000C2F200004FF0FF314FF00C0210F02CFA57
:1043D00040F2F460C2F20000026802F101020260E1
:1043E0004FF0000140F28863C2F20003197040F2FE
:1043F0008960C2F20000017056E040F28861C2F2AA
:1044000000014FF000030B7040F28960C2F200001F
:10441000027802F1010202703CE040F28862C2F2CE
:104420000002127840F28961C2F200010B7840F27A
:10443000ED61C2F20001097801FB032340F28C61B7
:10444000C2F20001C95C81421DD040F28C64C2F20C
:104450000004E0544FEA531040F2E061C2F2000160
:1044600003F01F034FF0010404FA03F351F8204056
:104470001C4341F8204040F2F460C2F200000168A1
:1044800001F10101016002F1010240F28863C2F210
:1044900000031A7040F28860C2F2000040F28961A5
:1044A000C2F20001FFF75CFF4FF0000010BD00BF3B
:1044B00070B4039D049C064628B140F2F060C2F23D
:1044C00000000078307029B140F2F860C2F20000BC
:1044D000007808702AB140F2EC61C2F2000108785D
:1044E00010702BB140F2F962C2F20002117819701B
:1044F0002DB140F28863C2F20003187828702CB105
:1045000040F28962C2F200021178217070BC7047DB
:1045100006281DD8002808BF052040F2F063C2F22B
:104520000003187047F23463C0F6010313F810104B
:1045300040F2ED62C2F20002117003EB40004178DC
:1045400040F2EE63C2F2000319704FF001007047B1
:104550004FF00000704700BF08B540F2F863C2F2A8
:1045600000034FF001021A704FF00500FFF7D0FF73
:104570004FF00C004FF00001FFF70CFF08BD00BF2B
:1045800008B540F28862C2F20002107040F28963FE
:10459000C2F20003197010461946FFF7E1FE08BD8C
:1045A000034628B140F2ED60C2F2000000781870B6
:1045B00029B140F2EE63C2F20003187808702AB104
:1045C00040F2F461C2F200010B68136040F28C60AB
:1045D000C2F20000704700BF2DE9F00140F28C6785
:1045E000C2F200073F1853284BD8002A49D03B4657
:1045F00007F1010702F1FF3257FA82F74FF0000688
:1046000040F2E064C2F200044FF001056FEA030CCF
:104610000CEB070202EA050C13F8018B01F1FF31E4
:1046200011F8012F90452FD13DE013F801CB01F196
:10463000010049788C450ED003F8011C4FEA521155
:1046400002F01F0605FA06FC54F821604CEA060643
:1046500044F821602E4602F10102D2B2542A07D05A
:1046600013F801CB00F101014078844542D150E0BC
:104670003EB140F2F463C2F20003196801F1010196
:104680001960BDE8F001704703F8012C4FEA50169D
:1046900000F01F0805FA08F854F8262048EA02023C
:1046A00044F826202E4600F10100C2B2542ADFD081
:1046B000BB42DDD0BCF1000FB7D013F801CB11F82D
:1046C000010F84450ED003F8010C4FEA521002F09E
:1046D0001F0605FA06FC54F820604CEA060644F86A
:1046E00020602E4602F10102D2B2542AC0D0BB4251
:1046F0009BD1BDE703F8010C4FEA521002F01F06F0
:1047000005FA06FC54F820604CEA060644F82060DE
:104710002E4602F10102D2B2542AA9D0BB4284D162
:10472000A6E700BF003018BF012040F2F863C2F2D4
:1047300000031870003118BF012140F2EC60C2F292
:1047400000000170003218BF012240F2F963C2F28A
:1047500000031A70704700BF40F2EF63C2F200031B
:104760004FF000021A7070474FF05400704700BFBE
:1047700040F2EF63C2F200034FF001021A7070477B
:10478000034628B10868834214BF00200120704707
:104790004FF00000704700BF10B440F22073C2F227
:1047A000000353E8002F02F1010243E80021012930
:1047B000F7D00468C4B16268824202D19268626034
:1047C00002E04368816899602368834202D15B6894
:1047D000236002E0826841685160A26802F1FF3103
:1047E000A1604FF00004046040F22073C2F20003A5
:1047F00053E8002FA2F1010243E80024012CF7D076
:1048000053E8002FB2F1004F0DD14FF0000243E802
:104810000024012CF4D04EF60450CEF200000168C2
:1048200041F080510160BFF32F8F10BC704700BF73
:1048300038B504460D464FF000014FF010020FF05E
:10484000F3FFE56038BD00BFF8B504460F46C66803
:104850008D192946FFF794FF00283CD140F22073C0
:10486000C2F2000353E8002F02F1010243E80021E5
:104870000129F7D04FF0000068606168A96001B1BC
:104880004D60226802B925606560BC51A36803F1E0
:104890000103A36040F22073C2F2000353E8002F2B
:1048A000A2F1010243E80024012CF7D053E8002FC5
:1048B000B2F1004F0DD14FF0000243E80024012C6B
:1048C000F4D04EF60450CEF20000016841F0805161
:1048D0000160BFF32F8FF8BD2DE9F04104468846F3
:1048E000C6688D199719C2B940F22073C2F200034D
:1048F00053E8002F02F1010243E800210129F7D01B
:1049000002686A6005604FF00000A860616809B93C
:10491000656020E06B689D601DE03946FFF730FF61
:1049200000283FD02846FFF737FF40F22073C2F23D
:10493000000353E8002F02F1010243E8002101299E
:10494000F7D0B868A8606F60BD602168B9420EBF3B
:104950002560A9684D6048F80640A26802F101028E
:10496000A26040F22073C2F2000353E8002FA2F1CC
:10497000010243E80024012CF7D053E8002FB2F1E4
:10498000004F0DD14FF0000243E80024012CF4D079
:104990004EF60450CEF20000016841F080510160F3
:1049A000BFF32F8FBDE8F081C368C918486808B10C
:1049B000C01A70474FF00000704700BF036813B182
:1049C000C068181A70474FF00000704708B5C368F8
:1049D000C918FFF7D5FE08BD08B5C0680818FFF76D
:1049E000DBFE08BD08B540F2FC60C2F200004FF0EB
:1049F0001C01FFF71DFF08BD70B5054600F1080654
:104A00003046FFF7DBFF0446686050B13046214670
:104A1000FFF7E2FF4FF00100A861204600F07EFAA8
:104A200070BD4FF00003AB6170BD00BF38B50446E8
:104A30000D464FF000014FF028020FF0F5FE204622
:104A400040F8085B4FF01C01FFF7F2FE40F2FC60FB
:104A5000C2F200002146FFF7F7FE38BD2DE9F04114
:104A60000746884643F26C43C2F2000318680028E8
:104A700000F0FE8040F22074C2F2000454E8002FDF
:104A800002F1010244E800210129F7D0796831B12F
:104A900043F26C42C2F20002136899422ED143F2F3
:104AA0006C40C2F2000004687C60B96901F1010148
:104AB000B96140F22073C2F2000353E8002FA2F163
:104AC000010243E80024012CF7D053E8002FB2F193
:104AD000004F0DD14FF0000243E80024012CF4D028
:104AE0004EF60450CEF20000016841F080510160A2
:104AF000BFF32F8F4FF00100BDE8F081B8F1FF3F09
:104B000024D140F22073C2F2000353E8002FA2F137
:104B1000010243E80024012CF7D053E8002FB2F142
:104B2000004F0DD14FF0000243E80024012CF4D0D7
:104B30004EF60450CEF20000016841F08051016051
:104B4000BFF32F8F4FF00000BDE8F08107F108059B
:104B50002846FFF733FF0246F0B143F26C46C2F23B
:104B60000006306892F8294090F829108C4208D944
:104B700012E0336892F8290093F82940A04204D942
:104B80000AE043F26C46C2F2000628461146FFF7DF
:104B90000BFF02460028ECD1284643F26C41C2F2DA
:104BA00000010968FFF798FE40F22076C2F2000685
:104BB00056E8002FA2F1010246E80024012CF7D0AC
:104BC00056E8002FB2F1004F0DD14FF0000246E839
:104BD0000024012CF4D04EF60450CEF200000168FF
:104BE00041F080510160BFF32F8FB8F1000F04D066
:104BF00008EB880000F028FB01E000F05DF940F2CE
:104C00002074C2F2000454E8003F03F1010344E8B9
:104C10000032012AF7D043F26C46C2F20006284661
:104C20003168FFF7D9FE54E8003FA3F1010344E8DF
:104C30000032012AF7D054E8003FB3F1004F0DD104
:104C40004FF0000344E80032012AF4D04EF604503D
:104C5000CEF20000016841F080510160BFF32F8F58
:104C600078683268904214BF00200120BDE8F081CE
:104C70004FF00100BDE8F08110B5044643F26C43EB
:104C8000C2F200031868002860D06268904201D028
:104C9000FBF7D4FC40F22073C2F2000353E8002F6C
:104CA00002F1010243E800210129F7D0A16901F1D5
:104CB000FF30A06118B340F22073C2F2000353E842
:104CC000002FA2F1010243E80024012CF7D053E8A1
:104CD000002FB2F1004F0DD14FF0000243E8002445
:104CE000012CF4D04EF60450CEF20000016841F0E1
:104CF00080510160BFF32F8F4FF0000010BD2046A0
:104D0000FFF77AFE40F22073C2F2000353E8002F4F
:104D1000A2F1010243E80024012CF7D053E8002F50
:104D2000B2F1004F0DD14FF0000243E80024012CF6
:104D3000F4D04EF60450CEF20000016841F08051EC
:104D40000160BFF32F8F4FF0010010BD4FF0010045
:104D500010BD00BFF8B5054640F22073C2F2000353
:104D600053E8002F02F1010243E800210129F7D0A6
:104D700040F2FC60C2F20000FFF720FE0446E0B102
:104D800040F2FC67C2F200076068A84203D12046E7
:104D9000FFF732FE0AE004F1080630462946FFF725
:104DA00015FE18B130462946FFF716FE3846214653
:104DB000FFF7FAFD04460028E6D140F22073C2F264
:104DC000000353E8002FA2F1010243E80024012C64
:104DD000F7D053E8002FB2F1004F0DD14FF0000291
:104DE00043E80024012CF4D04EF60450CEF200002B
:104DF000016841F080510160BFF32F8FF8BD00BF03
:104E000008B547F24063C0F60103195C012906D0DA
:104E100011B102290BD105E0FDF7FCFF08BD02F03E
:104E200001F908BDFBF70AFC4FF0000008BD4FF088
:104E3000000008BD4EF60453CEF200031A6842F09B
:104E400080501860704700BF4FF0010280F82820A2
:104E500040F21C73C2F2000390F8291002FA01F22A
:104E6000188802431A80704710B440F21873C2F2D7
:104E700000031A68C2B1904213D104E088420FD1F6
:104E800002F1140203E040F21872C2F20002436918
:104E90001BB19C698169611899614369136003E0E2
:104EA0000A4651690029E9D14FF0000282614FF0B2
:104EB000FF31416110BC704710B5FBF767FC044639
:104EC00043F26C43C2F20003186890F82820032ACA
:104ED0001BD0FBF75BFC43F26C43C2F20003196882
:104EE0004FF0000281F8282091F82920096940F646
:104EF0000C03C2F2000343F82210FBF751FC2046DA
:104F0000FBF74EFCFFF796FF10BD4FF0020180F853
:104F100028102046FBF744FC10BD00BF38B50446FE
:104F200090B3036883B3FBF731FC054694F828007F
:104F300010BB2046FFF788FF43F26C41C2F200012C
:104F40000B6843B194F8292093F8290020F001015F
:104F5000531A002B15DA40F22072C2F200021068D8
:104F600038B140F0004140F22073C2F200031960F2
:104F700007E0FFF75FFF04E0022804BF032084F886
:104F800028002846FBF70CFC38BD00BF2DE9F04F88
:104F900085B006460F46934698460F9DDDF8409033
:104FA000FBF7F4FB824640F26473C2F20003196817
:104FB000504881420FD248F20002C2F2000252F879
:104FC0002C4C54B14C4B1C468B4207D953F82C093E
:104FD0000028F8D102E0474C00E0464CA14206D13F
:104FE000A1F12C0140F26472C2F20002116020466D
:104FF0004FF000014FF02C020FF016FC4FF0FF3184
:1050000061611EB947F24466C0F601062660B8F138
:10501000000F08D00E9B042B08D9184600F103009E
:105020004FEA900604E04FF0000601E04FF0000662
:105030000DBB43F67079C2F2000940F20C75C2F262
:105040000005296845F2A940C0F600000090CDF89F
:105050000480029648464FF000025B46FBF7CEFE06
:105060002A68A260E0604FEA800153182B60C1EB10
:105070000900606020E028464FF0FF314A46FBF708
:105080003FFB4AF2ED52CDF6CE622A60E56005EBB9
:105090008905656045F2A941C0F600010091CDF88F
:1050A00004800296284629464FF001025B46FBF732
:1050B000A5FEA5EB800363606FEA0702C2F3C0118F
:1050C00001EB470707F0FF0784F8297040F22473CB
:1050D000C2F2000353F82700206143F827405046EE
:1050E000FBF75EFB2046FFF719FF204605B0BDE841
:1050F000F08F00BFD47F0020A87F002030B585B09E
:105100004FF0000143F26C43C2F200031960284CD7
:1051100048F20005C2F200052A1B20464FEAA2020F
:10512000FBF7EEFA40F20C70C2F200000460A5F149
:105130002C0540F26471C2F200010D6043F27073FD
:10514000C2F200034FF0B504CBF26B141C6003F104
:105150004C004FF0FF3243F8042F43F8042F43F87C
:10516000042F8342F9D14FF00004009440F268719B
:10517000C2F2000101914FF02803029347F2506000
:10518000C0F601004FF0070145F22922C0F60002E7
:105190002346FFF7FBFE40F60802C2F20002106051
:1051A00040F22470C2F20000C46305B030BD00BFFD
:1051B000743F002010B584B0069C00944FF00004AA
:1051C00001940294FFF7E2FE04B010BD00B585B073
:1051D0004FF00003009301930293FFF7D7FE05B051
:1051E00000BD00BF38B543F26C43C2F2000318683B
:1051F000C0B1FBF7CBFA054643F26C44C2F200049F
:105200002068FFF721FE216891F82920086940F6FF
:105210000C03C2F2000343F822002846FBF7C0FA51
:10522000FFF708FE38BD00BF38B543F26C45C2F247
:10523000000540F22474C2F200042B6822681A614F
:10524000FFF7D0FFF9E700BF38B543F26C43C2F275
:1052500000031968002900F0918020B9FFF7C2FF10
:105260004FF001029AE0B0F1FF3F04D1FFF724FEB6
:105270004FF0000292E040F22074C2F2000454E8C1
:10528000002F02F1010244E800210129F7D040F289
:105290001872C2F200021568002D7AD0AB699842EC
:1052A0006FD3C01A05F114016D691DB1AB6983425A
:1052B000F7D96AE043F26C45C2F200052B689861A9
:1052C000086858611846FBF7BDF940F22074C2F235
:1052D000000454E8003FA3F1010344E80032012A2E
:1052E000F7D054E8003FB3F1004F0DD14FF0000369
:1052F00044E80032012AF4D04EF60450CEF2000009
:10530000016841F080510160BFF32F8FFFF7D4FD9A
:1053100054E8003F03F1010344E80032012AF7D0CA
:1053200028684169B1F1FF3F04D0FFF79DFD4FF0C0
:10533000000201E04FF0010240F22073C2F20003CC
:1053400053E8004FA4F1010443E80045012DF7D0D4
:1053500053E8004FB4F1004F0DD14FF0000443E883
:105360000045012DF4D04EF60450CEF20000016845
:1053700041F080510160BFF32F8F0FE04FF0010229
:105380000CE040F21871C2F20001AC69221AAA6165
:1053900090E740F21871C2F200018BE7104638BD69
:1053A000F8B5044600287AD0FBF7F0F9064640F23B
:1053B0006473C2F2000319683948814211D248F27D
:1053C0000002C2F2000252F81C5CA54263D0354BC9
:1053D0001D468B4205D9A3F12C03D86BA042F7D10F
:1053E0005AE094F8293040F22472C2F2000252F8D6
:1053F0002300A04206D1016940F22472C2F20002E9
:1054000042F823102046FFF72FFD2046FFF7A2FCAD
:1054100094F82900236940F60C01C2F2000141F81A
:10542000203043F26C42C2F200021068A04229D040
:10543000A06838B3E76800EB870540F20C77C2F24A
:1054400000073B685A1B29464FEAA2024FF00003AF
:10545000FCF73AFFE1683868A0EB81033B6040F25B
:105460006472C2F2000211680D4B99420AD29A6826
:10547000954203D8E068A2EB80029A60A3F12C0366
:105480008B42F4D84FF00001216084F82810304698
:10549000FBF786F9F8BD024D21692961A1E7F8BD46
:1054A000D47F0020A87F002000BFF04772B643F2EF
:1054B0006C44C2F200042068FFF772FF4FF0000353
:1054C0002360FBF7EBFC00BF40F21873C2F200034D
:1054D000196849B1886950B100F1FF328A61D2F18F
:1054E000010038BF002070474FF0000070474FF0B8
:1054F0000000704770B540F21873C2F200031C68D8
:10550000A4B1A06990B940F21875C2F200054FF03D
:10551000FF3660692946FBF795F866612046FFF77C
:10552000FDFC2C6814B1A1690029F2D070BD00BF48
:10553000F0B472B640F21C73C2F200031C882CB99E
:1055400040F60803C2F2000318685FE047F2586CA7
:10555000C0F6010C40F60C05C2F2000540F22476BC
:10556000C2F20006C4F1000323401A0A1ABF1CF855
:10557000021008311CF8031011F0010F0AD141F09C
:10558000010055F8200038B190F82820012A38D8B9
:105590001F4602E01F4600E01F4655F82120B2B129
:1055A00092F828307BB140F21C70C2F200000480F7
:1055B00010462BE090F8283033B140F21C72C2F252
:1055C0000002148022E0104600690028F2D156F84B
:1055D0002100824207D1BC43C4D140F21C71C2F207
:1055E00000010C80ACE745F8210011F0010FD4D187
:1055F00014EA4703D1D04FEA4707BFB241F0010197
:10560000CBE740F21C71C2F200010C8062B6F0BC24
:10561000704700BF70B543F26C43C2F200031B68D1
:1056200083420FD193F82820012A9CBF022283F8DD
:10563000282093F8291040F60C00C2F2000040F830
:10564000213070BD40F21072C2F20002136043F2CA
:105650006C41C2F20001086090F8292040F60C036A
:10566000C2F2000343F8220090F8281001299CBFE1
:10567000022180F828108268AAB9C1684AF2ED5365
:10568000CDF6CE630868984201D0FAF7D7FF43F20F
:105690006C42C2F2000211684868CB6898427ED220
:1056A000FAF7CCFF70BD40F21473C2F200031B681E
:1056B000984274D093B3586843F67074C2F20004F1
:1056C000251A4FEAA501D96043F27072C2F20002B6
:1056D00090420AD34FF0B503CBF26B1343F27070D4
:1056E000C2F2000004689C4201D0FAF7A7FF40F222
:1056F0001475C2F200052A6840F20C74C2F200046C
:1057000020685168D2684FF00003FCF7DDFD29687E
:1057100023688B60C86803EB8002226043F26C410F
:10572000C2F200010B6840F21470C2F20000036084
:10573000DA68002A33D0586899684FF00103FCF703
:10574000C3FD43F26C46C2F200063568A868EC68F7
:1057500000EB840440F20C76C2F200063268131BA0
:1057600021464FEAA3024FF00003FCF7ADFDE968C4
:105770003068A0EB8102326040F26473C2F2000331
:105780001968074B99420AD29A68944203D8E8688C
:10579000A2EB80029A60A3F12C038B42F4D870BD77
:1057A000D47F002000B585B040F6A810C2F20000FA
:1057B0004FF00001FFF73CF840F65000C2F2000045
:1057C0004FF00001FFF734F84FF00003009340F66C
:1057D0006802C2F2000201924FF05000029047F2BC
:1057E0005870C0F60100194645F6F922C0F60002CD
:1057F000FFF7CCFB40F64C03C2F20003186005B083
:1058000000BD00BF08B5FFF7D9F8034648B1C0682E
:1058100050B100F1FF31D960D1F1010038BF002053
:1058200008BD4FF0000008BD4FF0000008BD00BFEC
:1058300070B505460E46144640F22073C2F20003CE
:1058400053E8002F02F1010243E800210129F7D0BB
:10585000FFF7B4F80246002839D0C06884422DD33F
:10586000241A28461146FFF79FF8024600282ED03A
:10587000C068A042F4D921E040F22073C2F20003D4
:1058800053E8002FA2F1010243E80024012CF7D0D5
:1058900053E8002FB2F1004F0DD14FF0000243E862
:1058A0000024012CF4D04EF60450CEF20000016822
:1058B00041F080510160BFF32F8F70BDF460D1685B
:1058C0000B1BD36028463146FFF706F8D4E7F46097
:1058D00028463146FEF7B8FFCEE700BFF8B50646CA
:1058E000FFF76CF80446F8B1C368EBB930462146BF
:1058F000FFF75AF80546FAF749FF074630462146B2
:10590000FFF76AF83846FAF74BFF22691AB13046BA
:105910002146FFF78DFF04F11400FDF7C9FF1DB10B
:105920002C46E8680028E1D0F8BD00BF08B540F675
:105930006403C2F200031A6802F101021A6040F621
:105940005000C2F20000FFF75DFF28B140F65000A2
:10595000C2F20000FFF7C2FF08BD00BF08B5014654
:1059600040F6A810C2F20000FFF730F820B140F670
:10597000A810C2F2000008BD40F65000C2F20000BC
:1059800008BD00BF70B5044640F22073C2F20003A8
:1059900053E8002F02F1010243E800210129F7D06A
:1059A000FFF7DCFF05462146FFF710F8002845D039
:1059B00040F22070C2F2000050E8002F02F1010214
:1059C00040E800210129F7D028462146FEF7ECFFE8
:1059D00018B1C168E2688B18C360FAF7D7FE0646B3
:1059E00028462146FEF7F8FF3046FAF7D9FE4FF079
:1059F000FF35E56040F22073C2F2000353E8002F48
:105A0000A2F1010243E80025012DF7D053E8002F51
:105A1000B2F1004F0DD14FF0000243E80025012DF7
:105A2000F4D04EF60450CEF20000016841F08051EF
:105A30000160BFF32F8F4FF0010501E04FF000052B
:105A400004F11400FDF72EFF40F22073C2F20003B0
:105A500053E8002FA2F1010243E80024012CF7D003
:105A600053E8002FB2F1004F0DD14FF0000243E890
:105A70000024012CF4D04EF60450CEF20000016850
:105A800041F080510160BFF32F8F284670BD00BFE9
:105A90002DE9F04105460F4614469846FFF772FF80
:105AA000064694B19DF82030002B14BF20460020FC
:105AB000286105F114004146069A079BFDF7D8FEC0
:105AC000384629462246FFF7B3FE3046BDE8F0814E
:105AD00070B584B00E4615460093089C01949DF85D
:105AE0002430029340F6A811C2F2000132462B4640
:105AF000FFF7CEFF04B070BD00B583B04FF00003D8
:105B000000934FF00100019040F6B810C2F200007F
:105B100041F288314FF0FF0245F62D13C0F6000325
:105B2000FFF7D6FF40F6A814C2F20004FFF7E2FC2C
:105B30002046FFF7D3FEFFF7BFF9F7E740F6600313
:105B4000C2F2000318681A689042FBD1704700BF88
:105B500010B540F66003C2F200031A6802F10102B8
:105B60001A60FFF7B1FC044640F6A810C2F200002C
:105B7000FFF748FE204310F0FF0F06D040F64C0020
:105B8000C2F200000068FFF7C9F910BD08B547F27E
:105B90008C70C0F601004FF0060145F6C972C0F6E0
:105BA0000002FFF713FB40F6E013C2F20003186097
:105BB00008BD00BF38B504460D4640F62023C2F2AA
:105BC0000003586AA0420AD040F62021C2F2000128
:105BD0004C620A681AB115B14948FDF769FE40F6F2
:105BE0002023C2F20003186F84420AD040F620211D
:105BF000C2F200010C67CA6C1AB115B14148FDF739
:105C000057FE40F62023C2F20003D3F8BC008442C2
:105C10000CD040F62021C2F20001C1F8BC40D1F8FE
:105C200098201AB115B13848FDF742FE40F62023FE
:105C3000C2F20003D3F8080184420CD040F62021C0
:105C4000C2F20001C1F80841D1F8E4201AB115B13F
:105C50002E48FDF72DFE40F62023C2F20003D3F8B4
:105C6000540184420CD040F62021C2F20001C1F858
:105C70005441D1F830211AB115B12548FDF718FE6D
:105C800040F62023C2F20003D3F8A00184420CD0D6
:105C900040F62021C2F20001C1F8A041D1F87C21D8
:105CA0001AB115B11B48FDF703FE40F62023C2F2DE
:105CB0000003D3F8EC0184420CD040F62021C2F25C
:105CC0000001C1F8EC41D1F8C8211AB115B1124850
:105CD000FDF7EEFD40F62023C2F20003D3F83802B0
:105CE000A0420CD040F62021C2F20001C1F8384297
:105CF000D1F814221AB115B10848FDF7D9FD38BD05
:105D0000300A00207C0A0020C80A0020140B002062
:105D1000600B0020AC0B0020F80B0020440C00208E
:105D20002DE9F04707460D4691460898DDF8288092
:105D30000C683E68D8F800108A19944202D80219FB
:105D4000964203D304192C60BDE8F087341B061B70
:105D5000B14234BF8A46B246099931B1D9F8000040
:105D60000818191952460EF03BFDD8F80030CAEB5E
:105D70000302C8F800203E6806EB0A013960D9F832
:105D8000000000EB0A03C9F800302E68A41954443F
:105D90002C60BDE8F08700BF70B584B09CF8196036
:105DA000157A947B4FF007038CF810304FF0050202
:105DB0008CF8112006F00F0260F3C7128CF8122045
:105DC0004FF0000065F301008CF813004FF0000263
:105DD00061F30A02ACF814208CF81640DCF80C10C1
:105DE0000093DCF804300193CDF808C001F1040001
:105DF0000CF108020CF11003FFF792FF04B070BD24
:105E00002DE9F04F8FB00746059114464FF000037F
:105E10000793136012896068131A8B4238BF059389
:105E20000599002900F0AA8040F61825C2F2000565
:105E30002D6815B34FEAC5054FF000024FF0FF0182
:105E4000134640F6D440C2F20000A5F10806C6F39E
:105E5000C00E1658F6798E4240F0958096E016589E
:105E6000F6798E421CBF0133314602F10802865892
:105E7000F6798E4240F09F80A0E04FF0000303EBE4
:105E800043024FEAC20000F1100008904FF4807105
:105E9000ADF824104FF00402ADF826208DF828301C
:105EA0000DF129004FF000014FF007020EF0BCFC8D
:105EB00004F1040B04944FF010030093019705A81C
:105EC00002905846214607AA08ABFFF729FF05991B
:105ED000002951D04FF001028DF821200DF1320040
:105EE0004FF000014FF006020EF09EFC40F6182322
:105EF000C2F20003186800283ED04FF0FF014FF0B7
:105F0000000440F6D449C2F2000947F29C78C0F67A
:105F1000010840F6182AC2F2000A59F83450ED7907
:105F20008D4223D08DF820404FEA05160DF1220056
:105F300008EB06014FF008020EF052FC06F10801D2
:105F40000DF12A0041444FF008020EF049FC4FF0D9
:105F500018020092019705AB02935846049907AACC
:105F600008ABFFF7DDFE059830B1294604F10104C6
:105F7000DAF80020A242D0D8079801E04FF0FF30B5
:105F80000FB0BDE8F08F03F10103314602F10802C2
:105F9000AA423FF474AFBEF1000F3FF460AF165851
:105FA000F6798E421CBF0133314602F10802AA4243
:105FB0007FF455AF63E703F10103314602F10802B4
:105FC000AA427FF44CAF5AE72DE9F0414FF00100AF
:105FD000FDF766FB47F27C70C0F60100FDF7DCF9C7
:105FE00040F6DC13C2F200034FF001021A7040F6D3
:105FF0000820C2F20000016841B940F60824C2F24C
:106000000004FEF759FF2568002DFAD040F60E2750
:10601000C2F2000740F6DC14C2F2000440F60D267E
:10602000C2F2000640F68145C2F2000540F6E418CF
:10603000C2F200083B783BB14FF000023A704FF0DB
:1060400002002070FDF774F9317859B14FF0000368
:106050003370227862F07F0020704FF0010001461B
:10606000FFF7A8FD297851B14FF000002870237880
:1060700003F07F0222704FF00101FFF79BFD98F8BB
:10608000000010B9FEF718FFD4E740F6DC11C2F2A9
:1060900000014FF002030B704FF00000FDF700FB12
:1060A000BDE8F08108B540F60823C2F2000318608D
:1060B00040F6E010C2F200000068FEF72FFF08BDB6
:1060C00070B505460E4640F61C23C2F20003186860
:1060D000032801D9FAF7B2FA40F61C22C2F20002F4
:1060E000116840F6E814C2F2000444F8316004EB91
:1060F000C104656001F10101116070BD70B5054614
:106100000C461646032801D9FAF798FA40F6D4430C
:10611000C2F2000353F8350008B1FAF78FFA40F6DF
:10612000D441C2F2000141F8354001EBC5056E6073
:1061300040F61823C2F200031A6802F101021A6045
:10614000206930B1FDF728F904F104042069002822
:10615000F8D170BD08B540F62023C2F200031968DB
:1061600081425AD040F62022C2F20002D36C834210
:1061700034D040F62021C2F20001D1F898208242AA
:106180002FD040F62023C2F20003D3F8E41081425E
:106190002AD040F62022C2F20002D2F830318342E7
:1061A00025D040F62021C2F20001D1F87C218242A4
:1061B00020D040F62023C2F20003D3F8C811814258
:1061C0001BD040F62022C2F20002D2F814328342E1
:1061D00016D0FAF733FA4FF0080013E04FF0010041
:1061E00010E04FF002000DE04FF003000AE04FF026
:1061F000040007E04FF0050004E04FF0060001E066
:106200004FF0070040F62021C2F200014FF04C028F
:1062100002FB001090F8200008BD4FF00000F1E7ED
:106220002DE9F04F8FB0089007910A924FF00003CC
:1062300009931360546813891B1B8B4238BF079363
:106240000799002900F04A81082C69D840F61824E3
:10625000C2F20004D4F800E040F61C25C2F20005AA
:106260002E680EEBCE0707EBC60404F109044FF0CD
:10627000000140F6D447C2F20007CB598BB1DD686C
:10628000641903F110051B695BB15E890EB104F15D
:1062900007049B890BB104F1070455F8043F002B58
:1062A000F3D101F108012029E7D140F60821C2F21B
:1062B00000010D682F7E6E7EEB8A03F10103C3F3AC
:1062C00047054FF000010C914FF009038DF82C3079
:1062D0004FF002018DF82D10ADF82E408DF830E012
:1062E0004FF001018DF831104FF0000167F34511B7
:1062F00066F3861161F07F018DF833108DF834500C
:106300000093019007A8029002F10400114609AA27
:106310000BABFFF705FD079A002A00F0DD80E0E0F7
:106320004FF009001060DCE05BF83640002C00F014
:10633000CE80059D286800284BD07A68B2420CD0E8
:106340004FF0000310F0010F3ED1DFE007EBC30276
:106350005268B24240F0E38001E04FF0000357F88A
:106360003300D2B290F8048090F805C090F806E0AF
:10637000C579016819B143F01000C3B201E04FF0D4
:1063800000034FF008008DF82C004FF00B018DF842
:106390002D108DF82E208DF82F808DF830C08DF8BF
:1063A00031E08DF832508DF833300A990090089A18
:1063B000019207AB029301F1040009AA0BABFFF7AE
:1063C000AFFC079828B987E003F101052B46854209
:1063D000BCD104F1100523697BB129464FF00002BE
:1063E000588908B102F101029B890BB102F1010247
:1063F00051F8043F002BF3D101E04FF000025FFAA7
:1064000086FCD2B294F804E06079A17923681BB1CC
:1064100046F02003DBB201E04FF000038DF82CA022
:106420004FF004088DF82D808DF82EC04FF0000C31
:106430008DF82FC08DF830208DF831E08DF83200C6
:106440008DF833108DF834300A99CDF800A0089AF1
:10645000019207A8029001EB080009AA0BABFFF715
:106460005FFC0799002937D0A3686BB10A99E268ED
:1064700000920898019007AA029201EB080009AA6D
:10648000FFF74EFC079B3BB3246904B34FF00108B0
:106490004FF000092046FFF75DFE8DF83500618959
:1064A00039B10DF11C0C40462246FFF775FC0799E7
:1064B00091B1A18939B10DF11C0C48462246FFF774
:1064C0006BFC079840B155F8044F002CE2D106F15F
:1064D0000106042E7FF428AF099814E04FF0FF3036
:1064E00011E04FF0000640F6D44BC2F2000B40F62C
:1064F0001C24C2F2000405944FF0090A40F6E81784
:10650000C2F2000710E70FB0BDE8F08F03F10103FE
:1065100007EBC3014A68B2427FF456AF1FE705F1AB
:10652000010307EBC3014A68B2427FF44DAF16E79F
:1065300008B540F68443C2F200031A5C40F62021FD
:10654000C2F200014FF04C0000FB0210436AD3F18D
:10655000010238BF002242634FF00001C1630164B1
:10656000416400F11000FDF7A3F908BD2DE9F047E3
:1065700090B081468A4640F68443C2F200031A5C1A
:1065800040F62020C2F200004FF04C0404FB02044D
:1065900004F148064FF001084FF000073546404629
:1065A0003146FAF74FF828B14FF002003146FAF7BA
:1065B00049F836E0BAF1000F05D148464146FCF7EC
:1065C0008BFD032827D0256C75B16846A168E26B66
:1065D000A8470546B0F1FF3F14D0606448466946BD
:1065E0002A46FCF7B1FD0EE0616CA5688D4228BF1C
:1065F0000D464846E16B2A46FCF7A6FDE36B5A19A7
:10660000E26300E03D46606CA16888423CBFE763FE
:106610002764451B656438463146FAF713F80228AB
:10662000BCD010B0BDE8F087F8B505460E46174659
:1066300040F68443C2F200031A5C40F62020C2F206
:1066400000004FF04C0404FB02044FF00000FCF784
:1066500039FDE76326644FF00001616428464FF07E
:106660000101FFF783FF4FF00100FCF72BFDF8BDA0
:10667000F8B505460F46164640F68443C2F20003BD
:106680001A5C40F62020C2F200004FF04C0404FBDC
:106690000204A168B1420DD243F27073C2F200034A
:1066A0009F4207D343F67072C2F20002974201D2B2
:1066B000F9F7C4FF4FF00000FCF704FDE7634FF06B
:1066C00000002064666428464FF00101FFF74EFF8A
:1066D0004FF00100FCF7F6FCF8BD00BF08B5FCF771
:1066E000ABFD08BD70B586B005460C46164602A83F
:1066F000FAF7F6FF01462EB102A82A46234600F01B
:106700009BFD07E04FF00103009302A82A462346B1
:1067100000F044FE06B070BD70B58AB00378212B3E
:1067200000F0938004D86BB1012B40F0D88186E053
:10673000A12B00F0A781C02B00F0B481802B40F08A
:10674000CE8195E04178052903D0092940F0CA811E
:1067500046E0408840F6DC12C2F200021378022BB9
:1067600002D0032B33D118E000F1FF318AB27E2A28
:1067700030D8C0B240F68043C2F2000318704FF028
:106780000201FCF781FF40F6DC10C2F200004FF07E
:10679000030101704FF00100C3E170B940F680427F
:1067A000C2F20002107040F6DC10C2F200004FF09E
:1067B000020303704FF00100B3E17F280DD840F6CB
:1067C0008041C2F2000108704FF00100A9E14FF0D2
:1067D0000200A6E14FF00200A3E14FF00200A0E1A9
:1067E000827840F6DC13C2F200031978022923D91B
:1067F00072B940F6DC13C2F200034FF003011970C6
:106800004FF001000146FFF7D5F94FF0010088E194
:10681000012A18BF022040F0848140F6DC10C2F249
:1068200000004FF0040202704FF000000146FFF735
:10683000C1F94FF0010074E14FF0020071E14078BE
:106840000B280CBF012002206BE18388032B00F290
:106850004C8140F6D444C2F2000404EBC3035B68ED
:10686000002B00F045819847002808BF022058E11E
:1068700042781AB1062A40F03E8121E0C1880229FF
:106880001BD14FF00000ADF8040040F60822C2F220
:10689000000212680346517E61F30003ADF8043034
:1068A000127E62F341030AA921F8243D4FF002024F
:1068B000FFF7DEFE4FF0030033E14FF0020030E15E
:1068C0008278C1888CB2C378022B2ED0032B3DD0A6
:1068D000012B40F0D48040F69445C2F200052846D2
:1068E00047F26871C0F601014FF012020DF078FF17
:1068F00040F60820C2F2000001688A892A81CB890B
:106900006B81088AA8818A7C2A71CB7C6B71097D96
:10691000A9714FF000002946122C34BF22461222E2
:10692000FFF7A6FE4FF00300FBE040F6F442C2F290
:10693000000211814FF00000506046F22121C0F6A4
:106940000001FFF771FE4FF00300EAE0D2B940F614
:106950009444C2F2000404F1020047F26471C0F6EC
:1069600001014FF002020DF03BFF4FF004022270D4
:106970004FF0030565704FF000002146FFF778FEE9
:106980002846CEE0012A06D140F60823C2F20003D1
:10699000196809682FE0022A06D140F60822C2F2DF
:1069A00000021068416826E0032A06D140F6082359
:1069B000C2F20003196889681DE002F00F0022F09E
:1069C0000F03102B08D15A4B196888420EDA594A26
:1069D00052F8300001680EE0202B07D1032805D8BB
:1069E000554951F8300008B1016804E0EE2A04D09E
:1069F0004FF0020095E009B93EE05049B1F1FF3F88
:106A000040F0888001A84FF020014FF00102FFF70D
:106A100069FE0AAD2A184FF0000002F8240C01A903
:106A200078E000F10206428003F10102134611F8FA
:106A3000015F5DB100F10400758002F1010311F8FE
:106A4000012F002A6FD101E04FF0000340F694417E
:106A5000C2F200014FF003054D7003F101034FEA4C
:106A60004303DAB20A704FF00000A24228BF224668
:106A7000FFF7FEFD284654E04FF0020051E04FF0D2
:106A800002004EE08388032B38D840F6D444C2F28B
:106A9000000404EBC3035B689BB39847002808BF5E
:106AA00002203EE04378212B2ED1C18840F6F443EA
:106AB000C2F2000319814FF000025A608088042856
:106AC00025D1104645F60161C0F6000140F6F442BA
:106AD000C2F20002FFF7A8FD4FF0030021E04FF0E3
:106AE00002001EE04FF002001BE04FF0020018E031
:106AF0004FF0020015E04FF0020012E04FF00200EC
:106B00000FE04FF002000CE04FF0020009E04FF000
:106B1000020006E00A78002A96D009484FF00003E8
:106B20007FE70AB070BD1E2B7FF47BAF8EE700BFFE
:106B30001C0A0020E8090020D40C002090770108EE
:106B4000940C002010B50446436993B14FF0000047
:106B5000606140F6DC11C2F200010A78032A08D114
:106B600040F68043C2F2000318784FF00301FCF7AF
:106B70008BFD206958B34FF000002061E06040F6C3
:106B80000C21C2F20001087040F61021C2F200018F
:106B90004FF00802FFF7A2FD082853D140F610225B
:106BA000C2F20002137813F0800F06D140F61020D5
:106BB000C2F20000C188002944D140F61020C2F280
:106BC00000004FF000010A46FFF7A6FD2DE0E16846
:106BD000002937D04FF00000E06040F60C22C2F2EE
:106BE0000002137840F69441C2F20001C3F1400262
:106BF000FFF774FD034628B340F60C20C2F20000F4
:106C000001785A18D2B2027040F61023C2F2000383
:106C1000D888904216D140F61020C2F2000040F60B
:106C20009441C2F20001FFF777FD012804D0022849
:106C300008D1FCF76FFA10BD4FF000000146024684
:106C4000FFF716FD10BD00BF08B540F60053C2F2B5
:106C500000031B693BB14FF0000140F60052C2F245
:106C600000025269984740F60050C2F200004FF00F
:106C70000001017041608160C1600161416108BD36
:106C800040F60050C2F20000816147F6BC01C0F638
:106C900001018A5C42778377037F6FF307030377F1
:106CA0004FF000014162704730B583B040F60054A8
:106CB000C2F200042070089D6560099DA5600A9DD0
:106CC000E5600B9D25610C9D65619DF81840009461
:106CD0009DF81C400194FFF7D3FF03B030BD00BF07
:106CE00040F60053C2F200035B6AB3F1FF3F09D1E3
:106CF00040F60051C2F200014FF000034B624FF02A
:106D0000010070473F2B0BD840F60052C2F2000240
:106D1000106AC15403F1010353624FF00100704740
:106D20004FF00000704700BF704700BF70B540F6DD
:106D30000054C2F2000404F1180047F6F401C0F652
:106D400001014FF007020DF04BFD4FF0000047F638
:106D5000C001C0F60101FFF7B3F946F68976C0F627
:106D600000064FF0000047F66C01C0F60101324604
:106D7000FFF7C4F947F6C805C0F601054FF001005A
:106D800029463246FFF7BAF92869FFF7E3F984F894
:106D9000280040F62C50C2F200004FF0070146F6E2
:106DA000B152C0F600024FF00003FCF761FD70BD68
:106DB00038B540F66053C2F200034FF001021A707A
:106DC00040F60054C2F2000494F828004FF000018D
:106DD0000A46FFF74DFC606868B140F60054C2F205
:106DE00000044FF0FF356562636820786169984759
:106DF000616A0029F7D040F60050C2F200004FF05F
:106E000000024262836833B140F60051C2F20001D1
:106E100008784969984738BD2DE9F047A2B0804607
:106E200043680BB9806828B14FF00001C8F808101A
:106E3000FFF7BEFFD8F80C20002A3ED04FF0000725
:106E4000C8F80C70D8F8000012A94FF04002FFF704
:106E500045FC074640F60053C2F20003D86860B311
:106E60005FB340F60054C2F200044FF0000507F192
:106E7000FF3606F0010A20789DF848102A4663691B
:106E8000E668B0474FF001094F456CD115E0E66860
:106E9000207812AA12F809102A466369B04709F14E
:106EA0000109E668207812AB13F809102A466369D5
:106EB000B04709F101094F45E9D1D8F8140000287D
:106EC0004ED04FF0000440F66051C2F200010C7049
:106ED000C8F8144040F63C50C2F20000FEF752FDE4
:106EE00040F60052C2F2000254625368002B30D0C8
:106EF00040F60055C2F2000502AC2C622C46656AD1
:106F00006268207861699047606A8542F7D105B36D
:106F1000D8F8000002A92A46FFF7AAFB4FF00001AB
:106F20000091019140F63C50C2F200004FF04B013D
:106F30004FF0FF0246F6B153C0F60003FEF7C8FD5E
:106F40000EE040F60052C2F20002107851699847F4
:106F500006E040F60053C2F200039B68002BF0D11C
:106F600022B0BDE8F087BAF1000F90D0E668207833
:106F700012A911F809102A466369B04709F10109FD
:106F80004F4584D199E700BF10B544780378212B91
:106F900002D0A12B19D10CE0202C02D0222C08D138
:106FA00019E0072A1AD10F480DF01AFC4FF0010022
:106FB00010BD212C0CD14FF000000A494FF0070200
:106FC000FFF756FB4FF0030010BD4FF0000010BD5F
:106FD0004FF0000010BD4FF0010010BD4FF0020057
:106FE00010BD00BF180D002008B540F66053C2F276
:106FF0000003187870B940F60051C2F200014A6AE5
:1070000072B940F60053C2F2000393F82800FFF76C
:107010008FFA08BD40F62C50C2F20000FCF748FC85
:1070200008BD00BF47F63C00C0F60100704700BF36
:1070300070B4037801298CBF4478002402298CBFE6
:1070400085780025DCF8000048B34FEA930647F640
:10705000FC10C0F60100365C16704FEA031343EAD9
:10706000141303F03F031B5C5370012907D94FEA47
:10707000840444EA951303F03F04205C01E04FF0E0
:107080003D009070022907D905F03F0547F6FC1333
:10709000C0F60103E95C01E04FF03D01D17070BC26
:1070A000704700BF82B04FF009010CE00191019BD5
:1070B00003F1FF32019233B100BF019B03F1FF32B4
:1070C0000192002BF8D100F1FF30B0F1FF3FEDD17C
:1070D00002B0704770B4C4B24FEA102047F6902651
:1070E000C0F6010647F6FC05C0F6010511F8013BA4
:1070F0001AB94BB944EA00200BE06340F45C444009
:10710000E85C013AF2D1F5E76340F45C4440E85CA6
:10711000ECE770BC704700BF10B444F6FB43C0F20C
:10712000861311F8014B02B9ACB380EA04404FEA70
:10713000400010F0807F18BF58404FEA400010F028
:10714000807F18BF58404FEA400010F0807F18BF82
:1071500058404FEA400010F0807F18BF58404FEA77
:10716000400010F0807F18BF58404FEA400010F0F8
:10717000807F18BF58404FEA400010F0807F18BF52
:1071800058404FEA400010F0807F18BF5840002A56
:10719000C7D0013AC5D120F07F4010BC704700BF76
:1071A00082B001909DF806304FF0000063F30700B5
:1071B0009DF8052062F30F209DF8042062F317402C
:1071C0009DF8072012F0800F14BF63F07F0103F0D9
:1071D0007F0161F307004FEA4201CAB262F31F6008
:1071E00013F0800F18BF42F0010262F31F6002B07B
:1071F000704700BF84B0C0F307438DF80C30C0F374
:1072000007228DF80D20C3B24FEA10604FEA5002FA
:1072100010F0010F14BF63F07F0103F07F018DF8C0
:107220000E1013F0800F18BF62F07F028DF80F2050
:10723000039804B0704700BF2DE9F04F83B00546B6
:107240000F4614461E46019201F1FF3313F1050F5C
:1072500044D8032E43D9A6F10400C0F380080DF1F1
:10726000040C2846FFF7E4FE05F10305A7F103012E
:1072700004F10404A6F10406A7F1040717F1050FB1
:1072800067D92CE00DF1040C284639462246FFF759
:10729000CFFE05F1030B5D46A7F1030104F1040ADB
:1072A0005446A6F104094E46A7F1040717F1050F4D
:1072B00015D80F460DF1040C58465246FFF7B8FE9C
:1072C0000BF10305A7F103010AF10404A9F1040677
:1072D000A7F1040818F1050F59D900E0FFE799B3A9
:1072E00096B30DF1040C28466A46FFF7A1FE022E64
:1072F00011D0032E02D0012E26D11AE0019929B116
:107300009DF8002022704FF0010301E04FF00003D0
:1073100004F1010401E04FF00003019830B102A92B
:10732000CA1812F8080C207003F1010304F10104DB
:1073300001E04FF00003019921B102AAD31813F81C
:10734000080C207004F101040199601A03B0BDE833
:10735000F08F0F46032EC2D9B8F1000F92D00DF175
:10736000040C28462246FFF763FE05F10305A7F14A
:10737000030104F10404A6F10406A7F1040717F1C0
:10738000050FACD80F46032E3FF67CAFA7E7A7F159
:107390000307032E3FF676AFA1E700BFF0B49DF8D8
:1073A0001040ECB14FEA41079F421CD2DD1B1DD0BB
:1073B00056194FF030046FEA0203F31803F001038B
:1073C00002F8014BB24240F0928007E0134603F806
:1073D000014B547003F10102B242F7D13B4607E082
:1073E0004FF0000504E04FF0000501E04FF000050C
:1073F00000293CD003F1FF34002B3AD000F1010307
:1074000041182846521B04F1FF3515F0020F10D029
:1074100032E0A4F1020603F101031F46012C29D03A
:107420003446B44613F8016C4FEA1616092E42D9B9
:1074300044E01E4613F8015C4FEA1515092D8CBF78
:1074400037353035155414B900F1010012E013F846
:10745000016C06F00F05092D8CBF37353035161835
:10746000757000F1020528468B42D2D102E0284611
:1074700000E02846F0BC70471E4613F8015C4FEA56
:107480001515092D94BF303537351554002CDBD038
:1074900013F8016C06F00F05092D94BF3035373510
:1074A0001618757000F102008B42E3D003F101035E
:1074B000A4F10204BDE706F1300601E006F137064B
:1074C0005655BCF1000FBFD013F8016C06F00F0643
:1074D000092E94BF303637361018467005F1020079
:1074E0008F42C7D003F10103A4F10204A1E7002BEE
:1074F0003FF46CAF02F8014BB2427FF467AF6DE727
:10750000DCF8143093F8452083F84420DCF814109C
:1075100091F8463081F84530DCF8141091F8472096
:1075200081F84620DCF8143083F84700704700BF2C
:10753000DCF8143093F8470093F8462083F847208E
:10754000DCF8141091F8453081F84630DCF814105E
:1075500091F8442081F84520704700BF42F61C7224
:10756000C2F2000213684AF60001C0F60101C85CCD
:10757000C918497803F10203136041EA00207047FB
:10758000DCF80430DCF8082002EBD300CCF808006B
:1075900003F007014FF0010303FA01F2CCF80420D5
:1075A000704700BF2DE9F04F83B004468A469346EA
:1075B0001E46CDF804C04FF00007B846B9463DE07E
:1075C00025463046D047034600283DD0B9F1000F8C
:1075D0000CD1202829D0092829D00A2829D00D2803
:1075E00029D0022D4FF0010988BF0225A3F13002F6
:1075F000D1B2092910D9A3F14100C1B2052903D89C
:10760000A3F13703D9B207E0A3F16102D0B2052894
:107610001AD8A3F15703D9B24FEA0717FCB241EACF
:10762000040708F101082C4606E02C4604E02C462D
:1076300002E02C4600E02C463046D847FF2CBFD055
:1076400004F1FF35002CBCD1DDF804C03846FFF74B
:1076500057FF019B5A69D8F1010838BF4FF0000865
:1076600082F8508003B0BDE8F08F00BF42F6A4530B
:10767000C2F200031B684B634BB19A68824209D087
:10768000DB684B631BB19A688242F9D102E04FF08C
:107690001E0070474FF00000704700BF884204D8BA
:1076A000884234BF0220002070474FF0010070472D
:1076B000D0F80431D0F80021934214BFC05C002000
:1076C000704700BFD0F80431FF2B14BF01330023F3
:1076D000C0F80431704700BF10B4DCF81420D16C3E
:1076E0000B46044658B14FEA016343EA116301F4C3
:1076F0007F4043EA002301F47F0143EA1123DCF8D1
:10770000040030B199B24FEA134060F30F0361F304
:107710001F435CB94FEA036141EA136103F47F4000
:1077200041EA002103F47F0341EA1323D36410BC30
:10773000704700BFDCF80030FA2B05D840F66C52D9
:10774000C2F20002D05C70474FF00000704700BFEB
:10775000DCF8003003F10103CCF80030DCF8140051
:1077600090F8512002F1010280F85120704700BFCB
:1077700070B404460846A1B199188C4211D225185C
:10778000AA420ED294423ABFC4EB0206F6B20026D9
:10779000A94205D20019821AD31AF118C8B200E022
:1077A000304670BC704700BFF0B583B042F6AC53B2
:1077B000C2F200034FF00C021A7041F64400C2F20C
:1077C000000004683CB3154642F6AC57C2F200070D
:1077D0004FF0000621680B6873B10DF107000DF141
:1077E000060198479DF807009DF8061032463B7841
:1077F000FFF7BEFF4519EDB26468002CEAD142F6EE
:10780000AC52C2F200021078A84204D242F6AC5147
:10781000C2F200010D7042F6AC53C2F200034FF009
:1078200000025A7042F6C454C2F20004246834B311
:10783000154642F6AC57C2F20007164620680368A8
:1078400073B10DF107000DF1060198479DF807008F
:107850009DF8061032467B78FFF78AFF4519EDB296
:107860006468002CEAD142F6AC51C2F200014A78B9
:10787000AA4204D242F6AC50C2F20000457042F671
:10788000AC53C2F200034FF00101997041F2BC7495
:10789000C2F2000424683CB30D4642F6AC57C2F273
:1078A00000074FF000062268136873B10DF107005E
:1078B0000DF1060198479DF807009DF80610324625
:1078C000BB78FFF755FF4519EDB26468002CEAD18B
:1078D00042F6AC50C2F200008178A94204D242F6CE
:1078E000AC52C2F20002957042F6AC53C2F20003F1
:1078F0004FF00000D87042F62074C2F200042468F1
:1079000034B3054642F6AC57C2F20007064621687A
:107910000A6872B10DF107000DF1060190479DF85C
:1079200007009DF806103246FB78FFF721FF451946
:10793000EDB26468002CEAD142F6AC53C2F2000307
:10794000D878A84204D242F6AC51C2F20001CD7000
:1079500003B0F0BD42F61873C2F2000319684AF68C
:107960000000C0F60200401A704700BF034610B185
:1079700082688A4218D042F6A853C2F200031868FF
:1079800060B182688A4203D10BE083688B420AD0DF
:1079900040680028F9D14FF0000305E04FF00003E4
:1079A00002E0034600E003461846704710B540F673
:1079B000AC64C2F200044FF4117303FB0044D4F82A
:1079C0000811B1F1FF3F03D0D4F8042191420DD149
:1079D00023689A6A4FF0FF019047002834D0D4F80A
:1079E000080100F10100C4F8080110BD91422BD834
:1079F0006318197942F62472C2F2000213787BB937
:107A0000FD290FD923689A6A4FF0FE019047D8B13B
:107A100042F62470C2F200004FF00101017010BD67
:107A20006FEA01012268936AC9B2984760B1D4F83D
:107A3000080100F10100C4F8080142F62471C2F205
:107A400000014FF000020A7010BD00BF70B506467D
:107A500040F6AC65C2F200054FF4117404FB00F46B
:107A60002B194FF00101C3F80C112A59936998475B
:107A70002859016A3046884770BD00BF38B540F6C6
:107A8000AC61C2F200014FF4117202FB00F28C18DB
:107A9000D4F80831D4F80451AB420DD08958E3181A
:107AA0008A6A1979904738B1D4F80801FF2814BFC1
:107AB00001300020C4F8080138BD00BF38B540F6D9
:107AC000AC64C2F200044FF4117202FB00F2A3187E
:107AD000D3F80451D3F808118D4206D14FF00001BC
:107AE000C3F80C11A2589369984738BD10B440F6FA
:107AF000AC63C2F200034FF4117202FB003000F5D8
:107B00008870D0F80031FF2B14BF5A1C0022D0F827
:107B10000441A2421CBFC154C0F8002110BC7047F0
:107B2000F8B542F61874C2F2000424688568C76884
:107B3000466807FB05604518611911D2CE180B483D
:107B4000864210D8012B04D1635D13704FF0000002
:107B5000F8BD10461A460CF043FE4FF00000F8BD89
:107B60004FF01F00F8BD4FF01F00F8BD01A802083C
:107B700010B542F6B053C2F200031A7840F6AC607A
:107B8000C2F200004FF4117404FB0204F8F7FEFD8A
:107B90004FF0FF31C4F810124FF00003C4F8183250
:107BA00004F58874F8F7FCFD10BD00BFF8B5064673
:107BB0004FF00203037049F60000C0F60100C28BCB
:107BC0004FF6FF718A4221D03F4C404BA34222D254
:107BD00003F110033E4DEF1A4FEA17124FF6FF75EF
:107BE00002F1010002F001071C46D98BA9424FD1D6
:107BF00015E01C46D98BA94211D002F1010203F114
:107C000010031C46D98BA94257D108E049F600045D
:107C1000C0F6010403E049F60004C0F601044FF683
:107C2000FF7021464FF00D02FFF754FA4FF6FF7335
:107C3000984208BF0020E28982421BD0A4F11005BF
:107C400049F60000C0F6010085421AD34FF6FF70D6
:107C500029464FF00D02FFF73DFA4FF6FF718842BB
:107C600008BF002034F8024C84420AD12C464FF061
:107C7000010201E04FF00002607BFF2806D1327064
:107C800004E04FF0020333704FF000042046F8BDCB
:107C90004FF0000202F1010203F110038242BED054
:107CA000002FA6D01C46D98BA942B8D002F1010200
:107CB00003F1100382429CD1B1E702F1010203F10A
:107CC0001003824295D1AAE700A00108009801089C
:107CD0000FA0010870B5C0B005460E4620F0FF04A5
:107CE000684621464FF04002F8F7B8FC00AB53FA63
:107CF00085F031464FF010020CF072FD68462146C7
:107D00004FF48072FAF7DEFB40B070BD38B505461F
:107D100040F6AC64C2F200044FF4117303FB00445C
:107D2000D4F81C02FDF73CFB42F6B050C2F2000052
:107D30000178A94206D142F6B053C2F200034FF0D7
:107D4000FF021A704FF00000C4F81C0238BD00BFDB
:107D500010B54FF00000FBF7CBFD41F64403C2F233
:107D600000031C6834B12068016901B18847646868
:107D7000002CF8D110BD00BF10B50446072822D84A
:107D8000032894BF4FF4FA73322303FB01F141F24D
:107D9000FC73C2F2000303EBC000416059B1FDF770
:107DA000CDFE002808BF012041F2FC73C2F200039F
:107DB00043F8340010BD41F2FC71C2F200014FF0F3
:107DC000000241F8342010BD38B5044607284BD8CE
:107DD00041F2FC73C2F2000303EBC00045680DB32F
:107DE00041F2FC71C2F2000151F83420D2B1FDF72A
:107DF000A5FE002808BF012041F2FC73C2F2000377
:107E000053F83410401A85420BD241F2FC73C2F28F
:107E1000000303EBC4024FF00005556043F83450F3
:107E200000E02D1A05F104054CF6CD41CCF6CC410D
:107E3000A1FB05204FEA9003032C0AD803F163034A
:107E400048F21F51C5F2EB11A1FB03324FEA521069
:107E500038BD03F109014CF6CD42CCF6CC42A2FB71
:107E600001304FEAD00038BD4FF0000038BD00BFF0
:107E700070B506466446DCF814305D6AFDF75EFEB8
:107E80006169CA6A0AB9C86208E0801A05EB85050B
:107E900006FB05F6B04224BF0020C8626369D96AB8
:107EA000D1F1010038BF002070BD00BF10B540F611
:107EB000AC63C2F200034FF4117404FB003303F50A
:107EC0008873D3F80841002C5FD15AB14FF0FF31CD
:107ED000C3F8001142F62573C2F200034FF0000010
:107EE000187010BDD3F80021B2F1FF3F06D1FF2971
:107EF0004BD14FF00002C3F8002110BDFF291ED165
:107F000042F62571C2F200014FF000040C70012A04
:107F100010D94FF00102C3F8082140F6AC63C2F259
:107F200000034FF4117101FB0030D0F81C02FCF784
:107F3000F5FF10BD4FF00000C3F8000110BDFE2991
:107F400007D142F62573C2F200034FF00101197008
:107F500010BD42F62570C2F20000007848B16FEA09
:107F60000101C9B242F62570C2F200004FF00004D0
:107F70000470FF2A05D8995402F10102C3F80021C8
:107F800010BD4FF0FF32C3F8002110BD08B540F618
:107F9000AC63C2F200034FF4117202FB0030D0F860
:107FA0000811D0F8043100F1040099420AD94FF0C9
:107FB0000002C0F8002142F6F450C2F2000040680E
:107FC000FCF7ACFF08BD00BFF8B5654641F63C03C1
:107FD000C2F200031C7804F00802D7B227B1DCF823
:107FE000146096F8516007E014F0110F06BFDCF83A
:107FF000144094F85260002601EB800411F8203000
:108000004FEA9312012A08D0022A10D111F82070E9
:10801000C7F3C20303FB06F70BE06A6992F851301D
:1080200011F82070C7F3C20202FB03F701E04FF022
:10803000000711F8200000F00701042950D8DFE8FC
:1080400011F0940140003B002200050042F61C7133
:10805000C2F200010B684AF60007C0F60107FA18E1
:1080600092F802E0D0784FEA006040EA0E40527881
:1080700040EA0220FF5C03F104030B603843FFF782
:10808000B9F868602CE042F61C72C2F20002136874
:108090004AF60000C0F60100C11891F801C0C05CAA
:1080A0004FEA004040EA0C208978084303F10303BB
:1080B00013603F186F6013E0FFF750FAC2196A604F
:1080C0000EE042F61C73C2F2000318684AF6000183
:1080D000C0F601010A5CBF186F6000F10100186072
:1080E00063784FEA9310012807D002280ED16178F7
:1080F000C1F3C20202FB06F70AE06F6997F851303C
:108100006078C0F3C20101FB03F701E04FF0000704
:10811000627802F00703042B50D8DFE813F0260141
:1081200040003B002200050042F61C71C2F2000133
:108130000B684AF60007C0F60107FA1892F802E049
:10814000D0784FEA006040EA0E40527840EA0220C0
:10815000FF5C03F104030B603843FFF74BF8A860A2
:108160002CE042F61C72C2F2000213684AF60000CC
:10817000C0F60100C11891F801C0C05C4FEA004090
:1081800040EA0C208978084303F1030313603F1889
:10819000AF6013E0FFF7E2F9C219AA600EE042F601
:1081A0001C73C2F2000318684AF60001C0F6010110
:1081B0000A5CBF18AF6000F101001860A3784FEAB5
:1081C0009310012807D002280ED1A178C1F3C20272
:1081D00002FB06F70AE06F6997F85130A078C0F308
:1081E000C20101FB03F701E04FF00007A27802F0A3
:1081F0000703042B4ED8DFE803F0B83E3920030014
:1082000042F61C71C2F200010B684AF60007C0F684
:108210000107FA1892F802E0D0784FEA006040EACD
:108220000E40527840EA0220FA5C03F104030B602E
:108230001043FEF7DFFFE8602CE042F61C72C2F24A
:10824000000213684AF60000C0F60100C11891F858
:1082500001C0C05C4FEA004040EA0C208978084326
:1082600003F1030313603F18EF6013E0FFF776F9A3
:10827000C219EA600EE042F61C73C2F200031868ED
:108280004AF60001C0F601010A5CBF18EF6000F178
:1082900001001860E3784FEA9310012802D0022809
:1082A0000FD108E06E6996F85130E078C0F3C20152
:1082B00001FB03F607E0E178C1F3C20202FB06F618
:1082C00001E04FF00006E27802F00703042B4CD8DF
:1082D000DFE803F04B031318300042F61C73C2F2C0
:1082E000000318684AF60001C0F601010A5CB618DE
:1082F0002E6100F101001860F8BDFFF72FF9821917
:108300002A61F8BD42F61C72C2F2000213684AF6F6
:108310000000C0F60100C1184C78C05C4FEA004074
:1083200040EA04208978084303F1030313603618F8
:108330002E61F8BD42F61C71C2F200010B684AF6CC
:108340000004C0F60104E2189678D0784FEA006085
:1083500040EA0640527840EA0220E25C03F104035E
:108360000B601043FEF746FF2861F8BD08B50328EF
:108370001ED8DFE800F00209101748F6F040C0F6FA
:1083800001000EF01DF808BD48F6F440C0F60100EB
:108390000EF016F808BD48F60850C0F601000EF0C1
:1083A0000FF808BD48F62050C0F601000EF008F89E
:1083B00008BD00BF2DE9F8430546884616461F460E
:1083C00042F6B053C2F2000393F8009043F26C40BF
:1083D000C2F20000016841F64002C2F200021368D6
:1083E000994201D0FFF7C4FB072D6ED81F2E6CD821
:1083F00040F6AC64C2F200044FF4117000FB094473
:1084000042F6F450C2F200004FF00001FCF726FBE8
:10841000217965F34711072D14BF00250125AA19FD
:1084200062F304012171CBB22DB184F8058043447D
:108430004FF0020001E04FF0010006F1FF3E5FFA4D
:108440008EFE46B302463F1A0EF0010C3D5C04F16D
:10845000040635545B1902F101020EF1FF31C9B275
:10846000FF2934D114E0BD5C04F10406B5545B1956
:1084700002F1010201F1FF3101F0FF01BD5CB554D1
:108480005B1902F1010201F1FF31C9B2FF29EAD102
:1084900000F1010070442218137100F10100C4F8CA
:1084A00004014FF0FF33C4F8083121680B6A42F62B
:1084B000B050C2F2000000789847FCF7FDFC42F68D
:1084C000F450C2F20000FCF7D7FBBDE8F8834FFA86
:1084D0008CF5002DC7D0BD5C04F10406B5545B19C2
:1084E00002F1010201F1FF31C9B2FF29BBD1CFE78F
:1084F00038B5054641F2C074C2F200042046FCF7CC
:10850000BBFBF9F7E5F92846FCF79EFE20464FF045
:108510000001FCF7A3FA38BD10B586B00DF10700D5
:10852000FFF744FB044618B19DF8073023B90FE06C
:1085300049F60004C0F60104E2894FF6FF7082425A
:108540002BD04AF20001C0F601018C4209D32AE087
:10855000304821464FF00D020BF0ECFC002848D0CB
:10856000EAE74FF6FF724AF20000C0F601006FEA38
:108570000403C118C1F3001104F11004E38993420C
:1085800039D10AE004F110031C46D989914204D084
:1085900003F11004E389934239D14AF20002C0F694
:1085A0000102944207D349F60004C0F601042046B4
:1085B0002146F9F71DFF02A816494FF00D020CF0F5
:1085C0000FF94FF0FF008DF815004FF6FF7002A96C
:1085D0004FF00D02FEF77EFD4FF6FF71884212BF8D
:1085E000ADF816000021ADF81610204602A9FFF7DD
:1085F00071FB06B010BD8442D5D20029C2D004F16F
:108600001004E1899142C8D08442BBD3CBE78442B5
:10861000B8D3C8E7720D00202DE9F04F85B0884629
:1086200091461D46E2464FF0000426464FF0020BED
:108630002DE007462846C047034670B324B92028DA
:1086400022D0092802D11FE0012C05D12B2B0DD0FF
:108650002D2B0DD05C4601E0022C01D12E2B09D030
:10866000A3F13002D0B2092817D805E05C4603E038
:108670005C4601E04FF003040E2E05D804A98A19C8
:1086800002F8103C06F101062846C8473846FF2884
:10869000CFD000F1FF370028CCD1012C12D98EB1F8
:1086A00004ACA6194FF0000406F8104C68462146A9
:1086B0000BF09AFCDAF81410C864DAF8142082F887
:1086C000504005E0DAF814304FF0010083F8500014
:1086D00005B0BDE8F08F00BF10B586B04AF60000C7
:1086E000C0F601003449F9F783FE00284BD1334B23
:1086F000334A9A421DD24AF60001C0F601010B68C6
:10870000B3F1FF3F42D102F104032E4AD01A20F008
:108710000302991812F0040F3FD118468B420CD077
:1087200003F104021B68B3F1FF3F3ED04FF000009D
:1087300031E04AF60000C0F601004AF60003C0F638
:108740000203984225D10DF10700FFF72FFA0446E6
:10875000B0B19DF80710022912D002A821464FF0AF
:1087600010020CF03DF89DF815006FF307008DF82E
:108770001500204602A9FFF7ADFA4FF001000AE00C
:108780004FF0010007E04FF0000004E04FF0000060
:1087900001E04FF0000006B010BD184603F10403DD
:1087A0000268B2F1FF3FB8D0C0E702F104031068DD
:1087B000B0F1FF3FB1D0B9E7FFA7020800A8020857
:1087C00000A8010803A802082DE9F00303460028C9
:1087D00042D040F20022C0F6000292F8468092F8A1
:1087E00047C042F6AC50C2F20000457892F848709B
:1087F000047842F6EC56C2F20006306896F804900F
:1088000076794FF000021A7083F8018083F802C075
:10881000DA704FF0FB0C83F804C04FF0060C83F8BD
:1088200005C09C71DD714FF004051D725D729F7271
:10883000DC721A734FEA10245C73987383F80F90FC
:108840001E745A744FF01D0098744FF00202DA74CF
:108850004FF0FE001875587529B142F6AC53C2F2BC
:1088600000031A680A60BDE8F0037047034628B1A8
:1088700042F6EC52C2F200021068186042F6EC5167
:10888000C2F200010879704770B505460E461446DD
:108890004FF000002946FFF769F808B1F7F7CEFE60
:1088A00042F6A853C2F200031A686260A56026600F
:1088B0001C6070BD08B539B141F64403C2F2000333
:1088C0001A68426018601EE041F64403C2F20003D9
:1088D0001B6883420FD1586841F64401C2F200017F
:1088E000086010E042685A6041605A688242F9D0DC
:1088F00013461BB907E033B14FF000015A688242BA
:10890000F0D01346F5E7FEF74FFF08BD08B539B1C3
:1089100042F6C453C2F200031A68426018601EE0B7
:1089200042F6C453C2F200031B6883420FD1586859
:1089300042F6C451C2F20001086010E042685A6079
:1089400041605A688242F9D013461BB907E033B13F
:108950004FF000015A688242F0D01346F5E7FEF767
:1089600023FF08BD08B539B141F2BC73C2F2000360
:108970001A68426018601EE041F2BC73C2F2000344
:108980001B6883420FD1586841F2BC71C2F20001EA
:10899000086010E042685A6041605A688242F9D02B
:1089A00013461BB907E033B14FF000015A68824209
:1089B000F0D01346F5E7FEF7F7FE08BD08B539B16C
:1089C00042F62073C2F200031A68426018601EE08B
:1089D00042F62073C2F200031B6883420FD158682D
:1089E00042F62071C2F20001086010E042685A604D
:1089F00041605A688242F9D013461BB907E033B18F
:108A00004FF000015A688242F0D01346F5E7FEF7B6
:108A1000CBFE08BD01604360826042F6A453C2F2FF
:108A200000031A68C2601860704700BF70B582B05A
:108A300006464FF000038DF807300D4601B10B706C
:108A400041F64400C2F20000046874B121684B682A
:108A500043B130460DF107012A46984710B19DF801
:108A6000070011E06468002CF0D10B2E03D83046CB
:108A7000FAF782FF08E02DB14FF005022A704FF09F
:108A8000000001E04FF0000002B070BD70B582B090
:108A900006464FF000038DF807300D4601B10B700C
:108AA00041F64400C2F20000046874B121688B688A
:108AB00043B130460DF107012A46984710B19DF8A1
:108AC000070019E06468002CF0D10B2E0BD830465B
:108AD000FAF768FF8DF8070010B13046FAF7A8FFE3
:108AE0009DF8070008E02DB14FF005022A704FF005
:108AF000000001E04FF0000002B070BD70B582B020
:108B000006464FF000038DF807300D4601B10B709B
:108B100041F64400C2F20000046874B12168CB68D9
:108B200043B130460DF107012A46984710B19DF830
:108B3000070011E06468002CF0D10B2E03D83046FA
:108B4000FAF700FF08E02DB14FF005022A704FF050
:108B5000000001E04FF0000002B070BD70B582B0BF
:108B600006464FF000038DF807300D4601B10B703B
:108B700042F6C450C2F20000046894B121688B68C8
:108B80002BB130460DF107012A46984718B96468A1
:108B9000002CF3D105E09DF80700003018BF01203C
:108BA00008E02DB14FF006022A704FF0000001E0FE
:108BB0004FF0000002B070BDF0B583B005460E4620
:108BC0004FF000038DF8073042F6C450C2F20000A7
:108BD00004681CB34FF000072168CA681AB1284620
:108BE00031469047E8B923689B6833B128460DF1B8
:108BF00006010DF10702984700E038469DF807107E
:108C000091B9646814B10028E6D000E070B128463C
:108C1000314606F05DFA4FF0000009E04FF0060023
:108C200006E04FF0000003E0084601E04FF00600C8
:108C300003B0F0BD70B582B005460E464FF000039C
:108C40008DF8073012B11946FFF7B6FF42F6C4504F
:108C5000C2F20000046884B121684B68284631469E
:108C60000DF10702984710B19DF8070007E064680E
:108C7000002CF1D14FF0060001E04FF0060002B0E9
:108C800070BD00BF08B54FF0000001464FF0010273
:108C9000FFF7D0FF08BD00BF70B582B005460E4695
:108CA0004FF000038DF8073041F2BC70C2F20000B3
:108CB00004689CB121684B68284669460DF107029B
:108CC000984728B10EB1009830609DF8070014E075
:108CD00064681CB19DF80720002AEBD045B956B155
:108CE0004FF00000F9F73EF830604FF0000004E06C
:108CF0004FF00F0001E04FF0000002B070BD00BF68
:108D000070B582B005460E464FF000038DF807306F
:108D100042F62070C2F2000004689CB121684B68E2
:108D2000284631460DF10702984710B19DF807001B
:108D30000DE064684CB19DF80720002AEED04FF09A
:108D40000E0004E04FF00E0001E04FF00E0002B004
:108D500070BD00BF70B582B005460E464FF00003EF
:108D60008DF8073042F62070C2F200000468BCB1F2
:108D700021688B685BB1284669460DF10702984768
:108D800028B10EB1009830609DF807000DE06468CE
:108D90004CB19DF80720002AEAD04FF0060004E00D
:108DA0004FF0060001E04FF0060002B070BD00BFBA
:108DB0002DE9F04F2DED048B8BB0074615469142FF
:108DC00059D289464FF0000B4FF000089FED908B71
:108DD0009FED919B6FEA0106B01800F00106CDF8F7
:108DE00004B0022F4CD150E0CDF804B0022F05D1D1
:108DF0005FFA89F001A9FFF7ADFF04E05FFA89F09F
:108E000001A9FFF749FF04EB44060AA88119A1F163
:108E1000200601F8209C01F81F8C01980AF044FB01
:108E200053EC182B0AF0DEFC53EC192B0AF096FBDE
:108E30000AF000FB83B2FF2B28BFFF23B37004F1BD
:108E400001040A2C04D005F1FF324A450AD14CB185
:108E500004EB44044FF007003946E2B202ABFFF7DF
:108E6000A9FA444609F101094E46CDF804B0022F93
:108E700040F089808DE00BB0BDEC048BBDE8F08F35
:108E8000C8B201A9FFF708FF03E0C8B201A9FFF7C4
:108E900061FF0AAC04F8209D84F8018001980AF073
:108EA00003FB53EC182B0AF09DFC53EC192B0AF032
:108EB00055FB0AF0BFFA81B2FF2934BF0B46FF23EE
:108EC000A3704FF0000404F1010405F1FF324A459C
:108ED0000DD10AE004EB44044FF007003946E2B23A
:108EE00002ABFFF767FA444601E0002CF2D109F12A
:108EF00001094D45BFD9002E3FF476AFCDF804B03F
:108F0000022F05D05FFA89F001A9FFF7C5FE04E042
:108F10005FFA89F001A9FFF71DFF04EB44060AA8D8
:108F2000861906F8209D86F8018001980AF0BCFA9F
:108F300053EC182B0AF056FC53EC192B0AF00EFBDD
:108F40000AF078FA81B2FF2934BF0B46FF23B370D1
:108F500004F101040A2C0AD104EB44044FF0070089
:108F60003946E2B202ABFFF725FA444605E005F1C7
:108F7000FF324A4501D1002CEED109F101094D45DE
:108F80003FF632AF77E75FFA89F001A9FFF784FE79
:108F900004E05FFA89F001A9FFF7DCFE04EB44006E
:108FA0000AA90B18A3F1200A03F8206C03F81F8C00
:108FB00001980AF079FA53EC182B0AF013FC53ECE1
:108FC000192B0AF0CBFA0AF035FA82B2FF2A28BF31
:108FD000FF228AF8022004F101040A2C0AD104EBD2
:108FE00044044FF007003946E2B202ABFFF7E2F962
:108FF000444605E005F1FF30B04201D1002CEED12E
:1090000009F101094D453FF6EFAE34E7AFF30080BB
:109010000000000000E06F40000000000000E03FA2
:109020002DE9F04F95B040F6C410FCF70DF94FF064
:1090300002004FF0000142F6AC53C2F20003DA78AE
:10904000FFF7B6FE4FF0000BDA46D9464FF00107A6
:109050004CF6CD44CCF6CC4401944FF07D00FCF7A7
:10906000F3F88DF82F90C8464E464C4613E045F075
:10907000800504F10804E4B20CABF05CA84202D015
:109080000CA97554B84606F101069DF82F50002D25
:1090900050D1202E4ED020460DF12F01FFF7C6FCF7
:1090A000051C18BF012504F10100C0B20DF12F010C
:1090B000FFF7BCFC10B145F00205EDB204F102016E
:1090C000C8B20DF12F01FFF7B1FC08B145F004055E
:1090D00004F10302D0B20DF12F01FFF7A7FC08B194
:1090E00045F0080504F10403D8B20DF12F01FFF794
:1090F0009DFC08B145F0100504F10500C0B20DF16A
:109100002F01FFF793FC08B145F0200504F106019B
:10911000C8B20DF12F01FFF789FC08B145F04005F9
:1091200004F10702D0B20DF12F01FFF77FFC0028F8
:109130009DD19EE7B8F1000F02D1BAF1000F0AD11C
:109140004FF002004946F2B20CABFFF733F94FF093
:109150003200FCF779F842F6AC52C2F20002927883
:109160008AB1019EA6FB0A434FEA131404EB840064
:10917000BAEB800F07D138464946FFF719FE4FF08A
:109180003200FCF761F8BBF1000F40F09B8003A8B0
:1091900049464FF020020BF047FB42F6AC51C2F2B9
:1091A00000018D78ADB34E466FEA0902531903F002
:1091B000010009F0070407FA04F29DF80C1042EAD6
:1091C00001038DF80C3006F10106AE42C0F2998021
:1091D0001FE014AA02EBD60306F0070407FA04F016
:1091E00013F8441C40EA010203F8442C06F101067E
:1091F00014AC04EBD60006F0070107FA01F210F8F0
:10920000443C42EA030400F8444C06F10106AE4235
:10921000DFDB4FF007004FF011014FF01E0203ABF0
:10922000FFF7C8F84FF03200FCF70EF803A84946E4
:109230004FF020020BF0F8FA42F6AC55C2F20005EE
:10924000EE78A6B348466FEA09018A1902F00103D5
:1092500009F0070407FA04F59DF80C1045EA01022D
:109260008DF80C2000F10100864236DC1FE014ADC1
:1092700005EBD00200F0070407FA04F312F8441CCF
:1092800043EA010502F8445C00F1010014AA02EB74
:10929000D00500F0070407FA04F315F8441C43EA6C
:1092A000010205F8442C00F101008642DFDC4FF09A
:1092B00007004FF012014FF01E0203ABFFF77AF8E0
:1092C0004FF0060BBAF1000F04D10BF1FF3B4FF04A
:1092D000280AC2E60AF1FF3ABFE6002BC7D014AB5A
:1092E00003EBD00500F0070407FA04F215F8441C5C
:1092F00042EA010305F8443C00F101008642B6DC75
:10930000D5E700283FF465AF14A800EBD60206F0BD
:10931000070407FA04F312F8441C43EA010002F8B8
:10932000440C06F10106AE42FFF653AF71E700BFF1
:109330002DE9F04F2DED028B87B008EE100A0C4698
:1093400017469946129E1399B5EEC08AF1EE10FAAF
:1093500054BF00250125A84604F1FF33D8B20828E0
:1093600007D8092A05D8A24601F1FF32944205D850
:1093700008E001F1FF339C4240F2CD8001F1FF345F
:10938000E4B2C8E018EE100A0AF062FC48B93046B0
:109390004FF03F0122460BF047FA4FF000013155E4
:1093A000C4E018EE100A0AF0BFFC06EE900AF2EED6
:1093B000047AF4EEE76AF1EE10FA0DDB4FF00100EB
:1093C000B0EE677A00F1010067EE877AF4EEE76AA3
:1093D000F1EE10FAF6DA03E04FF00100F2EE047A53
:1093E00021464319A34200F39680C0EB040EC5EB5F
:1093F0000E0202F1FF3E48F6B83AC0F6010ADFED70
:109400009C4AF6EE003AB2EE044AC0EB040CC5EBFF
:109410000C0303F0010BBEF1000F00F38F808AE014
:10942000BEF1000F04DDBE45B4BF72463A4601E00E
:109430004FF000025AF8223003EE103AB8EE430A19
:1094400020EE027AB4EEE47AF1EE10FA48BF37EE7D
:10945000237ABDEEC73A13EE10CABCFBF3FB06EE4F
:1094600010BAB8EEC65AB4EEE75AF1EE10FA0DDBB8
:1094700000F1010C87EE006A67EE847A0EF1FF3E80
:109480006046BEF1000200F3C380BEE013EE105A46
:10949000B5FBF3F403FB14542CB916EE107A002F2D
:1094A00008BF4FF00008B9F1000F07D0C8EB010367
:1094B000181A002A18BF0138831A01E04FF0000380
:1094C00001F10101B8F1000F04D048F64457C0F68D
:1094D000010703E046F2A447C0F6010722B148F6AF
:1094E0004850C0F6010003E046F2A440C0F6010077
:1094F00048F65C55C0F60105009501978DED026AAE
:10950000039004920594304648F64C52C0F601028E
:109510000AF054FD0AE03046002D0CBF2B212D210E
:1095200022460BF081F94FF00000305507B0BDEC3A
:10953000028BBDE8F08F4FF0000203E0BE45B4BFE0
:1095400072463A465AF8223000EE103AB8EE405AC7
:1095500065EE260AF4EEE40AF1EE10FA48BF70EE6A
:10956000A30ABDEEE03A13EE10CABCFBF3FC06EE14
:1095700010CAF8EEC65AF4EEE75AF1EE10FA85DB9F
:1095800000F1010080EE852A67EE847A0EF1FF3E3D
:1095900042199142BFDBBBF1000F3FF441AFBEF176
:1095A000000F02DC4FF0000203E0BE45B4BF72467C
:1095B0003A465AF8223001EE103AF8EE411A21EEFE
:1095C000822AB4EEE42AF1EE10FA48BF32EE232AE2
:1095D000BDEEC23A13EE10BABBFBF3FB06EE10BAB7
:1095E000F8EEC62AF4EEE72AF1EE10FAFFF64EAFD7
:1095F00000F1010082EE212A67EE847A0EF1FF3E2F
:1096000043199942BFF60CAF85E74FF0000202E024
:10961000BA42A8BF3A465AF8223006EE903AF8EE1F
:10962000660A20EE861AB4EEE41AF1EE10FA48BF8C
:1096300031EE231ABDEEC13A13EE10BABBFBF3FBB9
:1096400006EE10BAF8EEC65AF4EEE75AF1EE10FA4A
:10965000FFF61CAF0CF1010081EE202A67EE847A40
:109660000EF1FF3E42199142BFF6DAAE53E700BF5A
:109670000000004BF8B505460F46F7F787F8064699
:1096800040F6AC62C2F200024FF4117303FB05F026
:109690001418115811B18A682846904784F820722E
:1096A0004FF00005C4F81052C4F81452C4F8045125
:1096B000C4F808513046F7F773F804F509702946E5
:1096C0004FF00802F7F71CF8F8BD00BF70B588B07E
:1096D000054640F6AC64C2F200044FF4117303FB7C
:1096E000004494F82002002847D042F6B051C2F25C
:1096F00000010878FF2803D04FF00401FFF7BAFFFC
:1097000028464FF00001FFF7B5FF42F6B056C2F20F
:109710000006357048F66850C0F601004FF00701AA
:109720004EF2C172C0F60002FBF750FDC4F81C02F5
:10973000246830784FF0010200924FF0000201924D
:1097400047F6AD13C0F60003029347F68D71C0F6DD
:109750000001039147F6AD63C0F60003049347F69A
:109760000D51C0F600010591069264684FF4165140
:109770004FF00803A047FEF7FBF908B070BD00BF2B
:1097800038B505F099FC42F6B153C2F200034FF030
:1097900001021A704FF000042546E0B229462A461D
:1097A000FFF748FA40B904F10104E0B229462A461D
:1097B000FFF740FA00285BD042F62071C2F20001A8
:1097C0000C6834B12368DA6802B190476468002CF1
:1097D000F8D142F6A850C2F2000004683CB12168FA
:1097E0000B680BB1A06898476468002CF7D1FAF7B2
:1097F000FFFBFEF7ADFA40F6AC62C2F2000292F84F
:109800002002042806D028B14FF000004FF00401D8
:10981000FFF730FF40F6AC61C2F2000191F864340A
:10982000042B06D02BB14FF001004FF00401FFF7DD
:1098300021FF40F6AC62C2F2000292F8A8060428AA
:1098400006D028B14FF002004FF00401FFF712FFDD
:1098500040F6AC61C2F2000191F8EC38042B06D05E
:109860002BB14FF003004FF00401FFF703FF38BDA9
:1098700004F10104B4F5807F8FD19DE72DE9F04F0D
:109880002DED0A8BABB01CAF26AC47F69035C0F679
:10989000010595E80F0084E80F00A76047F23573D3
:1098A000C0F60003E36020462AA9F8F775FF22AE50
:1098B00095E80F0086E80F00B76047F25170C0F6D8
:1098C0000000F06030462146F8F766FF4FF00004D4
:1098D0001B9441F2C070C2F200002146FBF7BEF8B3
:1098E00042F6EC51C2F200010C71FFF749FF09F09A
:1098F00085F84FF00200FFF7E9FE42F61C72C2F253
:10990000000215680DBB0CF04BFDF0B9F7F7E2FE55
:1099100010F0C20F19D14FF00300FEF727FD4FF4EE
:109920007A744FF032052846FBF78EFCF7F7D0FF2C
:1099300004F1FF342846FBF787FCF7F7C9FF013C29
:10994000F1D14FF00000FEF711FD41F63C03C2F2E9
:1099500000034FF000041C604FF00100187041F646
:109960004805C2F200052846214641F254520AF049
:109970005BFF40F66C50C2F2000021464FF480724B
:109980000AF052FF41F2FC70C2F2000021464FF093
:1099900040020AF049FF42F61C60C2F20000214674
:1099A0004FF0FC020AF040FF21954FF00A01696276
:1099B00020462946FDF75AFE41F2F872C2F2000233
:1099C000146042F6A053C2F200031C6042F61C75FC
:1099D000C2F200054FF030042C604AF60004C0F6D5
:1099E000010494F82F0000F1010094F82E1000EB10
:1099F0000122101942F61873C2F200031860FCF736
:109A00009DF80B902868215CFF2924D142F6EC5286
:109A1000C2F200024FF00103137110604FF0FF011A
:109A2000517142F69C50C2F200004FF000020260F9
:109A300042F6B053C2F20003197840F6AC60C2F2AD
:109A400000004FF4117202FB0103D3F81C02FBF774
:109A500065FA04F0E5BD05F00DFB4FF000060A962F
:109A6000B2463446DFEDBF8A9FEDBF9ADFEDBFAA55
:109A70009FEDBF8ADFEDBF9A9FEDBFAA01E04FF0D7
:109A800000042CB94FF00000FEF732FD4FF06404E3
:109A900004F1FF3441F63C07C2F200073D7805F0BF
:109AA000F7026FF304123A7042F61C73C2F200031D
:109AB0001868099042F61C76C2F200064AF60007C2
:109AC000C0F6010741F63C08C2F2000848F2EC5922
:109AD000C0F6010931687D5C01F10101316098F83F
:109AE000002012F0010F0ED10AF1010A40F2FF33FB
:109AF0009A4508D942F6EC53C2F200034FF0360102
:109B0000197104F053BD0DF1700C28464946FEF75B
:109B10005BFA48F2EC10C0F6010050F8252047F639
:109B2000A44BC0F6010B42F0010108473268BB5C50
:109B30000C9302F1010232600F2B04F22F850DF11C
:109B4000700C18465946FEF73FFA48F2AC00C0F6D2
:109B500001000C9950F82120E5E73268BB5C0C93BA
:109B600002F101023260102B02D91D4604F017BD2C
:109B70000DF1700C0C9847F62861C0F60101FEF754
:109B800023FA47F6E450C0F601000C9950F8212062
:109B9000C9E73268BB5C0C9302F1010232600F2B03
:109BA00002D91D4604F0FBBC0DF1700C0C9847F671
:109BB0007C71C0F60101FEF707FA48F2EC00C0F62E
:109BC00001000C9950F82120ADE73268BB5C0C9382
:109BD00002F1010232602F2B02D91D4604F0DFBCD6
:109BE0000DF1700C0C9848F22C11C0F60101FEF733
:109BF000EBF948F6F820C0F601000C9950F8212046
:109C000091E73268BB5C0C9302F1010232603B2B9E
:109C100002D91D4604F0C3BC0DF1700C0C9847F638
:109C2000A031C0F60101FEF7CFF947F6BC70C0F6CF
:109C300001000C9950F8212075E73268BB5C0C9349
:109C400002F1010232603F2B02D91D4604F0A7BC8D
:109C50000DF1700C0C9848F6EC11C0F60101FEF7FE
:109C6000B3F947F6E440C0F601000C9950F8212002
:109C700059E73268BB5C0C9302F101023260432B5E
:109C800002D91D4604F08BBC0DF1700C0C9847F600
:109C90006C61C0F60101FEF797F948F6E030C0F6B6
:109CA00001000C9950F821203DE7219E96F846705E
:109CB0000DF1700CFDF73CFC219D3B1895F8500010
:109CC00000F001015A181C9285F84720FF2A94BF22
:109CD0000022012285F85020D3E6219E96F8467096
:109CE0000DF1700CFDF724FC3D181C95219B83F8A9
:109CF0004750FF2D94BF0025012583F85050C0E642
:109D00000DF1700CFDF714FC30B1219991F847204A
:109D1000101C18BF012001E04FF00000219E86F8C2
:109D20004700AEE60DF1700CFDF702FC219F97F89D
:109D30004750284087F84700A3E61D9BA3F1FB038B
:109D40001C9313E11D98A0F1FB001C909BE11D9951
:109D5000A1F1FB011C91CCE11D9AA2F1FB021C9226
:109D600068E200BF00000034FFFF7F4BFFFF7FCBA6
:109D700000000000FEFFFFCAFEFFFF4A1D9BA3F18B
:109D8000FB031C934FF002001B90F3E11D99A1F11E
:109D9000FB011C911E9A1B921DE21D9BA3F1FB036C
:109DA0001C9317E11D98A0F1FB001C9099E21D99EE
:109DB000A1F1FB011C91D5E21D9EA6F1FB061C96AC
:109DC0001E9F1B9712E31D9AA2F1FB021C921E9B81
:109DD0001B934FF000008DF86A00C0E31D99A1F1BC
:109DE000FB011C911E9A1B924FF001038DF86A3003
:109DF000B5E31D98A0F1FB001C9000F04DBC1D9D2B
:109E0000A5F1FB051C9500F0A2BC9DF874004FF075
:109E10000101FEF7D1FE8DF86B0000283FF431AE52
:109E200042F6EC54C2F20004207104F0BFBB1D9E48
:109E30001C964FF001038DF86A301E46219991F867
:109E40004720134205D09DF870003146FEF7B4FE5E
:109E500068B99DF86A304FEA43008DF86A001C9992
:109E600001F101011C9110F0FE03E7D10CE09DF817
:109E70006A20012A08D19DF86B4042F6EC50C2F2EC
:109E80000000047104F092BB0DF1700CFDF750FB63
:109E9000F7E59DF8740005F0DFF8F2E50DF1700CC0
:109EA000FDF746FB1C9042F61C73C2F200031A68D1
:109EB0001C9902EB41001860FDF750FB1C9001F06B
:109EC000CABC1D99FA2908D942F6EC54C2F2000422
:109ED0004FF01300207104F069BB40F66C53C2F2DE
:109EE00000035A5C1C92DEE7219991F852301C93D2
:109EF000D9E7219A92F850001C90D4E74FF0000A5D
:109F0000BFE50DF1700CFDF713FB1C90219F97F836
:109F100047101B91FDF7C2FB87F84700B1E5219D73
:109F200095F8470095F84610FDF7B8FB85F8500006
:109F3000A7E50DF1700CFDF723FB1E9E40F66C5358
:109F4000C2F200039A5D1D9922EA0100985598E536
:109F500042F61C60C2F200004FF000014FF0FB021D
:109F60000AF062FC8DE54FF000061C960DF1A80C7E
:109F70001CF8386DFDF7DCFA0146304606F0C4FFE8
:109F80008DF86B0000283FF47CAD42F6EC54C2F231
:109F90000004207104F00ABB05F044FE71E505F0F1
:109FA00049FE8DF86B0000283FF46BAD42F6EC5390
:109FB000C2F20003187104F0F9BA42F61877C2F23F
:109FC00000073D681D9AA81805F020FE59E54FF0DE
:109FD00000011C911C9840F6AC63C2F200034FF4E0
:109FE000117101FB003292F82032032B3FD140F671
:109FF000AC66C2F2000601FB00F000F58877F119AB
:10A00000331803F104034FF00000D1F80021FE2AB9
:10A0100094BF551C0025D1F80461B54214BF00253A
:10A02000012565F30000B24214BF0022012262F351
:10A030004100D3F80051FE2D94BF013500250DF1EC
:10A04000A80C4CF8385DD3F80471BD4214BF00254C
:10A05000012565F38200D3F80811D1F1010338BF5F
:10A06000002363F3C300C0B2FDF74AFA09E542F6E4
:10A07000EC54C2F200044FF04800207104F096BA8C
:10A080004FF000001C901C9B40F6AC62C2F2000234
:10A090004FF4117101FB032090F82022032A1CD1F8
:10A0A00040F6AC66C2F2000601FB0365D5F81072FB
:10A0B000D5F81412781AB0F5807F88BF00F580704B
:10A0C0001C901C9AFF2A84BFFF221C920DF1A80C41
:10A0D0001CF8380DFDF714FAD3E442F6EC54C2F242
:10A0E00000044FF04803237104F060BA4FF00003FE
:10A0F0001C931C9840F6AC62C2F200024FF411713E
:10A1000001FB002393F82022032A24D140F6AC66F9
:10A11000C2F2000601FB006505F58877D7F800114B
:10A12000D7F80431CA1AB2F5807F88BF02F5807271
:10A130001C920DF1700CFDF7FBF98DF86A001C9E66
:10A14000B04238BF1C90D7F804011C9D2918CBB22F
:10A15000C7F8043195E442F6EC54C2F200044FF023
:10A160004800207104F022BA4FF000021C924FF018
:10A1700002001B901C9B40F6AC62C2F200024FF43E
:10A18000117101FB032090F82022032A15D140F61B
:10A19000AC67C2F2000701FB03760DF1700C1B984F
:10A1A00047F2B161C0F6000147F2C562C0F6000295
:10A1B00006F58873FDF7F6F963E442F6EC54C2F253
:10A1C00000044FF04803237104F0F0B94FF0000190
:10A1D0001C911D981B901C9B40F6AC62C2F20002C1
:10A1E0004FF4117101FB032090F82022032A15D1AE
:10A1F00040F6AC65C2F2000501FB03570DF1700C8F
:10A200001B9847F2B161C0F6000147F2C562C0F683
:10A21000000207F58873FEF7FFF932E442F6EC54CA
:10A22000C2F200044FF04803237104F0BFB94FF0AD
:10A2300000011C911C9840F6AC62C2F200024FF47F
:10A24000117303FB002191F82022032A3DD140F62F
:10A25000AC66C2F2000603FB006505F588750DF1DA
:10A26000700CFDF765F98DF86A00D5F804111C91A2
:10A270004FF000071B97D5F800710B468F4207D0AF
:10A280006A5C824219D04FF001024FF0000E0CE0E0
:10A290004FF0FF001B9010E002F10106E95C8142E3
:10A2A00002D11C931B9208E03246FF2B14BF0133EE
:10A2B0007346BB42F0D11C93EAE70DF1700C9DF898
:10A2C0006C00FDF71DF9FFF7DCBB42F6EC54C2F25F
:10A2D00000044FF04800207104F068B94FF000030B
:10A2E0001C931C9840F6AC62C2F200024FF411714C
:10A2F00001FB002393F82022032A27D140F6AC6506
:10A30000C2F2000501FB005707F58875D7F8146203
:10A31000D7F810128E4212D00DF1700CFDF708F92B
:10A320008019C7B21C970DF1700CE85DFDF7E8F8D5
:10A330004FF00005219E86F85050FFF7A2BB4FF06A
:10A340000102219B83F85020FFF79BBB42F6EC549F
:10A35000C2F200044FF04800207104F027B94FF01A
:10A3600000011C911C9B40F6AC62C2F200024FF44B
:10A37000117000FB032191F82022032A28D140F616
:10A38000AC67C2F2000700FB037505F58876D6F8C6
:10A390000401D6F80011884213D00DF1700C305C26
:10A3A000FDF7AEF8D6F80471FF2F14BF0137002770
:10A3B000C6F804714FF00005219E86F85050FFF753
:10A3C00060BB4FF00102219B83F85020FFF759BB7F
:10A3D00042F6EC54C2F200044FF04803237104F03B
:10A3E000E5B84FF000001C901D991B9142F61872C1
:10A3F000C2F20002D2F800801B9F08EB07064AF663
:10A400000003C0F602039E4208D942F6EC54C2F2A1
:10A4100000044FF01F02227104F0C8B81C980328F2
:10A4200008D942F6EC50C2F200004FF03703037136
:10A4300004F0BCB8F1780D2908D942F6EC54C2F208
:10A4400000044FF03701217104F0B0B840F6AC655C
:10A45000C2F200054FF4117202FB005393F8200280
:10A4600038B118F8071021B10FE04846FEF740F860
:10A4700005E04CF24F354FF09609DDF82CB0FBF7B4
:10A480005DFBCBEB0002AA42EFD918F80770032F4F
:10A490003FF6F7AADFE807F002080F169DF87000F4
:10A4A000FFF714F9FFF7EDBA9DF87000314606F09A
:10A4B00045FDFFF7E6BA9DF87000314605F034FB24
:10A4C000FFF7DFBA9DF87050B77828464FF00301C8
:10A4D000FFF7D0F84FF4117303FB05F040F6AC61C1
:10A4E000C2F20001085800283FF4CBAA47F6904377
:10A4F000C0F6010307EB470703EB0708F67848F6B9
:10A50000E852C0F6010252F82610DA5D98F80130E0
:10A5100098F8027000974FF00006019647F67D27E5
:10A52000C0F60007029747F6BD27C0F6000703975D
:10A5300047F6ED27C0F60007049747F60D57C0F61B
:10A5400000070597069646682846B047FFF799BA70
:10A550004FF000011C911D981B908DF86A101C98FB
:10A5600040F6AC63C2F200034FF4117101FB0032FC
:10A5700092F82032032B79D140F6AC65C2F2000587
:10A5800001FB005707F5887942F61876C2F20006FB
:10A590003168219A936B01EB030BCB5CFF2B5CD0F2
:10A5A000D8464FF001054FF0000B0994CDF830A0CC
:10A5B000AA4698F8014004EB032742F61876C2F247
:10A5C00000063268D319D9F804111C919DF86A006D
:10A5D00018B1D75D03F1010300E05F4603F1FF34DA
:10A5E0009DF86A502DB177B9099C5046DDF830A02E
:10A5F00005E066783EB9099C5046DDF830A01C9A0B
:10A60000C9F804212BE01C9BD9F800219A4218D0EC
:10A6100014F8016F19F803501B9939B9304609F045
:10A6200071FCC6B2284609F06DFCC5B2AE4208D135
:10A630001C98FF2814BF013058461C9007F1FF37C3
:10A64000CEE70AF1010A18F8023FFF2BB1D1099CAD
:10A65000DDF830A04FF0000001E04FF000000DF1F8
:10A66000700CC0B2FCF74CFFFFF70BBA42F6EC548B
:10A67000C2F200044FF04800207103F097BF4FF082
:10A6800000031C931E9A1B924FF001018DF86A1073
:10A6900065E74FF000011C911C9840F6AC63C2F2D4
:10A6A00000034FF4117101FB003292F82032032BAA
:10A6B00031D140F6AC66C2F2000601FB006505F53B
:10A6C00088770DF1700CFCF733FF8DF86A004FF0BE
:10A6D00000011C91D7F80431D7F80051AB4212D0D9
:10A6E000FA5C82420FD14FF00006FF2B14BF0133FA
:10A6F0003346AB4202D1C7F8043104E0F95C814231
:10A70000F3D0C7F804310DF1700C4FF00000FCF7E6
:10A71000F7FEFFF7B6B942F6EC54C2F200044FF070
:10A720004800207103F042BFFBF708FA0B9FC01BE3
:10A730000DF1700C4CF24F3398428CBF0020012079
:10A74000FCF7DEFEFFF79DB94FF000001C901C9D4A
:10A7500040F6AC62C2F200024FF4117606FB05210E
:10A7600091F82072032F7FF48CA940F6AC63C2F2FB
:10A77000000306FB053000F10405D0F80861D5F8A8
:10A78000002102F10102964238BF06F58076B11A27
:10A79000FF2934BF0F46FF270DF1700CF8B2FCF70C
:10A7A000AFFEFFF76EB91D9B40F66C50C2F2000081
:10A7B000C55C05F1FF36C654FFF763B91D9BFA2B44
:10A7C00008D942F6EC54C2F200044FF01301217193
:10A7D00003F0ECBE40F66C51C2F20001CA5C02F11B
:10A7E000FF30C2B2CA54002A3FF44BA91E9B1C93EF
:10A7F00001F031B81D98FA2808D942F6EC54C2F29B
:10A8000000044FF01300207103F0D0BE40F66C53EB
:10A81000C2F200031A5C02F1FF31CAB21A54002AD4
:10A8200042F01D84FFF72DB91D9BFA2B08D942F683
:10A83000EC54C2F200044FF01303237103F0B6BED0
:10A8400040F66C51C2F20001CA5C02F1FF30C2B2A4
:10A85000CA54002A02F00384FFF713B9219F97F826
:10A86000515005F1FF3687F85160FFF70AB9219979
:10A8700091F8470000F1FF3281F84720FFF701B956
:10A88000219BD86C09F050FA219FF864FFF7F9B8C2
:10A89000219D95ED137AD5ED127A37EE270A85EDD5
:10A8A000130A219DE86C09F0B3F930B14FF00206AC
:10A8B000219D85F85060FFF7E4B8219FF86C09F0FE
:10A8C000B7F930B14FF00101219B83F85010FFF729
:10A8D000D8B84FF00002219880F85020FFF7D1B887
:10A8E0009DF87400219901F14C01FEF7D5F98DF81E
:10A8F0006B0000283FF4C5A842F6EC54C2F20004F5
:10A90000207103F053BE9DF874002199C96CFEF7C5
:10A91000F7F98DF86B0000283FF4B3A842F6EC522B
:10A92000C2F20002107103F041BE219EF06C09F0EA
:10A930007FF920B92198806C09F07AF930B14FF095
:10A940000306219880F85060FFF79BB8219BD3ED58
:10A9500013BA93ED12BA7BEECB0A10EE900A09F00F
:10A96000E3F90CEE100A1BEE900A1BEE101A09F028
:10A9700075F901464FF07E5009F070F901EE100AAA
:10A9800061EE281AB4EEE1CAF1EE10FA06D84FF0E3
:10A990000001219A82F85010FFF773B8219F97EDBC
:10A9A000132AD7ED122AB4EEE22AF1EE10FA05DDF1
:10A9B0004FF0010587F85050FFF763B8B4EEE22A74
:10A9C000F1EE10FA4CBF0222032287F85020FFF765
:10A9D00058B8219B93ED133AF7EE003A33EE634AF1
:10A9E00083ED134A2198C06C09F022F930B14FF081
:10A9F0000305219981F85050FFF743B8219A92ED51
:10AA000013BA7BEE49BA1BEE900A09F08DF90BEEF2
:10AA1000900A1BEE100A19EE101A09F01FF90146F0
:10AA20004FF07E5009F01AF900EE100A60EE280A85
:10AA3000F4EEE0BAF1EE10FA1ED9219E96ED13BAAB
:10AA40003BEE091A11EE100A09F06EF90BEE900AAE
:10AA50001BEE100A1AEE901A09F000F901464FF0A9
:10AA60007E5009F0FBF801EE900A21EEA82AF4EEE0
:10AA7000C2BAF1EE10FA06D84FF00406219B83F813
:10AA80005060FEF7FEBF219BDD6C284609F04CF9B3
:10AA90000BEE100A284618EE101A09F0DFF80146EE
:10AAA0004FF07E5009F0DAF802EE900A22EEA83A52
:10AAB000B4EEC3BAF1EE10FA06D84FF00000219AB6
:10AAC00082F85000FEF7DDBF2199D1ED133AF4EE84
:10AAD000C83AF1EE10FA05DD4FF0010781F8507029
:10AAE000FEF7CFBFF4EEC83AF1EE10FA4CBF0222E7
:10AAF000032281F85020FEF7C4BF219FD7ED124AF0
:10AB000097ED135AC4EE855AC7ED135AC9E6219939
:10AB1000C86C09F079F8002840F09B86FEF7B1BFB9
:10AB2000219AD66C304609F0FFF80BEE100A304639
:10AB300018EE101A09F092F801464FF07E5009F015
:10AB40008DF806EE100A66EE286AB4EEE6BAF1EE6B
:10AB500010FA00F37E86FEF794BF2198C06C09F0CE
:10AB600053F8002800F07586FEF78BBF219B93ED0C
:10AB7000137AD3ED127AB4EEE77AF1EE10FA80F29E
:10AB80006886FEF77EBF219991ED130AD1ED120A76
:10AB9000B4EEE00AF1EE10FA00F35B86FEF771BF47
:10ABA000219A92ED131AD2ED121AB4EEE11AF1EED7
:10ABB00010FA40F24E86FEF764BF219890ED132AFA
:10ABC000D0ED122AB4EEE22AF1EE10FA00F141863D
:10ABD000FEF757BF219EF66C304609F0A5F80BEE44
:10ABE000100A304618EE101A09F038F801464FF0F6
:10ABF0007E5009F033F803EE100A63EE283AB4EE03
:10AC0000E3BAF1EE10FA40F22486FEF73ABF219D36
:10AC1000E86CFCF7C5FAE8640DF1700C4FF0000029
:10AC2000FCF75AFDFEF72DBF1D9BF62B08D942F607
:10AC3000EC54C2F200044FF01203237103F0B6BCCF
:10AC4000219FF86C08F0E0FF38B9219AD2ED134A41
:10AC5000B6EE005A34EE85BA06E0219991ED13BAAA
:10AC6000B6EE004A3BEE44BA1BEE100A08F0CCFFE9
:10AC700088B9B4EECABAF1EE10FA04DC1BEE100A81
:10AC800008F0C6FF38B14FF00100219E86F8500051
:10AC90006FF000402CE01BEE100A08F0B5FF88B101
:10ACA000B4EEE9BAF1EE10FA04D41BEE100A08F083
:10ACB000AFFF38B14FF00101219A82F850104FF0E8
:10ACC000004015E01BEE100A08F0B2FF38B14FF05B
:10ACD0000207219B83F850704FF0000008E0BDEEA2
:10ACE000CBBA1BEE100A4FF00006219D85F850608C
:10ACF0004FEA006545EA106700F47F4347EA032105
:10AD000000F47F0241EA122042F61C66C2F20006FD
:10AD10001D9D7051FEF7B5BE1D99F62908D942F662
:10AD2000EC54C2F200044FF01203237103F03EBC56
:10AD300042F61C67C2F200077A584FEA026040EA06
:10AD4000126602F47F4546EA052302F47F0143EAD6
:10AD5000112705EE907AB8EEE56A219880ED136A26
:10AD6000B4EECA6AF1EE10FA04DCB4EEE96AF1EE70
:10AD700010FA05D54FF0010680F85060FEF781BE4D
:10AD80004FF0000280F85020FEF77BBE0DF1700CF2
:10AD90004FF00100FCF7A0FC219DE86CFCF72AFABB
:10ADA0002199C864FEF76DBE219FD7ED136AB7EEF7
:10ADB000007A76EE877AC7ED137A13E6219FF86C56
:10ADC00008F036FF50B1219D4FF0000185F8471083
:10ADD0004FF0040785F85070FEF753BE219890EDB0
:10ADE000134AB4EEC84AF1EE10FA23DB9FEDD46AA1
:10ADF000B4EEC64AF1EE10FA0FD5FCEEC46A16EEB8
:10AE0000902A0DF1700CD0B2FCF77AFB4FF00006DF
:10AE1000219B83F85060FEF734BE0DF1700C4FF0AB
:10AE2000FF00FCF76DFB4FF00207219880F850708F
:10AE3000FEF727BEB4EEC84AF1EE10FA7EF521AE59
:10AE4000DFEDC04AB4EEE44AF1EE10FA11DDB1EEE6
:10AE5000445AFCEEC55A15EE903A0DF1700CD8B27A
:10AE6000FCF74EFB4FF00105219981F85050FEF799
:10AE700008BE0DF1700C4FF0FF00FCF741FB4FF0E6
:10AE80000302219E86F85020FEF7FBBD1D98F9288D
:10AE900008D942F6EC54C2F200044FF013002071BE
:10AEA00003F084BB219A92ED137AFDEEC77A17EE78
:10AEB000906A33B21C939DB2C6F3072141EA05277D
:10AEC00040F66C52C2F200021752FEF7DABD1D9A2C
:10AED000F92A08D942F6EC54C2F200044FF01302EA
:10AEE000227103F063BB219E96ED130AFCEEC00AAB
:10AEF00010EE903A9DB21C954FEA152141EA0527C4
:10AF000040F66C50C2F200008752FEF7BABD1D9E9B
:10AF1000219B9E64FEF7B5BD1D9D2199CD64FEF772
:10AF2000B0BD0DF1700CFCF703FB01EE100AF8EE5A
:10AF3000411A219FC7ED131AFEF7A3BD1D98F928EA
:10AF400008D942F6EC54C2F200044FF0130020710D
:10AF500003F02CBB40F66C52C2F20002165A4FEAC4
:10AF6000162343EA0625A9B202EE101AF8EE422A89
:10AF7000219FC7ED132AFEF784BD1D9BF92B08D92D
:10AF800042F6EC54C2F200044FF01303237103F0B5
:10AF90000DBB40F66C52C2F20002D65A4FEA16259B
:10AFA00045EA06218FB203EE107AF8EE433A219873
:10AFB000C0ED133AFEF765BD1D98072808D942F683
:10AFC000EC51C2F200014FF00800087103F0EEBA34
:10AFD000FCF7FAFE04EE100AF8EE444A219AC2ED9C
:10AFE000134AFEF74EBD219E96ED135AD6ED125A26
:10AFF00025EE256A86ED136A53E4219DD5ED136A8B
:10B00000B1EE667A85ED137AFEF73BBD4FF0000096
:10B010004FF001010A46FDF70DFE219F97ED130A3F
:10B02000F1EE047A60EE270A4FF0000300930193DB
:10B0300042F6C850C2F20000BCEEE01A11EE101A3F
:10B040004FF0FF0248F68543C0F60003FAF740FDD3
:10B05000FEF717BD1D99F72908D942F6EC54C2F244
:10B0600000044FF01300207103F0A0BA40F66C52B8
:10B07000C2F200025058FCF7BDF8219EB064FEF702
:10B0800000BD1D9BF72B08D942F6EC51C2F200011E
:10B090004FF013020A7103F089BA40F66C55C2F200
:10B0A0000005E858FCF7A6F8219FF864FEF7E9BC14
:10B0B0001D98072808D942F6EC54C2F200044FF05C
:10B0C0000801217103F072BA219ED6ED131AF4EE35
:10B0D000C81AF1EE10FA0DDBF4EEC91AF1EE10FA0F
:10B0E00008D8BCEEE12A8DED1C2A4FF0000586F849
:10B0F00050501FE0F4EEC91AF1EE10FA07DD6FF0C0
:10B100007F401C904FF0010386F8503012E04FF062
:10B1100000031C9311EE900A08F076FD28B14FF061
:10B120000201219A82F8501004E04FF00305219F9C
:10B1300087F850501D981C99FCF71EFEFEF7A1BC25
:10B1400000008043000080C3219EF06C08F070FD79
:10B1500000287EF496AC219FD7ED132AF4EEC82A7E
:10B16000F1EE10FA04DD4FF07E50F864FEF789BC72
:10B17000F4EEC82AF1EE10FA7EF583AC4FF000022F
:10B18000CBF68072FA64FEF77CBC219B9D6ACDB140
:10B19000FAF7D4FC219EB76AC7F1040210184CF6E6
:10B1A000CD43CCF6CC43A3FB00154FEA9501776A5B
:10B1B000B1FBF7F203EE102AF8EE433AC6ED133A6C
:10B1C000FEF75FBC4FF6FF71C7F67F71D964FEF7DB
:10B1D00058BC1D9EF72E08D942F6EC54C2F200046A
:10B1E0004FF01301217103F0E1B92198C06CFBF716
:10B1F000D7FF40F66C53C2F200039851FEF741BCF2
:10B20000219E96ED124AD6ED134A34EE645A86ED2D
:10B21000135AFFF746BB219FFA6C1C92B86CF86476
:10B22000BA64FEF72EBC2199C86C08F001FD30B15C
:10B230004FF00305219F87F85050FEF722BC219B59
:10B24000D86C08F0E5FC30B14FF00406219B83F880
:10B250005060FEF716BC219EF56C284608F064FD90
:10B260000BEE100A284618EE101A08F0F7FC0146FB
:10B270004FF07E5008F0F2FC05EE900A25EEA86A29
:10B28000B4EEC6BAF1EE10FA06D84FF000002199DC
:10B2900081F85000FEF7F5BB219FD7ED136AF4EE5D
:10B2A000C86AF1EE10FA05DD4FF0010287F8502070
:10B2B000FEF7E7BBF4EEC86AF1EE10FA4CBF0222CB
:10B2C000032287F85020FEF7DCBB219AD2ED13BA97
:10B2D00092ED12BA3BEECBCA1CEE100A08F024FD28
:10B2E0000CEE100A1BEE900A1BEE101A08F0B6FCCA
:10B2F00001464FF07E5008F0B1FC07EE100A27EE31
:10B30000280AB4EEC0CAF1EE10FA0DF1700C8CBF31
:10B3100000200120FCF7F4F8FEF7B3BB2198C66CBF
:10B32000304608F001FD0BEE100A304618EE101AF8
:10B3300008F094FC01464FF07E5008F08FFC07EEB9
:10B34000900A67EEA80AB4EEE0BAF1EE10FA0DF139
:10B35000700C8CBF00200120FCF7D2F8FEF791BBE7
:10B36000219991ED131AD1ED121AB4EEE11AF1EE12
:10B3700010FA0DF1700CB4BF00200120FCF7C0F8EA
:10B38000FEF77FBB219B93ED132AB5EEC02AF1EEA9
:10B3900010FA0DF1700CB4BF00200120FCF7B0F8DA
:10B3A000FEF76FBB219DD5ED132A95ED123AF4EE11
:10B3B000C32AF1EE10FA0DF1700CD4BF0020012069
:10B3C000FCF79EF8FEF75DBB219FD7ED133A97ED92
:10B3D000124AF4EEC43AF1EE10FA0DF1700C8CBF83
:10B3E00000200120FCF78CF8FEF74BBB219AD2ED30
:10B3F000134A92ED125AF4EEC54AF1EE10FA0DF12D
:10B40000700C54BF00200120FCF77AF8FEF739BB1E
:10B410002198D0ED135AF5EEC05AF1EE10FA0DF165
:10B42000700C54BF00200120FCF76AF8FEF729BB1E
:10B43000219ED6ED13BA96ED12BA3BEECB6A16EE0C
:10B44000100A08F071FC0CEE100A1BEE900A1BEEBD
:10B45000101A08F003FC01464FF07E5008F0FEFB86
:10B4600006EE900A26EEA87AB4EEC7CAF1EE10FAFC
:10B470000DF1700CD4BF00200120FCF741F8FEF75D
:10B4800000BB2199CD6C284608F04EFC0BEE100A4B
:10B49000284618EE101A08F0E1FB01464FF07E50E6
:10B4A00008F0DCFB00EE100A60EE287AB4EEE7BA92
:10B4B000F1EE10FA0DF1700CD4BF00200120FCF762
:10B4C0001FF8FEF7DEBA1D9BF82B08D942F6EC54A4
:10B4D000C2F200044FF01303237103F067B8FAF7C8
:10B4E0002DFB219F00F104004CF6CD42CCF6CC425E
:10B4F000A2FB00104FEA9006796AB6FBF1F51D9B9E
:10B5000040F66C52C2F20002D1184878D65C4FEA7D
:10B51000064343EA00208A7840EA02011B916D1A33
:10B5200025F07F461C9600EE906AB8EE601A87ED13
:10B53000131AFEF7A6BA219FF86CB864FEF7A1BAF9
:10B54000219A92F85110002940F08381FEF799BAB0
:10B55000219B93F85100002800F07B81FEF791BAFF
:10B560001D99FA2908D942F6EC54C2F200044FF0B2
:10B570001301217103F01AB840F66C52C2F20002B6
:10B58000535C002B7EF47DAA1E981C9063E11D9BEA
:10B59000FA2B08D942F6EC54C2F200044FF0130320
:10B5A000237103F003B840F66C52C2F20002D05C83
:10B5B00000283EF466AA1E991C914CE142F6EC501C
:10B5C000C2F200004FF00102027102F0EFBF1D99BC
:10B5D000F92908D942F6EC54C2F200044FF01203E4
:10B5E000237102F0E3BF42F61C63C2F20003585C11
:10B5F0001E9A10427EF445AA1F991C912BE11D98BA
:10B60000F92808D942F6EC54C2F200044FF01202B5
:10B61000227102F0CBBF42F61C62C2F20002115C42
:10B620001E9B19423EF42DAA1F981C9013E11D99F0
:10B63000FA2908D942F6EC54C2F200044FF0130183
:10B64000217102F0B3BF40F66C53C2F20003585CA4
:10B6500000287EF416AA1E9A1C922DE11D9BFA2B3F
:10B6600008D942F6EC54C2F200044FF013032371E0
:10B6700002F09CBF40F66C50C2F20000C25C002A8F
:10B680003EF4FFA91E991C9116E11D98FA2808D9CD
:10B6900042F6EC54C2F200044FF01302227102F0A1
:10B6A00085BF40F66C52C2F20002115C1E9B9942AB
:10B6B0007EF6E7A91F981C90CDE01D99FA2908D9BC
:10B6C00042F6EC54C2F200044FF01303237102F06F
:10B6D0006DBF40F66C53C2F20003585C1E9A904254
:10B6E000FEF4CFA91F991C91B5E01D98FA2808D93E
:10B6F00042F6EC54C2F200044FF01302227102F041
:10B7000055BF40F66C52C2F20002115C1E9B99427A
:10B710007EF4B7A91F981C909DE01D99FA2908D9BD
:10B7200042F6EC54C2F200044FF01303237102F00E
:10B730003DBF40F66C53C2F20003585C1E9A904223
:10B740003EF49FA91F991C9185E01D98FA2808D9FD
:10B7500042F6EC54C2F200044FF01302227102F0E0
:10B7600025BF40F66C52C2F20002115C1E9B99424A
:10B770003EF687A91F981C906DE01D99FA2908D9FB
:10B7800042F6EC54C2F200044FF01303237102F0AE
:10B790000DBF40F66C53C2F20003585C1E9A9042F3
:10B7A000BEF46FA91F991C9155E0219890F847208D
:10B7B0001D998A427EF465A91E9B1C937CE021980A
:10B7C00090F847201D998A423EF45BA91E9B1C936A
:10B7D00072E0219890F847201D998A427EF651A97F
:10B7E0001E9B1C9368E0219890F847201D998A427F
:10B7F000FEF447A91E9B1C935EE0219890F8472019
:10B800001D998A42BEF43DA91E9B1C9354E02198C9
:10B8100090F847201D998A423EF633A91E9B1C933F
:10B820004AE09DF874000DF16B01FDF72FF98DF8DA
:10B830006A009DF86B1031B142F6EC54C2F200047C
:10B84000217102F0B3BE00283EF41BA91E981C9083
:10B8500001E01D9A1C921C984AF60003C0F60103F1
:10B8600093F82E1093F82F2042EA0123834208D246
:10B8700042F6EC54C2F200044FF00900207102F0CD
:10B8800095BE42F61C75C2F200052860FEF7F9B8B5
:10B890000DF1700CFBF74CFE1C900028D9D0FEF780
:10B8A000F0B80DF1700CFBF743FE1C900028D0D1CE
:10B8B000FEF7E7B81D9B1C93219A136A052B08D944
:10B8C00042F6EC54C2F200044FF00A03237102F076
:10B8D0006DBE03F1020042F61C71C2F2000109685C
:10B8E00042F8201003F10103219A1362B3E70DF12E
:10B8F000700CFBF71DFE1C900028DBD0FEF7C1B8D2
:10B900000DF1700CFBF714FE1C900028D2D1FEF74D
:10B91000B8B80DF1700CFBF70BFE1C901D99884216
:10B920007EF4AFA81E981C9095E70DF1700CFBF704
:10B93000FFFD1C901D9A90423EF4A3A81E9B1C93F1
:10B9400089E70DF1700CFBF7F3FD1C901D998842FF
:10B950007EF697A81E981C907DE70DF1700CFBF702
:10B96000E7FD1C901D9A9042FEF48BA81E9B1C9331
:10B9700071E70DF1700CFBF7DBFD1C901D998842FF
:10B98000BEF47FA81E981C9065E70DF1700CFBF7C4
:10B99000CFFD1C901D9A90423EF673A81E9B1C93EF
:10B9A00059E79DF874000DF16B01FDF73FF88DF834
:10B9B0006A009DF86B1031B142F6EC54C2F20004FB
:10B9C000217102F0F3BD00283EF45BA81E981C9084
:10B9D00041E79DF874000DF16B01FDF727F88DF834
:10B9E0006A009DF86B3033B142F6EC51C2F20001AF
:10B9F0000B7102F0DBBD00287EF443A81E9A1C9256
:10BA000029E70DF1700CFBF7BBFD40F66C50C2F25C
:10BA100000001E9BC25C1D990A423EF432A81F988A
:10BA20001C9018E70DF1700CFBF7AAFD40F66C5264
:10BA3000C2F200021E9BD15C1D9801427EF421A837
:10BA40001F9A1C9207E70DF1700CFBF799FD40F669
:10BA50006C51C2F200011E9BC85C1D9A10427EF41C
:10BA600010A81F991C9127E70DF1700CFBF788FDBA
:10BA700040F66C50C2F200001E9BC25C1D990A4247
:10BA80003DF4FFAF1F981C9016E798F8005045F062
:10BA9000080088F80000FEF71DB80DF1700CFBF7E8
:10BAA00047FD8DF86A00219991F851201D9BD1180E
:10BAB0001C911E9AC2F1FB03994208D942F6EC543C
:10BAC000C2F200044FF01303237102F06FBD4FF078
:10BAD00000061B961E9FEFB11C9940F66C55C2F2F2
:10BAE00000056A5C824236D007F1FF3240F66C53A3
:10BAF000C2F200035B1840F66C56C2F20006C6F1B3
:10BB00000107C1F10101C6EB010E12F0010F1AD0BD
:10BB100002F0AABD4FF0FF001B901CE013F8019F3C
:10BB200002F1FF35484504D11C91CDF86CC01E923E
:10BB300011E02A46F9180EEB030C13F8016FB0421E
:10BB400042F09F85F0E7F9180EEB030C002AE5D1CF
:10BB50001C911E92DEE70DF1700C9DF86C00FBF756
:10BB6000CFFCFDF78EBF0DF1700CFBF7E1FC41F24D
:10BB7000E87BC2F2000B8BF800004FF001011C9132
:10BB8000CDF834B095E0219A92F851001D9BC11870
:10BB90001C91F92908D942F6EC54C2F200044FF086
:10BBA0001302227102F002BD1E981B900DF1700C61
:10BBB00026AF47F0010122AD45F001024FF000032E
:10BBC000FBF7F0FCFDF75DBF219890F851101D9B2D
:10BBD000CA181C92FA2A08D942F6EC54C2F20004A0
:10BBE0004FF01300207102F0E1BC1F9E1E98B0427E
:10BBF00028BF30461B900DF1700C26AF47F00101B5
:10BC000022AD45F001024FF00003FCF705FDFDF702
:10BC100038BF0DF1700CFBF78BFC034641F2E87B5B
:10BC2000C2F2000B58464FF0100148F67852C0F6A9
:10BC3000010208F0C3F91C90CDF834B039E01E9928
:10BC40001C911F9B1B934FF000020D9231E04FF0AF
:10BC5000FF301C900D902CE0219EF06C9DF8781028
:10BC60009DF87C2041F2E876C2F2000600964FF083
:10BC7000100301934FF00103FDF75AFB4FF0FF3122
:10BC80001C910D9615E0219AD06C9DF878109DF8C6
:10BC90007C2041F2E876C2F2000600964FF01003D5
:10BCA00001934FF00003FDF743FB4FF0FF301C9072
:10BCB0000D961D9B03F10500C1B20C91A3F1FB028F
:10BCC000032A23D840F6AC63C2F200034FF411708C
:10BCD0000C9900FB013292F82032032B08D042F677
:10BCE000EC54C2F200044FF04802227102F05EBC34
:10BCF00040F6AC66C2F200064FF411770C9807FBD1
:10BD0000006707F104074FF0000605E0219F97F850
:10BD10005160F6184FF00007DDF870B0BBF1FF3F3F
:10BD20000CD14FF0FF0B4FF00009C84640F66C51A4
:10BD3000C2F200010E910F950D9D05E0BBF1000FC1
:10BD4000F1D14FF0000961E01D9AA2F1FB02032A34
:10BD500010D8D7F80061FF2E14BF01364646D7F839
:10BD600004319E4206D14046FCF7C2FBD7F80401DD
:10BD70008642F8D0B5F1FF3F15D1219850F8343FF5
:10BD80001968D1F800C0494610AA4FF00103E047F6
:10BD90008DF86B0080B10F9D42F6EC51C2F20001AC
:10BDA000087102F003BC25B115F809208DF8402078
:10BDB00002E01B998DF840101C98B0F1FF3F02D1B2
:10BDC0009DF8402012B31D9BA3F1FB03032B07D862
:10BDD000D7F800319DF84000F854C7F8006111E031
:10BDE000FA2E09D90F9D42F6EC54C2F200044FF02E
:10BDF0001302227102F0DABB9DF840000E998855BB
:10BE000006F1010609F10109D9459DD31D9EA6F150
:10BE1000FB06032E04D80C98FBF718FEFDF731BE85
:10BE2000219F97F8515009EB050E87F851E0FDF777
:10BE300028BE1D9AA2F1FB0103295AD802F105027E
:10BE4000D7B240F6AC61C2F200014FF4117202FBAE
:10BE5000071393F82002032808D042F6EC54C2F2EC
:10BE600000044FF04803237102F0A0BB40F6AC661B
:10BE7000C2F200064FF4117505FB076505F10405D4
:10BE80001E9901F1FF321E9271B34FF0000842F685
:10BE90001C79C2F200094AF600039B46C0F6010B6A
:10BEA000D5F80061FF2E14BF01364646D5F80401CF
:10BEB000864206D14046FCF71BFBD5F804118E42A2
:10BEC000F8D0D9F80030D5F800211BF80300A854A9
:10BED00003F10103C9F80030C5F800611E9E06F1A8
:10BEE000FF311E91002EDBD13846FBF7AFFDFDF789
:10BEF000C8BD1E9B1C93219991F8510082181B927A
:10BF0000C3F1FB06B24208D942F6EC54C2F2000477
:10BF10004FF01300207102F049BBC71881F851702F
:10BF20001C9A02F1FF351C95002A3DF4AAAD42F699
:10BF30001C76C2F2000636681B9F40F66C53C2F2B4
:10BF40000003D9194AF60000C0F6010030184FF07E
:10BF5000000305F0010E10F803C001F803C003F15F
:10BF60000103934242F071830DE010F8038001F861
:10BF7000038003F1010310F803E001F803E003F18B
:10BF800001039342F1D1E819A91901F1010142F627
:10BF90001C72C2F2000211604FF0FF331C9300F1DB
:10BFA00001001B90FDF76DBD4FF000028DF86A2077
:10BFB000219991F851201D9BD0181C901E9A1B921C
:10BFC000C2F1FB03984208D942F6EC54C2F20004D5
:10BFD0004FF01302227102F0E9BA40F66C57C2F238
:10BFE000000707EB00099DF87CB042F61875C2F215
:10BFF00000052E68886B3118335CFF2B52D08846C1
:10C000004FF0010709970C9498F8014004EB0323C3
:10C0100042F61875C2F200052E68F0184FF00001C4
:10C020001C919DF86A20002A02F0E482F75C00F17E
:10C03000010002F0E1BA9DF86A5015B15FB90C9C9D
:10C0400002E0607838B90C9C219E96F851001D18CA
:10C0500086F8515029E014F8015F19F803B046B989
:10C06000284607F04FFFC5B2584607F04BFF5FFA6E
:10C0700080FB5D4508D11C9B03F101031C9307F174
:10C08000FF371B999942D6D2B346099A02F10102B1
:10C09000099218F8023FFF2BB6D10C9C4FF0000715
:10C0A000099702E04FF0000209920DF1700C099916
:10C0B000C8B2FBF725FAFDF7E4BC4FF001008DF89C
:10C0C0006A0075E70DF1700CFBF732FA034641F296
:10C0D000E87BC2F2000B58464FF0100148F6805240
:10C0E000C0F6010207F06AFF1C90CDF834B0E0E51D
:10C0F0000DF1700CFBF71CFA034641F2E87BC2F22B
:10C10000000B58464FF0100148F68852C0F6010265
:10C1100007F054FF1C90CDF834B0CAE50DF1700C57
:10C12000FBF706FA034641F2E87BC2F2000B5846E1
:10C130004FF0100148F68C52C0F6010207F03EFFA6
:10C140001C90CDF834B0B4E50DF1700CFBF7F0F9AC
:10C15000034641F2E87BC2F2000B58464FF0100153
:10C1600048F69452C0F6010207F028FF1C90CDF863
:10C1700034B09EE5219B93F8510000F1010083F853
:10C180005100FDF77EBC1D9E40F66C57C2F20007C1
:10C19000BD5D05F10105BD55FDF773BC219991F811
:10C1A000472002F1010281F84720FDF76ABC9DF8A3
:10C1B00074000DF16B01FCF739FC0DF1700CFBF70D
:10C1C0009FF99DF86B30002B3DF45BAC42F6EC54CC
:10C1D000C2F20004237102F0E9B99DF874000DF178
:10C1E0006B01FCF78BFC0DF1700CFBF789F99DF8E6
:10C1F0006B0000283DF445AC42F6EC51C2F2000160
:10C20000087102F0D3B91D9A1C924FF000031B93E2
:10C210004FF001008DF86A009DF870000DF16B0180
:10C22000FCF704FC9DF86B1099B920B19DF86A20C9
:10C230001B9B13431B939DF86A004FEA40018DF846
:10C240006A101C9A02F101021C9211F0FE0FE3D158
:10C250000AE09DF86A30012B06D142F6EC54C2F296
:10C260000004217102F0A2B90DF1700C9DF86C0070
:10C27000FBF746F9FDF705BC1D981C904FF0000137
:10C280001B914FF001028DF86A209DF870000DF1AE
:10C290006B01FCF733FC9DF86B309BB920B19DF826
:10C2A0006A001B9901431B919DF86A204FEA4203E3
:10C2B0008DF86A301C9800F101001C9013F0FE0FFD
:10C2C000E3D10AE09DF86A10012906D142F6EC5448
:10C2D000C2F20004237102F069B90DF1700C9DF8EF
:10C2E0006C00FBF70DF9FDF7CCBB9DF874000DF168
:10C2F0006B01FCF7CBFB8DF86A009DF86B3033B116
:10C3000042F6EC52C2F20002137102F04FB90DF185
:10C31000700CFBF7F5F8FDF7B4BB1D981C904FF0BF
:10C3200000011B914FF001038DF86A30219A92F8B9
:10C33000470003420ED09DF870000DF16B01FCF731
:10C34000A5FB9DF86B309BB920B19DF86A101B9A34
:10C350000A431B929DF86A004FEA40038DF86A3049
:10C360001C9901F101011C9113F0FE03DED10AE0DA
:10C370009DF86A20012A06D142F6EC54C2F200046C
:10C38000237102F013B91B9E219F87F84760FDF7C8
:10C3900078BB9DF874000DF16B01FCF7DFFB0DF12C
:10C3A000700CFBF7ADF89DF86B0000283DF469AB0D
:10C3B00042F6EC51C2F20001087102F0F7B81D9B81
:10C3C0001C93D8B20DF16B01FCF7C8FB1B909DF8D4
:10C3D0006B0030B142F6EC54C2F20004207102F05E
:10C3E000E5B84FF001058DF86A501C9A51191C915F
:10C3F000C8B20DF16B01FCF7B1FB9DF86A6000FA61
:10C4000006F01B9F07431B9706F101068DF86A6033
:10C410001C9901F101011C91F3B2072BE8D90DF130
:10C42000700C9DF86C00FBF76BF8FDF72ABB0DF163
:10C43000700C219890F85100FBF762F8FDF721BBD2
:10C44000FDF71FBB42F6B155C2F200054FF00102E5
:10C450002A70FDF716BB42F6B156C2F200064FF045
:10C4600000073770FDF70DBB21984FF000014FF02A
:10C47000540208F0D9F94FF00001219141F2F8730C
:10C48000C2F200031C6804F1FF30186001F0F7BF2E
:10C4900041F2F873C2F2000318683F2808D942F647
:10C4A000EC54C2F200044FF03002227102F07EB868
:10C4B0004FF001051C9541F64806C2F20006B76D23
:10C4C000002F42F0A48005E0D2F8AC10002949D139
:10C4D0001C9301E04FF001031D9F41F64805C2F295
:10C4E00000054FF0540606FB03F3EA18EF505760BF
:10C4F0001E9982F852104FF00A005062104600F167
:10C500003400219901F134014FF0100208F068F96C
:10C510001C9B06FB035000F14400219901F14401EA
:10C520004FF0040208F05CF91C9F06FB075000F175
:10C530004800219901F148014FF0080208F050F934
:10C54000219A92F851101C9806FB005585F851105D
:10C5500041F2F876C2F20006336803F1010333605A
:10C56000FDF78FBA03F101052B4602F15402D2F810
:10C57000AC00002842F05980AAE71C93FDF781BA6D
:10C58000219A92F852101E9182E70DF1700CFAF781
:10C59000CFFF1E907CE71D9F219981F85170FDF718
:10C5A00070BA0DF1700C9DF87400FAF7A9FFFDF751
:10C5B00068BA2198836A002B3DF463AAF9F7BEFAA2
:10C5C00021998A6A801A496A1D9B01FB03F303EBD8
:10C5D00083029042BDF455AA1E981C90FFF73BB908
:10C5E000F9F7ACFA219DA862FDF74BBA42F61C613F
:10C5F000C2F2000191F8FB201E995318FB2B08D9B9
:10C6000042F6EC51C2F200014FF012030B7101F03F
:10C61000CDBF1D9BC2F1FB00834208DD42F6EC5406
:10C62000C2F200044FF01302227101F0BFBF42F6C4
:10C630001C66C2F20006701840F66C57C2F2000782
:10C64000F91808F0CDF8FDF71CBA98F8005045F03D
:10C65000100088F80000FDF73DBA219E96F847705B
:10C66000002F0CBFFF22002286F84720FDF709BAF1
:10C67000219991F847306FEA030581F84750FDF79B
:10C6800000BA0DF1700CFAF77BFF1E9E40F66C5756
:10C69000C2F20007B85D1D9A4240BA55FDF7F1B9E4
:10C6A0002199886B1D9B1A181C92A1E12199C86BD6
:10C6B0008B6BC2181C929BE12199086C40B942F621
:10C6C000EC54C2F200044FF02003237101F06EBF5E
:10C6D00000F1FF350D64FDF7D4B9219A116C01F119
:10C6E0000101116400297DF4CCA942F6EC50C2F29C
:10C6F00000004FF02004047101F058BF219B5A6BD9
:10C700001168486840B942F6EC51C2F200014FF09E
:10C710001E020A7101F04ABF0DF1700CFAF708FF12
:10C720001C90219850F8346F33685E681D991CAADC
:10C730004FF00103B0478DF86B0000283DF4A1A92C
:10C7400042F6EC54C2F20004207101F02FBF0DF14B
:10C75000700CFAF7EDFE1C9038E10DF1700CFAF751
:10C76000E7FE219FF863FDF78CB90DF1700CFAF725
:10C77000DFFE219D2864FDF784B9219850F8346FBD
:10C7800033681E681D991CAA4FF00103B0478DF84D
:10C790006B0030B142F6EC54C2F20004207101F09B
:10C7A00005BF0DF1A80C1CF8380DFAF7A9FEFDF72E
:10C7B00068B92198416B0DF1700C087AFAF7A0FE68
:10C7C000FDF75FB90DF1700C219A92F83C00FAF771
:10C7D00097FEFDF756B9219B186CFF2808D942F641
:10C7E000EC54C2F200044FF02001217101F0DEBED2
:10C7F0000DF1700CC0B2FAF783FEFDF742B9219833
:10C8000050F8347F3D68AE68B04701EE900AB8EE4C
:10C81000612A219A82ED132AFDF733B9219BD3EDCA
:10C820000E2AB8EE623A83ED133AFDF72AB9219841
:10C83000D0ED103AB8EE634A80ED134AFDF721B906
:10C840002199D1ED134ABCEEE45A8DED1C5ACFE08C
:10C85000219AD2ED135A9FEDC16AF4EEC65AF1EE59
:10C8600010FA08DB42F6EC54C2F200044FF0200349
:10C87000237101F09BBEFCEEE56AC2ED106AFDF784
:10C8800000B9219850F8346F31680E681D991CAAC0
:10C890004FF00403B0478DF86B0030B142F6EC5214
:10C8A000C2F20002107101F081BE1C98FAF7A2FCDE
:10C8B000219FB864FDF7E5B8219850F8343F1E6811
:10C8C00036681D991CAA4FF00403B0478DF86B0021
:10C8D00030B142F6EC54C2F20004207101F066BEA1
:10C8E0001C98FAF787FC219DE864FDF7CAB82198E7
:10C8F000416B0A68536843B942F6EC50C2F200003B
:10C900004FF01E02027101F051BEC06CFAF748FCF4
:10C910001C90219850F8346F31684E681D991CAAFC
:10C920004FF00403B0478DF86B0000283DF4A9A830
:10C9300042F6EC54C2F20004207101F037BE1D9A99
:10C940002198C36BC3F1FB018A4208D942F6EC542B
:10C95000C2F200044FF01300207101F027BE50F81E
:10C96000347F3E6836684FF0000140F66C57C2F2E3
:10C970000007BA18B0478DF86B0000283DF481A875
:10C9800042F6EC53C2F20003187101F00FBE219879
:10C9900050F8342F11680E681D991BAA4FF004033C
:10C9A000B0478DF86B0030B142F6EC54C2F200048F
:10C9B000207101F0FBBD1B9B98B2C3F3072242EA32
:10C9C00000218BB21C9313E01D981C901C98219998
:10C9D000FAF74CFE8DF86B0000283DF452A842F6A1
:10C9E000EC52C2F20002107101F0E0BD1D991C91E1
:10C9F0001C98B0F5803F08D342F6EC54C2F2000414
:10CA00004FF01F02227101F0D1BD219DA863FDF7F7
:10CA100038B81D9D219FFD63FDF733B81D9E219BF6
:10CA20001E64FDF72EB82198826B1D99531A1C9332
:10CA3000DEE71E9A219BD96B8818FB2808D942F69D
:10CA4000EC53C2F200034FF012021A7101F0AEBDB6
:10CA500042F61C67C2F2000787F8FB10184650F830
:10CA6000346F31680E681D99BA18DB6BB0478DF8CA
:10CA70006B0000283DF405A842F6EC54C2F2000415
:10CA8000207101F093BD2198466B31684E6846B91C
:10CA900042F6EC51C2F200014FF01E020A7101F0A1
:10CAA00085BD1D9AC36BC3F1FB018A4208D942F6CA
:10CAB000EC50C2F200004FF01303037101F076BD99
:10CAC00000F134004FF0000140F66C57C2F200074D
:10CAD000BA18B0478DF86B0000283CF4D2AF42F68C
:10CAE000EC54C2F20004207101F060BDF7F78EFB38
:10CAF00000287CF4C6AF1D981C90FEF7ACBEF7F77B
:10CB000085FB00283CF4BDAF1D9B1C93FEF7A3BE24
:10CB10001D990B2908D942F6EC54C2F200044FF0DB
:10CB20000502227101F042BDC8B24FF00001F7F7D3
:10CB30002BFB07EE100AB8EE470A219F87ED130A78
:10CB4000FCF79FBF1D980B280AD942F6EC53C2F29E
:10CB500000034FF00501197101F028BD0000804766
:10CB6000C0B24FF00101F7F70FFB07EE900AF8EEA5
:10CB7000670A219DC5ED130AFCF783BF1D9A0B2A96
:10CB800008D942F6EC54C2F200044FF005002071BF
:10CB900001F00CBDD0B24FF00001F7F765FAFCF7D9
:10CBA00070BF1D9B0B2B08D942F6EC51C2F200015D
:10CBB0004FF005020A7101F0F9BCD8B24FF0010143
:10CBC000F7F752FAFCF75DBF1D980B2808D942F61B
:10CBD000EC54C2F200044FF00503237101F0E6BCEF
:10CBE000C0B24FF00001F7F78FFAFCF74ABF1D996A
:10CBF0000B2908D942F6EC50C2F200004FF00502B2
:10CC0000027101F0D3BCC8B24FF00101F7F77CFA12
:10CC1000FCF737BF9DF87400F4F78EFC00287CF415
:10CC200030AF42F6EC54C2F200044FF028032371F7
:10CC300001F0BCBC9DF87400219901F14C01F4F79E
:10CC40009BFC00287CF41DAF42F6EC51C2F20001BF
:10CC50004FF02800087101F0A9BC219A92ED131A37
:10CC60009DF87400FCEEC11A11EE901AF4F7B6FCB0
:10CC700000287CF406AF42F6EC54C2F200044FF0F8
:10CC80002803237101F092BCFCF7FBBE0DF1700C80
:10CC9000FAF74EFC30B9219E96F847703D1C18BF3C
:10CCA000012501E04FF00105219981F84750FCF77B
:10CCB000E8BE9DF874600DF1700CFAF739FC01467E
:10CCC00030464FF00102FBF7B5FF8DF86B000028EE
:10CCD0003CF4D7AE42F6EC52C2F20002107101F001
:10CCE00065BC0DF1700CFAF723FC01468DF86A0063
:10CCF0009DF87400FBF760FF8DF86B0000283CF492
:10CD0000C0AE42F6EC54C2F20004207101F04EBCF9
:10CD10001D981C904FF001038DF86A301E46219A31
:10CD200092F847100B420AD092F846109DF8700016
:10CD300019403246FBF77EFF8DF86B0068B99DF80D
:10CD40006A304FEA43008DF86A001C9A02F1010232
:10CD50001C9210F0FE03E2D10AE09DF86A1001294E
:10CD600006D142F6EC54C2F20004207101F01EBC60
:10CD70004FF000068DF86B600DF1700CFAF7D8FBE0
:10CD80000DF1700CFAF7D4FBFCF77BBE9DF8740034
:10CD90004FF001010A46FBF74DFF8DF86B000028AC
:10CDA0003CF46FAE42F6EC52C2F20002107101F098
:10CDB000FDBB9DF874004FF000014FF00102FBF73E
:10CDC00039FF8DF86B0000283CF45BAE42F6EC5363
:10CDD000C2F20003187101F0E9BB0DF1700CFAF713
:10CDE000A7FB219F97F84750284387F84700FCF797
:10CDF00048BE1D980DF1A80C4CF8380DFBF738F81B
:10CE000000287CF43EAE42F61C70C2F20000099984
:10CE1000016001F04BBB10A8FAF7C8FE014640B113
:10CE20009DF84060022E04D0D1484FF00D0207F06B
:10CE3000D7FC0DF1700C9DF84000FAF761FBFCF790
:10CE400020BEFBF769FBFCF71CBE0DF1700CFAF776
:10CE50006FFBFCF716BE1D9EFA2E08D942F6EC5465
:10CE6000C2F200044FF01203237101F09FBB0DF1D9
:10CE7000700CFAF75DFB42F61C62C2F2000290559C
:10CE8000FCF7FFBD0DF1700CFAF752FB42F61C6780
:10CE9000C2F2000787F8FB00FCF7F3BD0DF1700C40
:10CEA000219D95F84700FAF72BFBFCF7EABD1D988A
:10CEB000FA2808D942F6EC54C2F200044FF01202EC
:10CEC000227101F073BB0DF1700C42F61C61C2F2CD
:10CED0000001085CFAF714FBFCF7D3BD0DF1700CF0
:10CEE00042F61C66C2F2000696F8FB00FAF708FB51
:10CEF000FCF7C7BD1D9EF62E08D942F6EC50C2F2D3
:10CF000000004FF01201017101F050BB219B986CA1
:10CF1000FAF746F942F61C67C2F20007B851FCF76F
:10CF2000B0BD1D9BFA2B08D942F6EC54C2F20004A6
:10CF30004FF01302227101F039BB0DF1700C40F675
:10CF40006C55C2F20005E85CFAF7DAFAFCF799BD15
:10CF50000DF1700CFAF714FB40F66C56C2F20006A5
:10CF60001E9FF05D1D9908420DF1700C0CBF002052
:10CF7000FF20FAF7C5FAFCF784BD1D9BF92B08D9F1
:10CF800042F6EC51C2F200014FF013020A7101F0B7
:10CF90000DBB40F66C52C2F20002D05CD1184B7847
:10CFA00043EA00221C92002A3CF46BADFEF753BC0E
:10CFB0001D9BFA2B08D942F6EC54C2F200044FF044
:10CFC0001302227101F0F2BA40F66C50C2F2000076
:10CFD000C15C002943D1FCF754BD1D9BFA2B08D935
:10CFE00042F6EC54C2F200044FF01302227101F039
:10CFF000DDBA40F66C50C2F20000C15C79B3FCF7B8
:10D0000040BD0DF1700CFAF793FA1C9038BBFCF799
:10D0100038BD0DF1700CFAF7B3FA40F66C50C2F25D
:10D0200000001E9BC15C1D9A114218D0FCF729BD5F
:10D030000DF1700CFAF7A4FA40F66C50C2F2000041
:10D040001E9BC15C1D9A114209D1FCF71ABD0DF15E
:10D05000700CFAF76DFA1C9000287CF412AD219840
:10D06000026A42B942F6EC54C2F200044FF00301E6
:10D07000217101F09BBA02F1FF35056202F1010254
:10D0800050F8226042F61C77C2F200073E60FCF7BF
:10D09000F8BC219E96F847704FEAD71545EA47003D
:10D0A00086F84700FCF7EDBC219B93F847204FEA38
:10D0B000520141EAC21683F84760FCF7E2BCFAF776
:10D0C00047FEFCF7DEBC40F66457C2F20007FD786D
:10D0D0004FF0010000FA05F03B7923EA00033B71B1
:10D0E000FCF7CFBC42F6EC54C2F200044FF0010250
:10D0F000227101F05BBA40F66451C2F20001CE78B1
:10D1000046B940F66450C2F200004FF00603C37007
:10D11000FCF7B7BC06F1FF3740F66455C2F20005D4
:10D12000EF70FCF7AEBC40F66452C2F20002117818
:10D1300001F1FF36F7B217701579FF2D0BD1632F70
:10D140007CF69FAC40F66451C2F200014FF06302DE
:10D150000A70FCF796BC172F7CF693AC40F664502F
:10D16000C2F200004FF017030370FCF78ABC00BF47
:10D17000720D002040F66456C2F20006777807F17F
:10D18000FF35E8B270703379FF2B0BD100287CF4A7
:10D1900078AC40F66456C2F200064FF00C07777088
:10D1A000FCF76FBC3B287CF66CAC40F66451C2F2D5
:10D1B00000014FF03B024A70FCF763BC42F6EC54AE
:10D1C000C2F200044FF00100207101F0EFB942F605
:10D1D000EC53C2F200034FF00101197101F0E6B9FE
:10D1E00042F6EC54C2F200044FF00102227101F049
:10D1F000DDB942F6EC50C2F200004FF001030371BA
:10D2000001F0D4B940F66455C2F20005EE78052E5F
:10D2100008D940F66451C2F200014FF00002CA7012
:10D22000FCF72FBC06F1010640F66457C2F2000776
:10D23000FE70FCF726BC40F66450C2F20000037892
:10D2400003F10103DDB205700679FF2E0BD1632DCA
:10D250007CF617AC40F66450C2F200004FF00002BA
:10D260000270FCF70EBC172D7CF60BAC40F6645731
:10D27000C2F200074FF000013970FCF702BC40F623
:10D280006455C2F200056B7803F10103DEB26E70E3
:10D290002F79FF2F0BD10C2E7CF6F3AB40F66455A3
:10D2A000C2F200054FF001026A70FCF7EABB3B2EA8
:10D2B0007CF6E7AB40F66451C2F200014FF000008B
:10D2C0004870FCF7DEBB42F6EC54C2F200044FF0AB
:10D2D0000103237101F06AB940F66456C2F20006F8
:10D2E000F7784FF0010101FA07F1307981EA000582
:10D2F0003571FCF7C6BB0DF1700CFAF719F940F661
:10D300006452C2F200021071FCF7BBBB0DF1700C4D
:10D31000FAF70EF9062840F66453C2F2000392BFF2
:10D32000D8700026DE70FCF7ACBB0DF1700CFAF77C
:10D33000FFF840F66457C2F200073870FCF7A1BB53
:10D340000DF1700CFAF7F4F840F66451C2F20001E6
:10D350004870FCF796BB0DF1700CFAF7E9F840F64F
:10D360006455C2F20005A870FCF78BBB0DF1700C80
:10D3700040F66450C2F200000079FAF7C1F8FCF7F9
:10D3800080BB0DF1700C40F66452C2F20002D078FE
:10D39000FAF7B6F8FCF775BB0DF1700C40F6645364
:10D3A000C2F200031878FAF7ABF8FCF76ABB0DF18C
:10D3B000700C40F66456C2F200067078FAF7A0F8D6
:10D3C000FCF75FBB0DF1700C40F66457C2F200072A
:10D3D000B878FAF795F8FCF754BB42F6EC54C2F271
:10D3E00000044FF00101217101F0E0B81D9A0F2AED
:10D3F00008D942F6EC54C2F200044FF02700207125
:10D4000001F0D4B840F66C65C2F2000505EB82006D
:10D4100040F66453C2F2000315F822601E7047788C
:10D420005F704FF000019970D97082781A71FCF723
:10D4300028BB42F6EC53C2F200034FF00101197110
:10D4400001F0B4B840F66455C2F20005EE784FF032
:10D45000010707FA06F72A7947EA02002871FCF764
:10D4600010BB42F6EC54C2F200044FF001032371EA
:10D4700001F09CB842F6EC51C2F200014FF00102FB
:10D480000A7101F093B84FF00005139512951195AC
:10D49000199540F66456C2F20006377807F1640722
:10D4A0001697707800F1FF331593B178149111A895
:10D4B00006F0BCFF179A1AB102F1FF36F5B201E08F
:10D4C0004FF0060540F66457C2F20007FD70FCF706
:10D4D000D8BA1D9A0F2A08D942F6EC54C2F20004B9
:10D4E0004FF02702227101F061B840F66C60C2F281
:10D4F000000000EB820140F66453C2F200031D7885
:10D5000000F822505E784E701F798F70FCF7B9BA20
:10D5100042F6EC50C2F200004FF00101017101F03F
:10D5200045B80DF1700C219B93F85000F9F7E8FF16
:10D53000FCF7A7BA41F63C04C2F20004227812F0CC
:10D54000010F08D142F6EC50C2F200004FF030015A
:10D55000017101F02BB841F2F870C2F200000168CD
:10D5600041B942F6EC54C2F200044FF0310222718C
:10D5700001F01CB841F63C03C2F200031C7804F031
:10D58000FE0242F00400187042F6A051C2F20001FF
:10D590004FF000030B6000F072BF41F63C03C2F293
:10D5A00000031C7814F0010F08D142F6EC50C2F2CF
:10D5B00000004FF03002027100F0F8BF41F2F87243
:10D5C000C2F20002106840B942F6EC53C2F2000306
:10D5D0004FF034041C7100F0E9BF41F63C01C2F287
:10D5E00000010B7803F0FE0444F002020A7042F6D8
:10D5F000A050C2F200004FF00001016000F03FBFF8
:10D60000219D95F846600DF1700CF9F791FF219F6F
:10D61000311A97F8503003F001000A1A1C9287F86B
:10D620004720FF2A94BF0022012287F85020FCF7F0
:10D6300028BA1D9BFA2B08D942F6EC54C2F200041A
:10D640004FF01301217100F0B1BF40F66C55C2F2EA
:10D6500000051E9EEE54FCF714BA4FF000071C970D
:10D660001AE04FF001001C9016E04FF002021C92ED
:10D6700012E04FF003031C930EE04FF004051C95DD
:10D680000AE04FF005061C9606E04FF006011C91DB
:10D6900002E04FF007071C971D991B911C98FAF7A1
:10D6A0006BFBFCF7EEB90DF1700CF9F769FF1E9BEF
:10D6B00040F66C52C2F20002D05C1D9D0543D55469
:10D6C000FCF7DFB91D9BF92B08D942F6EC54C2F2E6
:10D6D00000044FF01202227100F068BF42F61C668F
:10D6E000C2F200061E99F154FCF7CBB942F61C6752
:10D6F000C2F200071D9887F8FB00FCF7C2B943F29D
:10D700001823C2F20003196841B942F6EC50C2F284
:10D7100000004FF00102027100F048BF4E681D98F2
:10D720001E994FF001020DF16A03B0478DF86B00AE
:10D730009DF86A20D2F1010138BF0021219B83F8B6
:10D74000501000283CF49DA942F6EC54C2F20004AB
:10D75000207100F02BBF43F21821C2F200010B68C8
:10D7600043B942F6EC50C2F200004FF001010171E2
:10D7700000F01CBF1A681D981E9990478DF86B0029
:10D7800000283CF47EA942F6EC54C2F20004207159
:10D7900000F00CBF43F21823C2F200031A6842B92A
:10D7A00042F6EC50C2F200004FF00101017100F0AE
:10D7B000FDBE56681D981E994FF000020DF16A03D8
:10D7C000B0478DF86B009DF86A10D1F1010238BFA7
:10D7D0000022219B83F8502000283CF452A942F6F5
:10D7E000EC54C2F20004207100F0E0BE0A981E99C9
:10D7F000FAF7BCF80A9040B942F6EC53C2F20003C3
:10D800004FF01700187100F0D1BE0A9A13689B6A96
:10D8100043B942F6EC51C2F200014FF015020A7111
:10D8200000F0C4BE0A9880689DF8741042F61C622D
:10D83000C2F2000298478DF86B0000283CF421A941
:10D8400042F6EC54C2F20004207100F0AFBE0A9818
:10D850001E99FAF78BF80A9040B942F6EC53C2F2DF
:10D8600000034FF01700187100F0A0BE0A990A6873
:10D87000536943B942F6EC51C2F200014FF0150270
:10D880000A7100F093BE0A9880689DF8741042F601
:10D890001C62C2F2000298478DF86B0000283CF42D
:10D8A000F0A842F6EC54C2F20004207100F07EBEF3
:10D8B0000A981E99FAF75AF80A9040B942F6EC51C4
:10D8C000C2F200014FF017020A7100F06FBE0A9E0B
:10D8D00031688E6946B942F6EC53C2F200034FF04C
:10D8E0001500187100F062BE0A9A90689DF87410D5
:10D8F00042F61C62C2F200020DF16A03B0478DF8D5
:10D900006B0000283CF4BDA842F6EC54C2F20004BF
:10D91000207100F04BBE0A981E99FAF727F80A907A
:10D920001D997F2909D1051C18BF012542F61C67E6
:10D93000C2F200073D70FCF7A4B80A9B43B942F657
:10D94000EC53C2F200034FF01700187100F02EBE26
:10D950000A980268536843B942F6EC51C2F20001DA
:10D960004FF015020A7100F021BE0A988068C9B212
:10D9700042F61C62C2F2000298478DF86B00002844
:10D980003CF47FA842F6EC54C2F20004207100F08F
:10D990000DBE0A981E99F9F7E9FF0A9040B942F6C0
:10D9A000EC53C2F200034FF01701197100F0FEBDF5
:10D9B0000A990A68976847B942F6EC50C2F200002B
:10D9C0004FF01502027100F0F1BD42F61C66C2F282
:10D9D00000060A9B98689DF8741032780DF16A036E
:10D9E000B8478DF86B009DF86A10317000283CF440
:10D9F00048A842F6EC54C2F20004207100F0D6BDF3
:10DA00000A981E99F9F7B2FF0A9040B942F6EC5312
:10DA1000C2F200034FF017021A7100F0C7BD0A9F4F
:10DA20003868C76847B942F6EC51C2F200014FF0BE
:10DA30001500087100F0BABD42F61C66C2F200067D
:10DA40000A9A90689DF8741032460DF16A03B8473F
:10DA50008DF86B009DF86A30337000283CF411A8F3
:10DA600042F6EC54C2F20004207100F09FBD0A9807
:10DA70001E99F9F77BFF0A9040B942F6EC51C2F2C9
:10DA800000014FF017030B7100F090BD0A9F396839
:10DA90000F6947B942F6EC50C2F200004FF0150290
:10DAA000027100F083BD0A9ED6F808809DF874903C
:10DAB00042F61C66C2F200063068F9F79BFB02468C
:10DAC000404649460DF16A03B8478DF86B009DF852
:10DAD0006A30337000283BF4D4AF42F6EC54C2F203
:10DAE0000004207100F062BD0A984FF00001F9F7C0
:10DAF0003DFF0A9040B942F6EC53C2F200034FF0EA
:10DB00001701197100F052BD0A980268D36A43B92F
:10DB100042F6EC50C2F200004FF01502027100F024
:10DB200045BD0A9988689DF8741098478DF86B0078
:10DB300000283BF4A6AF42F6EC54C2F20004207178
:10DB400000F034BD0A981E99F9F710FF0A9040B909
:10DB500042F6EC53C2F200034FF01701197100F0C6
:10DB600025BD0A980268D36943B942F6EC50C2F267
:10DB700000004FF01502027100F018BD0A99886884
:10DB80009DF8741042F61C62C2F2000298478DF8AC
:10DB90006B0000283BF475AF42F6EC54C2F200046F
:10DBA000207100F003BD0A981E99F9F7DFFE0A9074
:10DBB00040B942F6EC53C2F200034FF0170119715D
:10DBC00000F0F4BC0A980268136A43B942F6EC50BC
:10DBD000C2F200004FF01502027100F0E7BC0A9992
:10DBE00088689DF8741042F61C62C2F200029847E1
:10DBF0008DF86B0000283BF444AF42F6EC54C2F2BF
:10DC00000004207100F0D2BC0A981E99F9F7AEFE0C
:10DC10000A9040B942F6EC50C2F200004FF01702F1
:10DC2000027100F0C3BC0A980268536A43B942F615
:10DC3000EC53C2F200034FF01501197100F0B6BCAD
:10DC40000A9988689DF8741010AA98478DF86B009F
:10DC50001098F9F7A5FA42F61C62C2F200021060B1
:10DC60009DF86B0000283BF40CAF42F6EC54C2F276
:10DC70000004207100F09ABC0A984FF00001F9F7F7
:10DC800075FE0A9040B942F6EC53C2F200034FF021
:10DC90001700187100F08ABC0A9B19680B6B43B916
:10DCA00042F6EC51C2F200014FF015020A7100F089
:10DCB0007DBC0A9880689DF8741042F61C62C2F21E
:10DCC000000298478DF86B0000283BF4DAAE42F66C
:10DCD000EC54C2F20004207100F068BC1D990729C1
:10DCE00008D942F6EC54C2F200044FF00803237145
:10DCF00000F05CBC41F2FC75C2F2000555F83170D1
:10DD0000002F7BF4BEAEF7F719FF002808BF0120F3
:10DD100041F2FC76C2F200061D9A46F83200FBF78B
:10DD2000B0BE1D98072808D942F6EC54C2F2000490
:10DD30004FF00800207100F039BC41F2FC71C2F2D2
:10DD4000000151F83050002D3BF49BAEF7F7F6FE82
:10DD50001D9F41F2FC76C2F2000656F83720831A66
:10DD60001C9306EBC70041688B428CBF0021C3EBBC
:10DD700001011B9141F2FC75C2F2000505EBC706DB
:10DD80001B9A72604FF0000345F83730FBF779BEFD
:10DD90001D9EFA2E08D942F6EC51C2F200014FF056
:10DDA00013020A7100F002BC0DF1700CF9F7C0FB10
:10DDB00040F66C57C2F20007B855FBF762BE0DF192
:10DDC000700CF9F7DDFB0DF1700CF9F7B1FB1C904D
:10DDD00050B11E9D40F66C52C2F20002565D1D9974
:10DDE00031435155FBF74DBE1E9D40F66C56C2F2B5
:10DDF0000006735D1D9823EA00077755FBF741BEC7
:10DE00001D9B1E9AD018C1B242F61C60C2F20000DF
:10DE100080F8FB10FA2907D942F6EC54C2F200044C
:10DE20004FF012032371C1E342F61C77C2F20007E0
:10DE30003D6842F61C66C2F20006F0184AF600037E
:10DE4000C0F60103E91806F0CBFC3A681E99501899
:10DE50003860FBF716BE1D9AF82A07D942F6EC5433
:10DE6000C2F200044FF0130020719FE3F7F766FE43
:10DE700000F104004CF6CD47CCF6CC47A7FB0015CB
:10DE80004FEA95062199486AB6FBF0F31C931D9A58
:10DE900040F66C57C2F200074FEA1345BD54BE1856
:10DEA0004FEA13217170B370FBF7EBBD1D9BF82B8C
:10DEB00007D942F6EC54C2F200044FF0130121716D
:10DEC00074E3F7F73BFE00F104004CF6CD42CCF6CC
:10DED000CC42A2FB00274FEA9705219E716AB5FB51
:10DEE000F1F01D9B40F66C57C2F20007FA18557806
:10DEF000FE5C4FEA064141EA0527937847EA0302B0
:10DF00001B92801A20F07F451C950DF1700C1E9815
:10DF100085422CBF00200120F9F7F2FAFBF7B1BDD2
:10DF2000219E96F846700DF1700CF9F701FB3A1A34
:10DF30001C92219B83F84720FF2A94BF00220122D4
:10DF400083F85020FBF79DBD1D9BF92B07D942F6A6
:10DF5000EC53C2F200034FF01300187126E342F6AF
:10DF60001C70C2F20000026840F66C51C2F200015F
:10DF70004FEA1220C854CB185A70FFF770B8219D91
:10DF800095F847201C9295F8466085F8476085F81B
:10DF90004620FBF776BD1D98072807D942F6EC54BA
:10DFA000C2F200044FF008012171FFE2F9F70CFF03
:10DFB0000DF1A80C4CF8380D003018BF0120F9F70E
:10DFC0009FFAFBF75EBD219F97F8470097F8463010
:10DFD0000DF1700C984214BF00200120F9F790FA5F
:10DFE000FBF74FBD219D95F8470095F846200DF1B0
:10DFF000700C801A18BF0120F9F782FAFBF741BDB7
:10E00000219E96F8470096F846100DF1700C884254
:10E010002CBF00200120F9F773FAFBF732BD219FD6
:10E0200097F8470097F846300DF1700C984294BF6E
:10E0300000200120F9F764FAFBF723BD219D95F834
:10E04000470095F846200DF1700C90428CBF0020DF
:10E050000120F9F755FAFBF714BD219E96F8470009
:10E0600096F846100DF1700C884234BF0020012054
:10E07000F9F746FAFBF705BD1D98F62807D942F6D1
:10E08000EC54C2F200044FF0120222718EE242F60A
:10E090001C67C2F200073858F9F7ACF8219BD86426
:10E0A000FBF7EFBC1D99F62907D942F6EC50C2F2F6
:10E0B00000004FF01203037178E242F61C65C2F2D1
:10E0C00000056858F9F796F8219EB064FBF7D9BCB3
:10E0D00042F61C62C2F2000292F8FB201D9BD1188E
:10E0E000FB2907D942F6EC53C2F200034FF01201AC
:10E0F00019715BE21E99C2F1FB00814207DD42F615
:10E10000EC54C2F200044FF0130222714EE240F6CA
:10E110006C57C2F20007781842F61C65C2F200057F
:10E12000E91806F05DFBFBF7ACBC2198466B326842
:10E1300056683EB942F6EC53C2F200034FF01E019E
:10E14000197133E21E9A42F61C63C2F2000393F87F
:10E15000FB309918FB2907D942F6EC50C2F20000B7
:10E160004FF01202027121E200F134001D9942F6D3
:10E170001C67C2F20007BA18B0478DF86B00002880
:10E180003BF47FAC42F6EC54C2F2000420710DE285
:10E1900042F6EC54C2F200044FF00100207105E297
:10E1A0000DF1700CF9F7ECF940F66C57C2F200076C
:10E1B0001E9D7E5D1D9A16423BF463AC42F61C73B5
:10E1C000C2F200030999196070E10DF1700CF9F7C2
:10E1D000D7F940F66C50C2F200001E9FC55D1D9E2F
:10E1E00035427BF44EAC42F61C74C2F20004099A2C
:10E1F00022605BE19DF874000DF16B01FAF716FCEB
:10E200008DF86A009DF86B302BB142F6EC54C2F2E7
:10E2100000042371CAE100283BF433AC42F61C70C1
:10E22000C2F200000999016040E19DF874000DF10F
:10E230006B01FAF7FBFBD0F1010238BF00228DF829
:10E240006A209DF86B1029B142F6EC52C2F200022E
:10E250001171ABE1219FFD6A15B98DF86A5002E09A
:10E260009DF86A6066B90DF1700C1E98F9F700FE12
:10E2700030B942F61C74C2F200040998206015E11E
:10E280000DF1700C9DF86A00F9F73AF94FF00002B1
:10E29000219BDA62FBF7F5BB9DF874000DF16B0171
:10E2A000FAF7C4FB8DF86A009DF86B302BB142F68B
:10E2B000EC50C2F20000037178E100287BF4E1AB7E
:10E2C00042F61C77C2F20007099D3D60EEE09DF822
:10E2D00074000DF16B01FAF7D9FB8DF86A009DF817
:10E2E0006B1029B142F6EC52C2F2000211715DE1ED
:10E2F00000287BF4C6AB42F61C76C2F20006099CED
:10E300003460D3E09DF874000DF16B01FAF7BEFBA9
:10E31000031C18BF01238DF86A3092E79DF8740042
:10E320000DF16B01FAF782FB003018BF01208DF868
:10E330006A0086E71D9EF62E07D942F6EC53C2F21C
:10E3400000034FF012041C7130E12199C86CF8F7FA
:10E3500027FF42F61C67C2F20007B851FBF791BBDA
:10E360000DF1700CF9F7E4F8219D95F84760D6F1AE
:10E37000010238BF0022002814BF104682F00100BD
:10E3800085F84700FBF77DBB0DF1700CF9F7D0F86D
:10E39000219991F84770784081F84700FBF771BBED
:10E3A0000DF1700CF9F7C4F8219B83F85100FBF7CD
:10E3B00068BB04F0A7FF0DF1A80C4CF8380DFF283E
:10E3C00028BFFF20C0B2F9F79BF8FBF75ABB04F057
:10E3D0008FFF0DF1A80C4CF8380DFF2828BFFF2047
:10E3E000C0B2F9F78DF8FBF74CBB04F095FF0DF1C7
:10E3F000A80C4CF8380DFF2828BFFF20C0B2F9F751
:10E400007FF8FBF73EBB04F069FF0DF1700C0028AC
:10E410000CBFFF200020F9F773F8FBF732BB42F680
:10E420001872C2F2000210681D99401804F0B8FA80
:10E430008DF86B0000283BF424AB42F6EC54C2F29A
:10E4400000042071B2E01D9804F068FAFBF719BBD4
:10E450000DF1700CF9F76CF804F05AFAFBF711BBE8
:10E4600042F61875C2F200052E681D9FF01904F0DF
:10E4700071FAFBF706BB04F055FAFBF702BB41F259
:10E48000F873C2F200031A6882B941F63C00C2F286
:10E490000000017801F00204E3B23BB142F6EC5413
:10E4A000C2F200044FF0350323717FE041F63C05D2
:10E4B000C2F200052E7816F0010F7BF4E0AA219F2E
:10E4C0002FB142F61C72C2F200021068786042F668
:10E4D000A051C2F200010C683F2C00F2948004F1BC
:10E4E00001041B941C9414B94FF001051B9541F6CF
:10E4F0004806C2F200064FF0540541F63C04C2F251
:10E50000000441F2F877C2F200071C9B05FB03628E
:10E5100021929BB9217801F00400C1B209B9386891
:10E5200040B9217841F001006FF3820020705068FB
:10E5300040B115E04FF001021C92E6E7506878B94F
:10E54000402B02D003F1010301E04FF000031C93C4
:10E550001B9A9342D9D14FF00000F9F7C9FFD4E7D5
:10E5600042F6A056C2F20006336042F61C75C2F2B3
:10E57000000528604FF0000A5446FBF782BA219F3D
:10E58000396A41F000403863FBF77BBA4FF0000670
:10E59000219D2E63FBF775BAFBF773BA0C9D42F60B
:10E5A000EC54C2F200044FF00102227142F6EC502A
:10E5B000C2F20000099C04604571F3F789F9F3F792
:10E5C00087F9219D2A6A7AB14FF000031C932199A3
:10E5D000086A48B1F3F77CF91C9C04F101041C940F
:10E5E000219D2A6AA242F5D84FF00000F9F780FF7A
:10E5F000FBF77BB94FF0000700F1FF344FF0000349
:10E600005E46FDF718BD4FF000031C936CE74FF01A
:10E6100002031C9341F64802C2F20002FDF754BF08
:10E620002BB0BDEC0A8BBDE8F08F05F10103D2F8E9
:10E630000061002E3DF44CAF05F1020302F1A80287
:10E64000412B7DF441AFFDF798BFBEF1000F3DF4C3
:10E650008CAC10F8039001F8039003F1010393428E
:10E660007DF483ACFDF78FBCF9180EEB030C13F8A7
:10E67000016F02F1FF35B0423DF456AA2A46FDF77C
:10E6800062BA05F1FF32FDF75EBA00BF38B5054644
:10E6900041F64004C2F200042068F6F781FE4FF014
:10E6A000000323608DB148F69850C0F601004FF08A
:10E6B000070149F67D02C0F60002F6F787FD42F633
:10E6C0009C52C2F20002106038BD42F69C54C2F265
:10E6D00000042068F6F764FE4FF000002060F6F7B3
:10E6E0003BF8FBF74DF804F089F942F6B051C2F25D
:10E6F00000010878FF2803D04FF00401FAF7BAFFB1
:10E7000038BD00BF70B542F6F450C2F2000048F6C2
:10E71000A851C0F60101F6F789F942F6B053C2F2EA
:10E7200000034FF0FF021A7040F6AC64C2F200041E
:10E730004FF0040684F820624FF00005C4F81C5224
:10E740002846F6F75DFB206084F86464C4F86054E2
:10E750004FF00100F6F754FBC4F8440284F8A866B1
:10E76000C4F8A4564FF00200F6F74AFBC4F8880438
:10E7700084F8EC68C4F8E8584FF00300F6F740FB63
:10E78000C4F8CC0641F2C070C2F2000048F6B451A1
:10E79000C0F60101F6F74AF942F6B450C2F20000A1
:10E7A00048F6EC21C0F601012A462B46FAF732F969
:10E7B000F8F7FAFF4FF00100FFF768FF70BD00BFE8
:10E7C0002DE9F04F2DED028B8FB04FF0000842F68F
:10E7D0009C57C2F2000741F64003C2F200030393C4
:10E7E00042F6B05BC2F2000B40F6AC66C2F2000625
:10E7F0009FEDB98B39684FF0FF3041B9F3F768F8F6
:10E80000386800280CBFFA204FF0FF30FFE7F6F71A
:10E810001BFD28B1B8F1320F09D808F1010806E054
:10E82000B8F1330F0CBF4FF034084FF000083A68CE
:10E83000D2B9F3F74DF8B8F1320F0ED1039C20682E
:10E84000F6F7AEFD4FF00005039B1D60F5F784FF62
:10E850004FF00200F9F78AFD06E0B8F1340F03D15A
:10E860004FF00100F9F782FD9BF800104FF4117092
:10E8700000FB0162D2F81842002CBBD04FF4117596
:10E8800005FB01F303F5887406EB0409315DE0290B
:10E890000CD199F801000E2808D14FF6FF704946B7
:10E8A000D9F80021F8F716FC10B36BE2325D02F0E4
:10E8B0001F0509EB05035A78294605F0010019F8F0
:10E8C0000550521B01F1FF33002940F078820BE024
:10E8D00019F80300151A03F1FF3119F80120AA1ADB
:10E8E00001F1FF330029F3D112F0FF0F40F04A820B
:10E8F000335D4FEA5310072800F23C82DFE810F046
:10E9000008003A023A023500A6003A028A002601BF
:10E91000335D09F1010513F01F0000F0338209F1A6
:10E92000020905F1020500F1FF3255FA82F4029462
:10E930004FF000054FF0010A15E019F8011CE8B28C
:10E9400021405246FAF776F9002840F01B8205F183
:10E9500001054FEA4404FF2CEFD909F1010902999E
:10E96000894500F00F825446E7E799F8014038687E
:10E9700070B1F6F715FD4FF000003860F5F7ECFECA
:10E98000FAF7FEFE4FF00100F9F7F0FCF2F7A0FFF6
:10E9900003990B686BB948F6BC50C0F601004FF004
:10E9A000070149F22102C0F60002F6F70FFC039DB1
:10E9B000286005A84FF00001F9F706FF7CB9F7F7CA
:10E9C000BDF8C1B201F1FF33DDB2FD2D42F6B25008
:10E9D000C2F2000092BF01700122027009E042F60B
:10E9E000B250C2F20000027802FB04F404EB1424DB
:10E9F000047042F6B254C2F2000421780EAB03F860
:10EA0000241D4FF003004FF000014FF01602F9F7FC
:10EA1000D1FCEFE60DF11300F9F7C8F801469DF8B7
:10EA200013508DF81450012D06D828B10DF11500A2
:10EA30004FF00D0205F0D4FE4FF006004FF000013C
:10EA40004FF00E0205ABF9F7B5FCD3E69BF80010CA
:10EA50004FF4117303FB01F499F80100032872D8F5
:10EA6000DFE800F002263E504FF00100FFF70EFEF7
:10EA70004FF000050EAB03F8255D4FF0040029466A
:10EA80004FF00102F9F796FC4FF0C800F8F70AFBC7
:10EA900032599BF800004FF0010400940195D2F820
:10EAA0000CC04FF416512A464FF00803E04766E1C8
:10EAB0004FF0000142F6EC53C2F2000319714FF01F
:10EAC00001040EAB03F8254D4FF004002246F9F780
:10EAD00071FC54E1AFF300800000000000E06F40E3
:10EAE000F9F71AFD0EAB4FF0020103F8251D4FF0A8
:10EAF00004004FF000014FF00102F9F75BFC4FF00A
:10EB000001043CE10EAB4FF0120203F8252D4FF04B
:10EB100004004FF000014FF00102F9F74BFC4FF0F9
:10EB2000C800F8F7BFFA35599BF800004FF0010410
:10EB300000944FF000020192ED684FF416414FF03F
:10EB40000803A8471BE14FF0000418E199F80150B1
:10EB5000A5F102050C2D00F21081DFE815F00D0083
:10EB600067007E000E010E010E010E010E010E0166
:10EB70000E010E010E019D00315DC1F30403DAB2F6
:10EB8000012A00F0FF8009F1050509F1080403EBF3
:10EB9000C30003EB400101EBC10303F15403DAB2FC
:10EBA00002EB42002418C5EB040CACF1030E0EF08E
:10EBB000010A99F8029015F8010C04F0B7FB53EC28
:10EBC000182B04F0C5FE04F08BFC01464846FAF70A
:10EBD00097F805F10305A54240F0D780D2E015F87B
:10EBE000039C15F8010C04F0A1FB53EC182B04F066
:10EBF000AFFE04F075FC01464846FAF781F805F1CE
:10EC0000030515F803AC15F8010C04F08FFB53EC69
:10EC1000182B04F09DFE04F063FC01465046FAF701
:10EC20006FF805F10305A542D9D1ABE099F80230A0
:10EC3000305DC0F30405A5F10305EAB209F1030153
:10EC40009C18FF2CC4BF5A42D2B240F66C50C2F29C
:10EC50000000C01805F0C4FD94E099F8023099F85E
:10EC600003500EAC04F8243D0DF1150040F66C5134
:10EC7000C2F20001C918202D34BF2A46202205F017
:10EC8000AFFD05F101024FF007004FF00301D2B2D2
:10EC90002346F9F78FFBADE599F80240C4B999F81E
:10ECA0000310A9B903F0AAFE039A1068F6F778FBDF
:10ECB0004FF0000303980360F5F74EFD48F6CC5083
:10ECC000C0F6010007F07CFBF9F706FD002848D0EC
:10ECD00099F8025099F8034048F6DC50C0F601005C
:10ECE00044EA052107F06CFB99F803A0494611F8A6
:10ECF000022F4AF60003C0F6010303EB022540F69B
:10ED00006C54C2F2000404EB0A0001F102014FF05E
:10ED1000800205F065FD4FF68071CFF6FF71CAEBFA
:10ED20000100C2B2A018A9184FF0800205F058FDEA
:10ED3000204629464FF48072F3F7C4FBA0B9204661
:10ED400029464FF4807205F0F5F880B94FF00100C4
:10ED50004FF000010A460B46F9F72CFB4FF0010477
:10ED60000DE04FF000040AE04FF0000407E04FF020
:10ED7000000404E04FF0000401E04FF00004002C18
:10ED80007FF438ADF8F7F4FE34E5BAF1000F3FF444
:10ED900026AF15F803AC15F8010C04F0C7FA53ECD4
:10EDA000182B04F0D5FD04F09BFB01465046F9F703
:10EDB000A7FF05F10305A5427FF411AFE2E70028A4
:10EDC0003FF486AD19F80310521A03F1FF33B3F183
:10EDD000FF3F7FF47DAD87E5704700BF42F62773A4
:10EDE000C2F200031A78027042F62670C2F20000E6
:10EDF00003780B70704700BF42F62773C2F200031E
:10EE00001B78834225D842F62672C2F2000212789D
:10EE10009A18904220DAC01A4FEA50034FF00102CC
:10EE200002FA03F310F0010F09D042F63070C2F27B
:10EE30000000026813400B704FF00100704742F66B
:10EE40002870C2F20000026813400B704FF00100FE
:10EE500070474FF0000070474FF00000704700BF50
:10EE600010B542F62773C2F200031B7883427AD8AA
:10EE700042F62672C2F2000212789A18904275DAAF
:10EE8000C31A03F0FE0442F63470C2F200000278A6
:10EE9000A418E4B24FEA53024FF0010000FA02F264
:10EEA00013F0010F12D041B142F63070C2F20000EF
:10EEB000016842EA010303601AE042F63070C2F2D0
:10EEC0000000036823EA0203036011E041B142F647
:10EED0002870C2F20000036842EA0301016007E003
:10EEE00042F62873C2F20003196821EA0201196090
:10EEF00042F62870C2F2000001680A4224D042F6AD
:10EF00003073C2F20003186802420ED020464FF060
:10EF10000001F2F779F904F10102D0B24FF00101DA
:10EF2000F2F772F94FF0010010BD20464FF00101D9
:10EF3000F2F76AF904F10101C8B24FF00001F2F7EB
:10EF400063F94FF0010010BD20464FF00001F2F7C9
:10EF50005BF904F10102D0B24FF00001F2F754F96D
:10EF60004FF0010010BD4FF0000010BD4FF0000049
:10EF700010BD00BF08B542F63473C2F2000318702A
:10EF800042F62C73C2F20003197042F62773C2F2E4
:10EF900000031A70091A01F10101C8B242F6267283
:10EFA000C2F200021070412801D9F1F747FB40F28C
:10EFB000C010C2F200004FF00101F9F7A7FC08BD34
:10EFC0002DE9F84342F63573C2F2000318784FEA90
:10EFD000400111F0FF0405D042F63572C2F2000282
:10EFE000147006E042F63575C2F200054FF00106D6
:10EFF0002E7042F65877C2F20007387842F6357321
:10F00000C2F20003197808420CBF4FF000094FF01C
:10F0100001094FF000052C464FF0010742F6387603
:10F02000C2F20006A84604F01F0207FA02F0AB592C
:10F03000184204D0204649464246F9F7FBFD04F148
:10F040000104E4B214F01F0FEDD105F10405202DE9
:10F05000E9D1BDE8F88300BF42F65873C2F200035D
:10F06000187042F63570C2F200004FF001020270D3
:10F07000704700BF00B583B042F63870C2F200009E
:10F080004FF000014FF00802F1F73AFB4FF0000398
:10F0900000934FF00100019042F65C70C2F2000054
:10F0A0004FF47A714FF006024EF6C173C0F60003BA
:10F0B000F6F70EFD03B000BD08B542F65C70C2F273
:10F0C0000000F6F75FFC4FF0CC00FFF7C5FF08BD6E
:10F0D00089B14FEA501242F63873C2F2000300F0D1
:10F0E0001F004FF0010101FA00F053F8221008430D
:10F0F00043F8220011E04FEA501242F63873C2F290
:10F10000000300F01F004FF0010101FA00F053F876
:10F11000221021EA000143F822104FF0000070474E
:10F1200008B54FF4404048F63461C0F6010142F69C
:10F130008072C2F20002F9F7A7FB08BD10B584B0D7
:10F14000144649BB0DF10D0300930DF10E00019023
:10F150004FF0000001460DF10A020DF10B03F5F727
:10F16000A7F94FF000018DF80C109DF80B201AB193
:10F170004FF001038DF80C309DF80A0028B19DF87E
:10F180000C1041F002028DF80C204FF000008DF8B9
:10F190000F00039B236001E04FF0140004B010BD8A
:10F1A00070B514468AB199B94FF000000146024685
:10F1B000F5F7F6F906462578F5F7D6FA85420AD22C
:10F1C000735D23704FF0000070BD4FF0160070BDEE
:10F1D0004FF0140070BD4FF0160070BD70B51546AD
:10F1E00091B992F8FB3093B14FF000042646285DA8
:10F1F0003146F5F7CFF804F1010495F8FB00A04281
:10F20000F5D84FF0000070BD4FF0140070BD4FF006
:10F21000000070BD10B586B0F1B942F68C73C2F231
:10F220000003197842F68D70C2F20000037802AC38
:10F2300000944FF01000019010461A464FF0010361
:10F24000FAF776F848F63060C0F60100214607F07C
:10F25000B7F84FF0000001E04FF0140006B010BD09
:10F260002DE9F0411546042975D8DFE801F0030BBC
:10F27000741B640068782978F5F782F94FF0000074
:10F28000BDE8F0812A7842F68C73C2F200031A704E
:10F29000687842F68D71C2F2000108704FF00000EC
:10F2A000BDE8F0812C786D7805F1040546F26763BE
:10F2B000C6F2666383FB05204FEA600101EB810221
:10F2C00012F0FF054BD04FF00007A5F1050808F03C
:10F2D0000108042C94BF2646052630463946F5F72A
:10F2E00059F8A41BE4B2A5F1050515F0FF053ED1C0
:10F2F0001DE0042C94BF2646052630463946F5F716
:10F3000049F8A01BA5F1050505F0FF0500F0FF0475
:10F31000042C94BF2646052630463946F5F73AF8C0
:10F32000A11BCCB2A5F1050515F0FF05E1D14FF009
:10F330000000BDE8F0812C78F5F716FA844212D26D
:10F34000204605F101014FF00102F5F745F94FF0B4
:10F350000000BDE8F0814FF01400BDE8F0814FF0EF
:10F360000000BDE8F0814FF01600BDE8F0814FFAD3
:10F3700088F6002EBDD0042C94BF264605263046C4
:10F380003946F5F707F8A31BDCB2A5F1050515F022
:10F39000FF05AED1CBE700BF08B505293ED8DFE8B1
:10F3A00001F0030B151F29331046F5F7B1F80028BB
:10F3B0000CBF1620002008BD48F69450C0F601008E
:10F3C000114606F0FDFF4FF0000008BD48F68C50D6
:10F3D000C0F60100114606F0F3FF4FF0000008BD33
:10F3E00048F68850C0F60100114606F0E9FF4FF0DC
:10F3F000000008BD48F68050C0F60100114606F036
:10F40000DFFF4FF0000008BD48F67850C0F601005D
:10F41000114606F0D5FF4FF0000008BD4FF0140074
:10F4200008BD00BF08B5012805D0022814BF00227E
:10F430000122114603E04FF000024FF001014FF0AE
:10F440000100F5F76FF908BD08B501F1FF31032997
:10F4500021D8DFE801F0020B121948F6F040C0F69F
:10F46000010006F0ADFF4FF0000008BD4FF00000B6
:10F47000FFF7D8FF4FF0000008BD4FF00100FFF785
:10F48000D1FF4FF0000008BD4FF00200FFF7CAFFA8
:10F490004FF0000008BD4FF0140008BD08B5F5F7A7
:10F4A0005BF94FF001004FF000010A46F5F73AF919
:10F4B000F5F75EF94FF00C004FF00001F4F76AFF2A
:10F4C000F5F74AF908BD00BF037B13B9437B13B9B5
:10F4D0000EE0994208D301F1FF318A18437B9A422A
:10F4E0008CBF0020012001E04FF00000C0B2704747
:10F4F0004FF00100704700BF70B4447A24B14FF060
:10F50000320606FB04F610E0C57848F6E854C0F66B
:10F51000010454F82550B5F5964F9DBF49F2646635
:10F52000B6FBF5F606EB86060826847A24B14FF082
:10F53000320505FB04F501E041F28835C07A18B1C7
:10F54000FF2808BF012001E04FF0010001B10E606B
:10F5500002B1156003B1186070BC704740F6AC632F
:10F56000C2F200034FF4117202FB00304FF00001B1
:10F57000C0F810124FF6FF73C0F82C32C0F8181202
:10F58000704700BFF8B505460E4640F6AC64C2F2BF
:10F5900000044FF4117303FB0044D4F8240200EB81
:10F5A0005007F6F7CBFAD4F82812421A974202D93C
:10F5B000B81AF5F749FE23689A6928464FF0010109
:10F5C000904740F6AC60C2F200004FF4117101FBAD
:10F5D00005014FF6FF7001F104013246F7F77AFD9D
:10F5E000A31918714FEA10225A7106F10206C4F8E5
:10F5F00004614FF00000C4F8080121680B6A284636
:10F600009847F5F759FC2846FFF7A8FFF8BD00BF5B
:10F6100038B504460D460368F92B08D840F66C50FF
:10F62000C2F20000185A03F1020323603DE0A3F583
:10F630007A72FA2A0AD840F66C51C2F200018A5C4A
:10F640004FEA022003F1010323602EE0A3F5FA60E4
:10F65000262811D84FF0000001460246F4F7A0FF1B
:10F660002368A3F5FA6281184978805C40EA01209A
:10F6700003F10203236018E0A3F6B8317C290DD80A
:10F6800003F10042A2F6B83040F66C51C2F200011C
:10F6900031F8100003F10103236006E055B14FF08B
:10F6A00001032B704FF0000038BD2DB14FF0000367
:10F6B0002B7038BD4FF0000038BD00BF30B583B0AF
:10F6C00004460D4602A840F8084D68460DF10701B2
:10F6D000FFF79EFF9DF8073083B904F1FF346519E9
:10F6E00002A941F8085D68460DF10701FFF790FF98
:10F6F0009DF80720101C18BF012001E04FF0010009
:10F7000003B030BD2DE9F0410D4617461E4640F6C8
:10F71000AC61C2F200014FF4117404FB0010D0F888
:10F720003002037BFF2B02D1427BFF2A56D02C688C
:10F73000F92C15D821464FF00202FFF7C5FE00282C
:10F7400050D0002E52D140F66C50C2F20000275229
:10F750002B6803F102032B604FF00100BDE8F0813C
:10F76000A4F57A78B8F1FA0F18D841464FF00102A3
:10F77000FFF7AAFE00283DD0002E3FD14FEA172701
:10F7800040F66C52C2F2000202F80870296801F1DA
:10F79000010129604FF00100BDE8F081A4F6B83105
:10F7A0007C292FD804F10044A4F6B8344FEA440170
:10F7B0004FF00202FFF788FE002827D0002E29D143
:10F7C00040F66C50C2F2000020F814702B6803F170
:10F7D00001032B604FF00100BDE8F0814FF0000005
:10F7E000BDE8F0814FF00000BDE8F0814FF001006E
:10F7F000BDE8F0814FF00000BDE8F0814FF001005E
:10F80000BDE8F0814FF00000BDE8F0814FF000004E
:10F81000BDE8F0814FF00100BDE8F08130B583B064
:10F8200040F6AC64C2F200044FF4117505FB0040D1
:10F83000D0F83002B1F57A7F1BD3A1F57A7163B1AC
:10F84000837B13B9C37B13B907E0994223D38A188A
:10F8500002F1FF32C07B824220D8C8B20DF107010D
:10F86000F9F77CF99DF80710D1F1010038BF0020AD
:10F8700019E04FEAD10402F107024FEAD20523B1A1
:10F8800021462A46FFF720FE58B12819FA288CBFD6
:10F890000020012007E04FF0000004E04FF00000DE
:10F8A00001E04FF0000003B030BD00BF08B5B0F577
:10F8B0007A7F21D279B14FEAD00340F66C52C2F27E
:10F8C000000200F007004FF0010101FA00F0D15CE6
:10F8D0000843D05408BD4FEAD00340F66C52C2F240
:10F8E000000200F007004FF0010101FA00F0D15CC6
:10F8F00021EA0000D05408BD00F11800C0B24FF05A
:10F900000102F9F797F908BD10B540F6AC64C2F2F0
:10F9100000044FF4117303FB0044D4F81C02F5F704
:10F920003FFD4FF00000C4F81C0210BD38B54FF485
:10F93000117101FB00F140F6AC62C2F200028C18BA
:10F94000D4F80831D4F80451AB420BD08958E318ED
:10F950008A6A1979904728B1D4F8080100F10100AA
:10F96000C4F8080138BD00BF08B540F6AC63C2F268
:10F9700000034FF4117202FB0031D1F8082101F1AC
:10F980000401D1F800319A420BD140F6AC61C2F2C9
:10F9900000014FF4117202FB0010D0F81C02F5F7C1
:10F9A000BDFA08BD70B582B005468DF8071040F667
:10F9B000AC64C2F200044FF4117303FB0044D4F8AA
:10F9C0001802002850D11AB12846FFF7C7FD4BE0B6
:10F9D000F6F7B4F8D4F82812431AC4F82802D4F879
:10F9E0001002D4F82422934204D800F10103B3F5A5
:10F9F000807F04D12846FFF7B1FD4FF00103D4F812
:10FA00001012621802A911F8010D82F81001C4F851
:10FA10001032B4F82C024FF00102F7F75BFBC4F888
:10FA20002C0208BB04F5887694F82032012B03D110
:10FA3000304601F0F3FA38B994F82012022913D1B4
:10FA4000304600F013F978B14FF00102C4F81822E3
:10FA500040F6AC60C2F200004FF4117303FB0505E1
:10FA6000D5F81C02F5F75AFA02B070BD10B542F68F
:10FA70008F73C2F200031B78032B47D840F6AC62A9
:10FA8000C2F200024FF4117101FB032340F2207215
:10FA9000C2F2000252E8001F01F1010142E8001425
:10FAA000012CF7D018B14FF00100C3F83C0242F628
:10FAB0008E74C2F200044FF001012170D3F840228D
:10FAC0001AB1D3F81C02F5F729FA40F22073C2F2FA
:10FAD000000353E8002FA2F1010243E80024012CA7
:10FAE000F7D053E8002FB2F1004F0DD14FF00002D4
:10FAF00043E80024012CF4D04EF60450CEF200006E
:10FB0000016841F080510160BFF32F8F10BD00BF2D
:10FB100010B542F68F73C2F200034FF004041C705C
:10FB2000FFF7F2FE10BD00BF2DE9F04F89B005468A
:10FB30000E4691F8029009EB490947F69048C0F645
:10FB4000010809EB08074FF4117B0BFB00FB40F6A3
:10FB5000AC6AC2F2000A0BEB0A044FF00201F9F79B
:10FB600089FD42F68F73C2F200031D70C4F8306243
:10FB7000304604F5097104F50D7204F50E73FFF7B4
:10FB8000BBFC2846FFF7EAFCF5F7D8FFC4F82802CB
:10FB90004FF00100009048F66860C0F601004FF099
:10FBA00004014FF69562C0F600022B46F5F702FB02
:10FBB000C4F81C025BF80A40F27848F6E851C0F637
:10FBC000010151F8221019F808207B78BE780096C0
:10FBD0004FF0000001904FF62D16C0F60006029679
:10FBE0004FF66916C0F6000603964FF6A516C0F646
:10FBF000000604964FF61136C0F6000605960690EC
:10FC000064682846A04709B0BDE8F08F08B542F601
:10FC10009073C2F2000318604FF00100FFF726FF57
:10FC200008BD00BF42F68E73C2F200034FF000021F
:10FC30001A70704708B542F69073C2F20003186854
:10FC400068B142F68F71C2F200010A78032A09D81E
:10FC50004FF00000FFF70AFF4FF0000008BD4FF023
:10FC6000480008BD4FF0480008BD00BF10B4D0F8F0
:10FC70000031032B20D94278102A20D890F9014076
:10FC80004FF0010101FA04F448F2600261F31F42EF
:10FC900014420CD114F00E0F11D0052B12D980781C
:10FCA00000F10500834214BF002001200CE0082B66
:10FCB00014BF0020012007E04FF0000004E04FF0E7
:10FCC000010001E04FF0000010BC7047072814D875
:10FCD00040B24FF0010303FA00F111F00A0F0FD107
:10FCE00011F0050F03D111F0F00F03D105E04FF033
:10FCF000010070474FF0040070474FF0000070475C
:10FD00004FF00200704700BF2DE9F04F83B0054669
:10FD10000E4617461C464FF0000001460246F4F717
:10FD20003FFC83463846FFF7D1FF8046002800F0AD
:10FD3000A980042805D04FF00100002E00F0A78014
:10FD400003E016F0010FF6D09FE0A7F1040A40F699
:10FD50006C53C2F200030193BAF1030F04D8019A65
:10FD6000A858F7F747FA8146072F00F28280DFE8AC
:10FD700007F0042416364C5E676FB5F5FA6F08D9A4
:10FD80000BEB0502A2F5FA6108784FEA0023238005
:10FD90006FE00199685C4FEA0023238069E0B5F5C4
:10FDA000FA6F06D90BEB0502A2F5FA610B782380F6
:10FDB0005FE0019BE85C20805BE0B5F5FA6F0AD953
:10FDC000A5F5FA618B449BF801009BF8003043EAEB
:10FDD000002222804DE001982A5A228049E0B5F5A0
:10FDE000FA6F0AD9A5F5FA639B449BF800009BF8CB
:10FDF000012042EA002121803BE0019BE85A4FEAC2
:10FE0000102242EA0021218033E04FEA19434FEAF1
:10FE1000132040EA0321234623F8021B1FFA89F22C
:10FE20004FEA122040EA022161801C4621E0C9F31A
:10FE30000F41224622F8021BA4F80290144618E053
:10FE4000234623F8029BC9F30F4060801C4610E054
:10FE50001FFA89F04FEA102141EA0022234623F8D5
:10FE6000022B4FEA19404FEA102141EA002262803A
:10FE70001C46454404F10204013E7FF46DAF4FF08F
:10FE8000010004E04FF0000001E04FF0000003B07B
:10FE9000BDE8F08F2DE9F04F8BB05FFA80FB40F6A4
:10FEA000AC63C2F200034FF4117404FB0B344FF047
:10FEB00000054FF4117000FB0BF1019101F58876FC
:10FEC00040F6AC62C2F200020392B71804970BE04E
:10FED0002668B36958464FF0000198474FF001007B
:10FEE000C4F84002F4F7E8FF42F68E73C2F2000352
:10FEF00018780028ECD042F69071C2F200010E682A
:10FF0000002EE5D04FF00002C4F84022DDF80CA02E
:10FF1000DDF8109060E3D4F83C0240B14FF00005EA
:10FF2000C4F83C5242F69071C2F200010D682E787E
:10FF3000062E00F0A4800CD8032E1CD003D8002E6F
:10FF400000F0AB811AE0042E42D0052E40F0A581CE
:10FF500067E0802E00F07F8106D80F2E00F0C08071
:10FF6000102E40F09A812DE1812E00F08D81822E9D
:10FF700040F093817EE14FF008062BE02A79B5F836
:10FF8000057002F1FF33B3F5FA6F19D24FEA17206B
:10FF900040EA072113FA81F6B6F5FB6F13D2019FF1
:10FFA00007EB0A0101F10403687808712E785E708E
:10FFB0006F885F804FEA02229A804FF0060104E0CA
:10FFC0004FF0FF3101E04FF0FF314FF007065FE1E6
:10FFD0004FF007062F79B5F8051007F1FF327C2A9C
:10FFE00019D84FEA112040EA012312FA83F1FA29C5
:10FFF00014D8DDF8048008EB0A0202F104036878E3
:020000040801F1
:100000001071297859706A885A804FEA07279F80B3
:100010004FF006013CE14FF0FF3139E14FF0FF3185
:1000200036E1A9884FEA112343EA012087B24FEA5B
:10003000D702FA2A1ED8019E06EB0A0303F1040137
:10004000687818712E784E706B884B8007F0070720
:100050004FF0010000FA07F040F66C56C2F20006BD
:10006000B25C0240002A14BFFF2300238B804FF0B4
:10007000060101E04FF0FF314FF0060608E1A879D4
:10008000FFF724FEAB88024610B34FEA132141EA82
:10009000032080B200F1FF37BE18FA2E1BD8DDF81E
:1000A00004C00CEB0A0202F10403697811712F7885
:1000B0005F706E885E804FF00101AA7903F104033E
:1000C000FFF722FE002814BF06214FF0FF3104E0A5
:1000D0004FF0FF3101E04FF0FF314FF00706D7E05E
:1000E0002A791646B5F8053002F1FF30B0F5F66F03
:1000F00060D24FEA132141EA0327B9B24FEAD10394
:100100001818FA2859D8019F07EB0A0808F1040CBF
:10011000687888F804002F788CF801706888ACF84B
:1001200002004FEA0227ACF8047002F107004FEA20
:10013000D0078CF8067008F10B00002A35D001F0CA
:1001400007014FF0010202FA01F7079740F66C57DA
:10015000C2F20007964606F1FF3111400591029266
:10016000002A00F0C182BBE2A846029E01E0A84638
:10017000029E012A04BF00250570FD5C0D4202D0DD
:100180000578154305704FEA4101802984BF01338A
:1001900071464FEA4202802A84BF0130724606F15E
:1001A000FF35012A40F0E082DBE29CF8061001F105
:1001B000070104E04FF0FF3101E04FF0FF314FF055
:1001C000070665E0E879FFF781FD2979B5F8056054
:1001D00001F1FF337A2B2DD878B34FEA162242EA89
:1001E0000627BAB202F1FF3601FB0063FA2B05D9EC
:1001F000A2F5FA67262F23D8022824D8019800EB0D
:100200000A0303F104066F781F71287858716F880C
:10021000DF804FEA012018814FEA41079F721046A4
:10022000EA7903F10B03FFF76FFD78B1B17901F1C2
:1002300007010DE04FF0FF310AE04FF0FF3107E01A
:100240004FF0FF3104E04FF0FF3101E04FF0FF319C
:100250004FF008061CE0B5F801104FEA112242EAFF
:10026000012042F61873C2F200031F6817FA80F6E5
:10027000771BBAE16B784FF0320000FB03F0F4F724
:10028000E3FF4FF00207B0E16FF001014FF001060C
:10029000AE19B1F1FF3F0ED100E02E464FF0000342
:1002A00042F69072C2F20002136042F68E77C2F2FA
:1002B00000073B708FE1002940F383815846FFF728
:1002C00061F92068826958464FF00001904794F820
:1002D0003872002F00F07F8107F1FF3E0EF0010819
:1002E000D4F83402F4F7B0FF002840F0DA8106E0D9
:1002F000D4F83402F4F7A8FF002840F0568199F8AA
:1003000000006B78984240F0668199F801202978C6
:100310008A4240F0608141F2C070C2F200004FF0AA
:100320000001F4F79BFB2F7807F1FF30032800F260
:100330003581DFE800F00202595995F804E099F898
:1003400002700EF10702B7EBD20F40F02781B5F82B
:1003500005504FEA152040EA05239FB207F0070237
:100360004FF0010101FA02F14FEAD703BEF1000F8D
:1003700000F014814FF0010040F66C52C2F200020E
:1003800007460EF1FF3C0CEA000C4FF0000599F80F
:10039000038018EA000F00F02A812FE109EB05081D
:1003A00098F803C01CEA000F12F8038014BF41EA5A
:1003B000080828EA010802F803804FEA4000802874
:1003C00084BF013538464FEA4101802984BF01339B
:1003D00039460EF1FF3E09EB050C9CF8038018EA44
:1003E000000F00F0408145E199F802202B79B2EB33
:1003F000430F40F0D380E979072900F2CF8095F9C7
:1004000007704FF0010000FA07F313F00A0F16D13E
:1004100013F0050F03D113F0F00F09D1BEE04FF038
:10042000020ECDF808E04FF00108CDF814800CE082
:100430004FF0040CCDF808C0CDF814C005E04FF023
:10044000020CCDF808C0CDF814C0B5F805004FEA8D
:10045000102343EA00211FFA81F8002A00F09E8051
:100460004FF0000740F66C52C2F200020792CDF83E
:1004700020B00994DDF818B01446E87907287AD836
:10048000DFE800F004140D1D2844536209EB470017
:10049000B0F803204FEA122308F804306BE009EBB0
:1004A0004703B3F8031008F8041064E009EB4700B1
:1004B000C278037942EA032128F804105BE009EBD3
:1004C0004703B3F803104FEA112242EA012028F84B
:1004D000040050E009EB4703B3F8031007F10107EC
:1004E0004FEA112242EA012060F31F4B09EB470358
:1004F000B3F803104FEA112242EA012060F30F0B18
:100500005846F6F74DFE48F8040034E009EB47037F
:10051000B3F8031061F31F4B07F1010709EB470222
:10052000B2F8030060F30F0BEAE709EB4703B3F8F7
:10053000031061F30F0B07F1010709EB4702B2F853
:10054000030060F31F4BDBE709EB4703B3F803102D
:1005500007F101074FEA112242EA012060F30F0B75
:1005600009EB4703B3F803104FEA112242EA0120D6
:1005700060F31F4BC4E70599884407F1010799F818
:1005800002200298131AD9B289F8021000297FF4C8
:1005900074AF099CCDF818B0DDF820B041F2C070FE
:1005A000C2F20000F4F768FB15E007F1FF3202F039
:1005B000FF07D4F83402F4F747FE002840F08980A2
:1005C0009DE611F1020F06D142F68E75C2F20005CA
:1005D0004FF000032B70354642F68E77C2F20007CB
:1005E0003B78002B7FF497AC7EE4EE19F3E712F82A
:1005F000038028EA010802F8038005E012F803806E
:1006000041EA080802F803804FEA40004FEA41013E
:10061000802984BF01333946BEF1010EBED0BCF142
:10062000000F3FF4BBAE09EB050C9CF8038018EA01
:10063000000F12F803C00CBF2CEA010C41EA0C0CAD
:1006400002F803C04FEA4000802884BF01353846D5
:100650004FEA4101802984BF01333946BEF1010EC2
:100660007FF49CAE9AE712F803C02CEA010802F866
:10067000038005E012F803C041EA0C0802F8038089
:100680004FEA4000802884BF013538464FEA4101D7
:10069000802984BF01333946BEF1010E7FF47EAE5E
:1006A0007CE707F1FF3111F0FF0794D04FFA88F390
:1006B000002B3FF41DAED4F83402F4F7C5FD00283A
:1006C0003FF41DAE07F1FF3010F0FF077FF410AECE
:1006D00081E707F1FF3111F0FF077FF409AE7AE7F8
:1006E0004FF0000288F80B20FA5C07990A4205D007
:1006F00098F80B2002990A4388F80B2007994FEAD3
:100700004101802984BF01337146DDF808804FEA3A
:100710004802013E02963FF448AD059E002E3FF48C
:1007200023AD012A04BF0026067017F8038018EADB
:10073000010F04D0067842EA060880F800804FEAEC
:100740004101802984BF013371464FEA4202802A69
:1007500084BF01307246029E013E02967FF407ADCF
:1007600023E54FF000060670FE5C0E4202D00678CC
:10077000164306704FEA4101802984BF0133714658
:100780004FEA4202802A84BF013072466E1E7FF417
:10079000F0AC454609E500BF38B540F6AC65C2F29D
:1007A00000054FF4117404FB005505F10404297190
:1007B00062F07F026A71AB714FF00301FEF7E2FE57
:1007C00038BD00BF2DE9F04F89B05FFA80FA40F6DE
:1007D000AC63C2F200034FF4117404FB0A344FF40B
:1007E000117000FB0AF1029101F5887540F6AC62C8
:1007F000C2F20002039205EB020B2668B76950466D
:100800004FF00001B847F4F757FBD4F81002D4F8C2
:1008100014329842F1D094F81011D4F83452A9420D
:1008200040F00A8341F2C070C2F200004FF00001B4
:10083000F4F714F994F8112102F1FF360F2E00F2AB
:10084000EE82DFE816F010009E000F01EC02780146
:10085000C801EC02EC02EC02EC02EC02EC02EC024D
:10086000EC02FB016B02BBF80260BBF804504FEADC
:10087000152343EA052087B207F1FF32B2F5FA6F7C
:1008800009D350469BF800109BF801204FF003035A
:10089000FFF782FFCAE24FEA162141EA0626B5B207
:1008A000504629463A464FF00003FEF7B7FF48B9D5
:1008B00050469BF800109BF801204FF00203FFF711
:1008C0006BFFB3E2029B0398191801F10402019235
:1008D0009BF800600E719BF80130019843704FF057
:1008E0000008002F44D006E04FF001064FF0000949
:1008F00005F101050BE04FF000084FF00106C1467D
:1009000040F66C51C2F20001059104940C4640F28D
:10091000E73295420CD84FEAD500225C05F0070378
:1009200042FA03F111F0010F0ED049EA06090BE07B
:1009300005F11803D8B207A9F8F710F99DF81C10B3
:1009400011B908B149EA060907F1FF374FEA46062F
:10095000802E03D8002F00F08B82C9E7019A02EBAA
:10096000080383F8039008F10108002FBCD1049C10
:10097000019981F80280504608F10301FEF702FE5A
:1009800054E2BBF80250BBF804204FEA122646EAB4
:100990000227BEB206F1FF31B1F5FA6F09D3504616
:1009A0009BF800109BF801204FF00303FFF7F4FEC3
:1009B0003CE24FEA152343EA052085B2E8B207A9D5
:1009C000F8F734F89DF81C204AB150469BF8001007
:1009D0009BF801204FF00203FFF7DEFE26E2029FA4
:1009E00003997B1803F1040001909BF800201A7111
:1009F0009BF80170477056B3AFB24FF000084FF04C
:100A00000105C14605E04FF001054FF0000907F16F
:100A10000107F8B207A9F8F709F89DF81C1011B9F9
:100A200008B149EA050906F1FF364FEA4505802D70
:100A300003D8002E00F02582E9E7019A02EB0801B5
:100A400081F8039008F10108002EDCD101E04FF09D
:100A50000008019F87F80280504608F10301FEF765
:100A600091FDE3E1BBF802304FEA132646EA03208A
:100A700080B20790BBF804704FEA172242EA0725BC
:100A8000AEB206F1FF317C2909D950469BF800101F
:100A90009BF801204FF00303FFF77EFEC6E13146CD
:100AA000FEF70CFE48B150469BF800109BF8012061
:100AB0004FF00203FFF770FEB8E1029B03981D1888
:100AC00005F104079BF800202A719BF8011079704A
:100AD0003EB34FF0000806F1FF3303F0010907A809
:100AE0004146FEF795FDA7F803004FF00105AE4221
:100AF00040F0CF8115E007A84146FEF789FD07EBDE
:100B00004501A1F8030005F1010507A84146FEF7DC
:100B10007FFD07EB4503A3F8030005F10105AE4295
:100B2000E9D14FEA4600C1B2B970504601F1030164
:100B3000FEF728FD7AE1BBF80220BBF804504FEA2B
:100B4000152646EA0527BDB265B1B5F57F4F09D038
:100B500050469BF800109BF801204FF00303FFF76D
:100B60001BFE63E14FEA122141EA02239EB2504686
:100B700031464FF001021346FEF750FE48B9504689
:100B80009BF800109BF801204FF00203FFF704FED2
:100B90004CE10298039900EB01093046B5F57F4F0F
:100BA00014BF00210121FEF781FE9BF8002089F887
:100BB00004209BF8017089F80570BBF80250A9F871
:100BC0000650BBF80410A9F8081050464FF0060173
:100BD000FEF7D8FC2AE1BBF802604FEA162747EA85
:100BE00006218BB208A941F8043D5046BBF8042009
:100BF0004FF00003FEF786FD48B950469BF8001001
:100C00009BF801204FF00203FFF7C6FD0EE10298AA
:100C1000039A851805F104069BF800702F719BF864
:100C200001107170BBF802307380BBF80400B08013
:100C300050464FF00601FEF7A5FCF7E0BBF80200B6
:100C4000BBF804704FEA172646EA072295B205F171
:100C5000FF31B1F5FA6F06D29BF8063005F10707B0
:100C6000B3EBD70F09D050469BF800109BF801203A
:100C70004FF00303FFF790FDD8E04FEA102646EA55
:100C800000201FFA80F8504641462A464FF00103E3
:100C9000FEF7C4FD18B1002D40F0D28027E0504689
:100CA0009BF800109BF801204FF00203FFF774FD42
:100CB000BCE00BEB0700C17930462940FEF7F6FD9A
:100CC0004FEA4505802D84BF0137454606F10106F0
:100CD00030460BEB0702D1792940FEF7E7FD4FEADA
:100CE0004505802D00F2F780F8E04E45E1D1029DE8
:100CF00003982A1802F104069BF8007017719BF8FC
:100D000001107170BBF802307380BBF80450B580DD
:100D100050464FF00601FEF735FC87E0BBF8027045
:100D20004FEA172242EA072083B20693BBF8045029
:100D30004FEA152141EA0526B5B25F1907F1FF32E6
:100D4000079205F1FF307C2809D950469BF8001026
:100D50009BF801204FF00303FFF71EFD66E05046AD
:100D600006A94FF000024FF00103FEF7CBFC50B193
:100D7000504607A94FF000024FF00103FEF7C2FCF6
:100D800008B155B934E050469BF800109BF801209B
:100D90004FF00203FFF700FD48E04FF0000705F1B8
:100DA000FF3808F00109504606A9BBF807203B466A
:100DB000FEF7A8FC4FF00106B54240F0928017E024
:100DC0000BEB4602504606A9B2F807203B46FEF759
:100DD00099FC06F101060BEB4603504606A9B3F851
:100DE00007203B46FEF78EFC06F10106B542E7D12F
:100DF000029D03982F1807F104069BF800203A7112
:100E00009BF801107170BBF802307380BBF804507E
:100E1000B58050464FF00601FEF7B4FB06E05046A1
:100E200094F810114FF00103FFF7B6FC41F2C070C7
:100E3000C2F20000F3F720FF5046FEF78FFBDCE420
:100E40009BF80720404602F00101FEF72FFD08F154
:100E5000010608EB05094FF002054FF000074FF0BF
:100E60000108C6EB090111F0010F3FF43EAF22E08B
:100E7000049C019D05EB080080F8039008F101082F
:100E800076E5019B03EB080080F8039008F1010868
:100E9000DFE5B9F1000F3FF42EAE07A84146FEF79B
:100EA000B7FB07EB4502A2F8030005F10105AE42CE
:100EB0007FF421AE35E60BEB0703D97930462940A4
:100EC000FEF7F4FC4FEA4505802D84BF0137454607
:100ED00006F1010609E707F10107454606F101069B
:100EE00003E7B9F1000F3FF46BAF0BEB460350463D
:100EF00006A9B3F807203B46FEF704FC06F10106FD
:100F0000B5427FF45DAF73E740F6AC63C2F2000315
:100F10004FF4117202FB003393F82032012B0AD1F7
:100F200040F6AC63C2F2000302FB0030C0F834129A
:100F30004FF0000070474FF0370070472DE9F04F39
:100F400089B004460D4691F8029009EB490947F62D
:100F50009048C0F6010809EB08074FF4117B0BFB22
:100F600000FB40F6AC6AC2F2000A0BEB0A064FF037
:100F70000101F8F77FFBC6F83052284606F50971E3
:100F80004FF000021346FEF7B7FA20466978FFF7E4
:100F9000BBFF2046FEF7E2FAF4F7D0FDC6F82802C0
:100FA0004FF00103009348F67860C0F601004FF05F
:100FB000040140F2C572C0F601022346F4F7FAF8C4
:100FC000C6F81C025BF80A60EA7848F6E850C0F6FA
:100FD000010050F8221019F808207B78BD780095A0
:100FE0004FF0000001904FF62D15C0F60005029558
:100FF0004FF66915C0F6000503954FF6A515C0F626
:10100000000504954FF60915C0F6000505950690F4
:1010100075682046A84709B0BDE8F08FD0F80031C8
:10102000032B2BD94278102A2BD890F901204FF0AE
:10103000010101FA02F212F06E0F06D112F4803FA4
:1010400012D112F4004F05D11BE0082B14BF002071
:1010500001207047092B17D9807900F109008342DC
:1010600014BF002001207047092B10D9807900F1AE
:101070000900834214BF0020012070474FF0000098
:1010800070474FF0010070474FF0000070474FF07D
:101090000000704742F6D173C2F200031A78027062
:1010A00042F6C870C2F2000003780B70704700BFB0
:1010B00042F6D173C2F200031A78831A12D442F6B0
:1010C000C870C2F20000027893420EDA4FF00100BD
:1010D00000FA03F342F6CC72C2F200021268134027
:1010E0000B7070474FF0000070474FF000007047E2
:1010F00008B52DED028BB0EE408A42F6D073C2F2F5
:1011000000031878C0B94FF00000F0F72BFE00EE96
:10111000100AB4EEC80AF1EE10FA0ED988EE000AF1
:10112000F7EE007AB4EE670AF1EE10FAB0EE678AD5
:10113000C8BFB0EE670A02E001E0B7EE000ABDECFE
:10114000028B08BD08B542F6FC73C2F200031978A1
:101150004018C0B210EE101AF0F70CFD08BD00BF29
:1011600010B542F6D173C2F200031A78841A4DD436
:1011700042F6C870C2F2000003789C4249DA4FF090
:10118000010303FA04F3E1B142F6CC71C2F20001AB
:101190000A68134240D142F6BC71C2F200010868ED
:1011A00018430860134342F6CC72C2F20002136087
:1011B00042F6D473C2F2000393ED000AFFF798FFE2
:1011C0001EE042F6CC71C2F200010A68134226D03A
:1011D0006FEA030342F6BC71C2F2000108681840CE
:1011E000086042F6C071C2F2000108681840086049
:1011F000134042F6CC72C2F2000213609FED090A5E
:101200002046FFF79FFF4FF0010010BD4FF0000098
:1012100010BD4FF0000010BD4FF0010010BD4FF0A9
:10122000010010BD0000000070B52DED028B42F6EC
:10123000C073C2F200031C68C4B142F69470C2F2DB
:10124000000090ED008A4FF000054FF001062642A5
:1012500004D02846B0EE480AFFF774FF4FEA46066E
:1012600005F101052846264214D00FE042F6BC7372
:10127000C2F200031A6842F6C071C2F200010A60AD
:101280004FF000001860BDEC028B70BDB0EE480A54
:10129000FFF758FF4FEA460605F10105202DD6D18C
:1012A000E4E700BF000000002DE9F8432DED028BBC
:1012B00042F6C473C2F2000393ED000AFFF718FF71
:1012C000B0EE408A42F69470C2F20000D0ED007A8F
:1012D00037EEC00A10EE100A02F026FD02F0E4F824
:1012E00023A3D3E9002302F073FC00283CD142F68B
:1012F0009471C2F2000181ED008A42F6CC72C2F212
:101300000002136883B342F6C870C2F2000001788D
:1013100051B34FF001044FF0000542F6CC77C2F212
:10132000000742F6C079C2F2000942F6BC78C2F268
:10133000000842F6C876C2F200063A6814420CD0A1
:10134000D9F80000D8F8003040EA03010C4204D17B
:101350002846B0EE480AFFF7F5FE05F101054FEA11
:1013600044043278AA42E8DCBDEC028BBDE8F88385
:101370007B14AE47E17A943F70B582B005461646BD
:101380009DF8184042F6D072C2F20002107042F688
:10139000D470C2F20000016042F6C471C2F20001D2
:1013A0000E60A34242F6FC72C2F2000292BF1370BA
:1013B00014701C4642F6D173C2F200039DF81C0063
:1013C000187042F6FC71C2F200010A78C2F1010302
:1013D000E418E4B242F6C870C2F200000470202C97
:1013E00001D9EFF72BF940F2C810C2F200004FF01C
:1013F0000101F7F78BFA4FF0000100914FF0010265
:10140000019242F69870C2F200004FF0FA014FF0DC
:10141000060241F22923C0F60103F4F759FBBDB9D6
:101420004FF0000400944FF00100019042F6D87094
:10143000C2F2000040F6C4114FF0060241F2A923A7
:10144000C0F60103F4F744FB2046FFF72DFF04E04C
:1014500042F69473C2F200031E6002B070BD00BF7A
:1014600043F20003C2F200031A7802705878087041
:10147000704700BF43F20003C2F200031B788342AF
:101480001AD843F20002C2F2000252789A1890422F
:1014900015DAC01AC3B24FEAD30243F21400C2F203
:1014A0000000825C03F0070342FA03F000F001023F
:1014B0000A704FF0010070474FF0000070474FF086
:1014C0000000704770B443F20003C2F200031B78BF
:1014D00083424DD843F20002C2F2000252789A18B9
:1014E000904248DAC01AC0B200F007054FF001047C
:1014F00004FA05F540F22072C2F2000252E8003F01
:1015000003F1010342E80036012EF7D043F2140341
:10151000C2F2000303EBD00393F8200028420CBF73
:1015200000200120087093F8201021EA050583F8B7
:10153000205052E8003FA3F1010342E80035012D9D
:10154000F7D052E8003FB3F1004F0DD14FF0000348
:1015500042E80035012DF4D04EF60450CEF20000E2
:10156000016841F080510160BFF32F8F204604E0F5
:101570004FF0000001E04FF0000070BC704700BF6A
:1015800043F20003C2F200031A790270587908701E
:10159000704700BF43F20003C2F200039A78027062
:1015A000D8780870704700BF10B443F20003C2F24D
:1015B00000039B78834237D843F20002C2F2000254
:1015C000D2789A18904232DAC01AC3B24FEAD304E2
:1015D00003F007004FF0010202FA00F359B143F2A1
:1015E0001401C2F20001081990F8402043EA0201F8
:1015F00080F840100AE043F21401C2F20001081919
:1016000090F8402022EA030280F8402043F21400C0
:10161000C2F20000021992F8601021EA030382F876
:1016200060304FF0010004E04FF0000001E04FF0A7
:10163000000010BC704700BF43F20003C2F2000379
:101640009B7883421BD843F20002C2F20002D27898
:101650009A18904216DAC01AC3B243F21402C2F2C8
:10166000000202EBD30090F8402003F0070342FA97
:1016700003F000F001020A704FF0010070474FF0D4
:10168000000070474FF00000704700BF10B443F2F5
:101690000003C2F200039B78834237D843F2000272
:1016A000C2F20002D2789A18904232DAC01AC3B25B
:1016B0004FEAD30403F007004FF0010202FA00F3EF
:1016C00059B143F21401C2F20001081990F86020E8
:1016D00043EA020180F860100AE043F21401C2F20A
:1016E0000001081990F8602022EA030280F86020C7
:1016F00043F21400C2F20000021992F8401021EAED
:10170000030382F840304FF0010004E04FF0000086
:1017100001E04FF0000010BC704700BF43F200032F
:10172000C2F200039A790270D8790870704700BF3E
:10173000827802F107024FEAE2014FEA410202F128
:101740000102037902EB8301407A0818704700BF59
:1017500070B401F0070400EBD10000F1FF31C4F1D7
:10176000080611F8010F40FA04F00CB9C0B204E009
:101770004D7805FA06F52843C0B2082B08D8C3F106
:1017800008034FF0FF0141FA03F31840107005E021
:1017900002F8010BA3F10803DBB2E2E770BC70476B
:1017A0002DE9F00F9DF82070044618B948F6AC6496
:1017B000C0F6010402F0070C66464FF0FF0000FA85
:1017C0000CF5E8B201EBD20101F1FF31CCF10809CF
:1017D00048F6AC68C0F601084A786FB9082B09D8FA
:1017E0004FF0010000FA03F000F1FF3505FA06F5AD
:1017F00005F0FF0022EA0002C5B294F800A00AFA40
:1018000006FA05EA0A0A4AEA020201F101018A46D9
:101810000A70BCF1000F0DD04B450BDD4A7807B9BB
:10182000024094F800B04BFA09FB2BEA05052A4365
:101830008AF80120082B06D9444518BF0134A3F1CA
:101840000803DBB2C8E7BDE8F00F704708B50448ED
:101850004FF000014FF0400202F0E6FF08BD00BF6C
:10186000B431002008B504484FF000014FF02002C9
:1018700002F0DAFF08BD00BF3430002010B54FF091
:10188000000443F20C03C2F200031C6043F2140094
:10189000C2F2000021464FF4007202F0C5FF43F28D
:1018A0000000C2F2000021464FF0080202F0BCFF27
:1018B00010BD00BF10B50C4643F20003C2F2000396
:1018C0009979814217D843F20002C2F20002D3791B
:1018D000CA18904212DA401AC1B201F1680143F20B
:1018E0001403C2F2000353F82100F5F783FC2060D3
:1018F0004FF0010010BD4FF0000010BD4FF0000090
:1019000010BD00BF10B50C4643F20003C2F2000345
:101910001979814217D843F20002C2F200025379CA
:10192000CA18904212DA401AC1B201F1280143F2FA
:101930001403C2F2000353F82100F5F75BFC2060AA
:101940004FF0010010BD4FF0000010BD4FF000003F
:1019500010BD00BF38B5054643F20003C2F20003D4
:101960009C79844217D843F20000C2F20000C27989
:10197000A3189D4212DA0846F5F712FC2C1BE4B2BC
:1019800004F1680443F21401C2F2000141F824009A
:101990004FF0010038BD4FF0000038BD4FF000009F
:1019A00038BD00BF2DE9F0418AB00446FFF766FF5D
:1019B00002A84FF000014FF0200202F035FF4FF077
:1019C000000001A9F6F700FF43F20003C2F2000392
:1019D0009DF804201A709DF8050098709DF8061077
:1019E00019719DF807509D714FF000064FF00108E6
:1019F00043F20C07C2F200071D464AE06078FF2858
:101A000045D14FEA531203F01F0108FA01F3386879
:101A100008B93C6008E0D8B20DF1280C0CEB82014B
:101A200051F8201C08422FD106F101060AA800EB4C
:101A30008202DBB252F8201C43EA010042F8200C7B
:101A40002046FFF775FE402871D8E37803F10702BE
:101A50004FEAE2014FEA410000F10100627900EB38
:101A60008200E1794218402A64D8A0786978421847
:101A70006A70E8781B18EB7021796A7988186871A8
:101A80006179EB79CA18EA7104F10A0401E004F102
:101A900005042378FF2BB1D1102E4ED843F2000459
:101AA000C2F200046279402A4AD843F20000C2F22E
:101AB0000000C179102946D843F20003C2F20003A6
:101AC0005C783CB140F2E810C2F200004FF0010136
:101AD000F6F7F0FE43F20002C2F20002D07838B10D
:101AE00040F2E010C2F200004FF00101F6F70EFFE5
:101AF00043F20001C2F200014B793BB140F2D01039
:101B0000C2F200004FF00101F6F72CFF43F200048F
:101B1000C2F20004E279DAB140F2D810C2F2000059
:101B20004FF00101F6F74AFF4FF0000412E04FF0CA
:101B300045040AE04FF0430407E04FF0460404E098
:101B40004FF00F0401E04FF00E04FFF797FE01E0A5
:101B50004FF0000420460AB0BDE8F08108B540F21D
:101B6000E810C2F200004FF00001F6F7A3FE40F2C9
:101B7000E010C2F200004FF00001F6F7C7FE40F29D
:101B8000D010C2F200004FF00001F6F7EBFE40F279
:101B9000D810C2F200004FF00001F6F70FFF08BDA9
:101BA0002DE9F843044643F20C03C2F2000318681F
:101BB00084421AD14FF0000542F6FD76C2F20006CB
:101BC000357043F20803C2F200031D7043F21100A6
:101BD000C2F20000057042F6FE76C2F200063570D1
:101BE00043F21003C2F200031D70E57805F107050A
:101BF0004FEAE505E8B2667900EB860303F10103DD
:101C0000C018C6B296423ED843F21408C2F2000889
:101C100042F6FD72C2F20002177808EB070393F850
:101C2000E0010F4607F8010B43F21101C2F2000177
:101C300091F8009008F1400049463A46E378FFF7F2
:101C400087FDEDB27F1908F1600049463A46E37816
:101C5000FFF77EFD7A196379BBB143F21005C2F23A
:101C60000005297808EB81004FF000031946C518DC
